:020000040800F2
:100000000080002055260008491500084B150008FF
:100010004D1500084F15000851150008000000009C
:100020000000000000000000000000005315000860
:100030005515000800000000571500085915000864
:10004000A5260008A52600085D150008A5260008BD
:10005000A5260008A5260008691500086F150008E8
:10006000A5260008A5260008A5260008A526000844
:10007000A5260008A5260008A52600087515000875
:10008000A5260008A5260008A5260008A526000824
:1000900000000000A526000881150008A52600081C
:1000A000A5260008A5260008A5260008A526000804
:1000B000A5260008A5260008A5260008A5260008F4
:1000C000A5260008A5260008A5260008A5260008E4
:1000D000A526000889150008A5260008A526000801
:1000E000A5260008A526000895150008A5260008E5
:1000F000A52600080000000000000000A52600085A
:10010000A5260008A5260008A1150008A5260008B8
:10011000A5260008A5260008A5260008A526000893
:10012000A5260008A5260008A5260008A526000883
:08013000A5260008A526000821
:1001380010B5054C237833B9044B13B10448AFF319
:1001480000800123237010BD18010020000000006A
:10015800E0EF000808B5034B1BB103490348AFF3B0
:10016800008008BD000000001C010020E0EF00082E
:10017800034613F8012B002AFBD1181A01387047DF
:1001880081F0004102E000BF83F0004330B54FEA40
:1001980041044FEA430594EA050F08BF90EA020FAD
:1001A8001FBF54EA000C55EA020C7FEA645C7FEA40
:1001B800655C00F0E2804FEA5454D4EB5555B8BF63
:1001C8006D420CDD2C4480EA020281EA030382EAD4
:1001D800000083EA010180EA020281EA0303362D66
:1001E80088BF30BD11F0004F4FEA01314FF4801C39
:1001F8004CEA113102D0404261EB410113F0004F4B
:100208004FEA03334CEA133302D0524263EB430301
:1002180094EA050F00F0A780A4F10104D5F1200E9F
:100228000DDB02FA0EFC22FA05F2801841F10001FA
:1002380003FA0EF2801843FA05F359410EE0A5F1CE
:1002480020050EF1200E012A03FA0EFC28BF4CF0FF
:10025800020C43FA05F3C01851EBE37101F00045B5
:1002680007D54FF0000EDCF1000C7EEB00006EEBC2
:100278000101B1F5801F1BD3B1F5001F0CD349084C
:100288005FEA30004FEA3C0C04F101044FEA4452A3
:1002980012F5800F80F09A80BCF1004F08BF5FEA2A
:1002A800500C50F1000041EB045141EA050130BD0A
:1002B8005FEA4C0C404141EB0101013C28BFB1F51C
:1002C800801FE9D291F0000F04BF01460020B1FA67
:1002D80081F308BF2033A3F10B03B3F120020CDA3A
:1002E8000C3208DD02F1140CC2F10C0201FA0CF018
:1002F80021FA02F10CE002F11402D8BFC2F1200C7D
:1003080001FA02F120FA0CFCDCBF41EA0C01904032
:10031800E41AA2BF01EB0451294330BD6FEA04047B
:100328001F3C1CDA0C340EDC04F11404C4F1200266
:1003380020FA04F001FA02F340EA030021FA04F378
:1003480045EA030130BDC4F10C04C4F1200220FACF
:1003580002F001FA04F340EA0300294630BD21FA0D
:1003680004F0294630BD94F0000F83F4801306BFD3
:1003780081F480110134013D4EE77FEA645C18BFC7
:100388007FEA655C29D094EA050F08BF90EA020F5E
:1003980005D054EA000C04BF1946104630BD91EA56
:1003A800030F1EBF0021002030BD5FEA545C05D159
:1003B8004000494128BF41F0004130BD14F5800498
:1003C8003CBF01F5801130BD01F0004545F0FE410C
:1003D80041F470014FF0000030BD7FEA645C1ABF41
:1003E800194610467FEA655C1CBF0B46024650EA78
:1003F800013406BF52EA033591EA030F41F40021A4
:1004080030BD00BF90F0000F04BF0021704730B529
:100418004FF4806404F132044FF000054FF00001FE
:1004280050E700BF90F0000F04BF0021704730B5BF
:100438004FF4806404F1320410F0004548BF404294
:100448004FF000013EE700BF42004FEAE2014FEAE9
:1004580031014FEA02701FBF12F07F4393F07F4FC4
:1004680081F06051704732F07F4208BF704793F0C7
:100478007F4F04BF41F40021704730B54FF46074DA
:1004880001F0004521F000411CE700BF50EA0102DD
:1004980008BF704730B54FF000050AE050EA010286
:1004A80008BF704730B511F0004502D5404261EBF6
:1004B80041014FF4806404F132045FEA915C3FF437
:1004C800D8AE4FF003025FEADC0C18BF03325FEAD4
:1004D800DC0C18BF033202EBDC02C2F1200300FA85
:1004E80003FC20FA02F001FA03FE40EA0E0021FAAA
:1004F80002F11444BDE600BF4FF0FF3C06E000BF28
:100508004FF0010C02E000BF4FF0010C4DF804CD94
:100518004FEA410C7FEA6C5C4FEA430C18BF7FEA54
:100528006C5C1BD001B050EA410C0CBF52EA430C82
:1005380091EA030F02BF90EA020F0020704710F102
:10054800000F91EA030F58BF994208BF90422CBF91
:10055800D8176FEAE37040F0010070474FEA410C8A
:100568007FEA6C5C02D150EA013C07D14FEA430CA8
:100578007FEA6C5CD6D152EA033CD3D05DF8040B19
:10058800704700BF8446104662468C46194663464B
:1005980000E000BF01B5FFF7B7FF002848BF10F122
:1005A800000F01BD4DF808EDFFF7F4FF0CBF012067
:1005B80000205DF808FB00BF4DF808EDFFF7EAFFE3
:1005C80034BF012000205DF808FB00BF4DF808ED9E
:1005D800FFF7E0FF94BF012000205DF808FB00BF93
:1005E8004DF808EDFFF7CEFF94BF012000205DF81D
:1005F80008FB00BF4DF808EDFFF7C4FF34BF01202A
:1006080000205DF808FB00BF4FEA410212F5001216
:1006180015D211D56FF47873B3EB625212D94FEA41
:10062800C12343F0004343EA505311F0004F23FA2B
:1006380002F018BF404270474FF00000704750EA80
:10064800013005D111F0004008BF6FF0004070473D
:100658004FF00000704700BF80F0004002E000BF8C
:1006680081F0004142001FBF5FEA410392EA030F95
:100678007FEA226C7FEA236C6AD04FEA1262D2EBDF
:100688001363C1BFD218414048404140B8BF5B42E4
:10069800192B88BF704710F0004F40F4000020F07D
:1006A8007F4018BF404211F0004F41F4000121F093
:1006B8007F4118BF494292EA030F3FD0A2F10102DD
:1006C80041FA03FC10EB0C00C3F1200301FA03F11B
:1006D80000F0004302D5494260EB4000B0F5000F3E
:1006E80013D3B0F1807F06D340084FEA310102F1FD
:1006F8000102FE2A51D2B1F1004F40EBC25008BFAF
:1007080020F0010040EA03007047490040EB000078
:10071800013A28BFB0F5000FEDD2B0FA80FCACF179
:10072800080CB2EB0C0200FA0CF0AABF00EBC250A6
:1007380052421843BCBFD0401843704792F0000F94
:1007480081F4000106BF80F400000132013BB5E7E7
:100758004FEA41037FEA226C18BF7FEA236C21D05D
:1007680092EA030F04D092F0000F08BF08467047C2
:1007780090EA010F1CBF0020704712F07F4F04D190
:10078800400028BF40F00040704712F100723CBFA3
:1007980000F50000704700F0004343F0FE4040F4CD
:1007A800000070477FEA226216BF08467FEA23638B
:1007B8000146420206BF5FEA412390EA010F40F476
:1007C800800070474FF0000304E000BF10F00043C2
:1007D80048BF40425FEA000C08BF704743F09643A9
:1007E80001464FF000001CE050EA010208BF7047C4
:1007F8004FF000030AE000BF50EA010208BF70474B
:1008080011F0004302D5404261EB41015FEA010C5F
:1008180002BF84460146002043F0B64308BFA3F157
:100828008053A3F50003BCFA8CF2083AA3EBC25339
:1008380010DB01FA02FC634400FA02FCC2F1200258
:10084800BCF1004F20FA02F243EB020008BF20F08F
:100858000100704702F1200201FA02FCC2F12002F5
:1008680050EA4C0021FA02F243EB020008BF20EAEA
:10087800DC7070474FF0FF0C1CEAD0521EBF1CEA18
:10088800D15392EA0C0F93EA0C0F6FD01A4480EA06
:10089800010C400218BF5FEA41211ED04FF00063EF
:1008A80043EA501043EA5111A0FB01310CF000401B
:1008B800B1F5000F3EBF490041EAD3715B0040EA41
:1008C800010062F17F02FD2A1DD8B3F1004F40EB11
:1008D800C25008BF20F00100704790F0000F0CF0E4
:1008E800004C08BF49024CEA502040EA51207F3AA8
:1008F800C2BFD2F1FF0340EAC250704740F4000083
:100908004FF00003013A5DDC12F1190FDCBF00F073
:1009180000407047C2F10002410021FA02F1C2F121
:10092800200200FA02FC5FEA310040F1000053EABD
:100938004C0308BF20EADC70704792F0000F00F00B
:10094800004C02BF400010F4000F013AF9D040EA11
:100958000C0093F0000F01F0004C02BF490011F4A5
:10096800000F013BF9D041EA0C018FE70CEAD153A3
:1009780092EA0C0F18BF93EA0C0F0AD030F0004C23
:1009880018BF31F0004CD8D180EA010000F00040D7
:10099800704790F0000F17BF90F0004F084691F095
:1009A800000F91F0004F14D092EA0C0F01D14202CF
:1009B8000FD193EA0C0F03D14B0218BF084608D198
:1009C80080EA010000F0004040F0FE4040F40000E2
:1009D800704740F0FE4040F4400070474FF0FF0C75
:1009E8001CEAD0521EBF1CEAD15392EA0C0F93EABC
:1009F8000C0F69D0A2EB030280EA010C49024FEA0E
:100A0800402037D04FF0805343EA111143EA1013C6
:100A18000CF000408B4238BF5B0042F17D024FF47E
:100A2800000C8B4224BF5B1A40EA0C00B3EB510F59
:100A380024BFA3EB510340EA5C00B3EB910F24BF42
:100A4800A3EB910340EA9C00B3EBD10F24BFA3EBC7
:100A5800D10340EADC001B0118BF5FEA1C1CE0D18F
:100A6800FD2A3FF650AF8B4240EBC25008BF20F042
:100A7800010070470CF0004C4CEA50207F32C2BF96
:100A8800D2F1FF0340EAC250704740F400004FF033
:100A98000003013A37E792F0000F00F0004C02BF64
:100AA800400010F4000F013AF9D040EA0C0093F02E
:100AB800000F01F0004C02BF490011F4000F013B88
:100AC800F9D041EA0C0195E70CEAD15392EA0C0FF0
:100AD80008D142027FF47DAF93EA0C0F7FF470AF28
:100AE800084676E793EA0C0F04D14B023FF44CAF6B
:100AF80008466EE730F0004C18BF31F0004CCAD100
:100B080030F000427FF45CAF31F000437FF43CAF3B
:100B18005FE700BF4FEA4002B2F1FE4F0FD34FF03C
:100B28009E03B3EB12620DD94FEA002343F0004352
:100B380010F0004F23FA02F018BF404270474FF000
:100B48000000704712F1610F01D1420205D110F087
:100B5800004008BF6FF0004070474FF0000070473A
:100B680042000ED2B2F1FE4F0BD34FF09E03B3EB0F
:100B7800126209D44FEA002343F0004323FA02F03B
:100B880070474FF00000704712F1610F01D1420227
:100B980002D14FF0FF3070474FF00000704700BFA0
:100BA80053B94AB9002908BF00281CBF4FF0FF31CC
:100BB8004FF0FF3000F074B9ADF1080C6DE904CEC8
:100BC80000F006F8DDF804E0DDE9022304B0704720
:100BD8002DE9F047089E0D4604468846002B4DD166
:100BE8008A42944668D9B2FA82F252B101FA02F303
:100BF800C2F1200120FA01F10CFA02FC41EA0308D3
:100C080094404FEA1C45210CB8FBF5FE1FFA8CF7FF
:100C180005FB1E8341EA03430EFB07F199420BD9FA
:100C28001CEB03030EF1FF3080F01E81994240F265
:100C38001B81AEF1020E63445B1AA4B2B3FBF5F05C
:100C480005FB103344EA034400FB07F7A7420AD91F
:100C58001CEB040400F1FF3380F00881A74240F246
:100C6800058164440238E41B40EA0E4000211EB1AD
:100C7800D4400023C6E90043BDE8F0878B4208D979
:100C8800002E00F0EE800021C6E900050846BDE808
:100C9800F087B3FA83F100294AD1AB4202D38242EA
:100CA80000F2F980841A65EB030301209846002EB0
:100CB800E2D0C6E90048DFE702B9FFDEB2FA82F205
:100CC800002A40F09180A1EB0C054FEA1C471FFA5F
:100CD8008CFE0121B5FBF7F307FB1350250C45EA01
:100CE80000450EFB03F0A84208D91CEB050503F1EB
:100CF800FF3802D2A84200F2CB8043462D1AA4B294
:100D0800B5FBF7F007FB105544EA05440EFB00FE5F
:100D1800A64508D91CEB040400F1FF3502D2A6450C
:100D280000F2BB802846A4EB0E0440EA03409EE78D
:100D3800C1F120078B4022FA07FC4CEA030C20FA89
:100D480007F405FA01F31C43FD404FEA1C4900FA79
:100D580001F3B5FBF9F8200C1FFA8CFE09FB1855B6
:100D680040EA054508FB0EF0A84202FA01F20BD949
:100D78001CEB050508F1FF3A80F08880A84240F294
:100D88008580A8F1020865442D1AA4B2B5FBF9F0D4
:100D980009FB105544EA054500FB0EFEAE4508D98F
:100DA8001CEB050500F1FF346CD2AE456AD9023858
:100DB800654440EA0840A0FB0294A5EB0E05A54255
:100DC800C846A64656D353D05EB1B3EB080265EBCE
:100DD8000E0505FA07F722FA01F3CD401F43C6E9CD
:100DE80000750021BDE8F087C2F1200320FA03F165
:100DF8000CFA02FC25FA03F395400D434FEA1C4711
:100E08001FFA8CFEB3FBF7F107FB11302B0C43EAFA
:100E1800004301FB0EF0984204FA02F408D91CEBD7
:100E2800030301F1FF382FD298422DD902396344C8
:100E38001B1AADB2B3FBF7F007FB103345EA0345C5
:100E480000FB0EF3AB4208D91CEB050500F1FF3897
:100E580016D2AB4214D902386544ED1A40EA014172
:100E680038E73146304607E78646E5E61846FAE6AB
:100E78004B45A9D2B9EB020864EB0C0E0138A3E785
:100E88004046EAE7204694E74146D1E7D0467BE76B
:100E9800023B654432E7084609E76444023842E702
:100EA800704700BF1348144A08B54FF00043C0E923
:100EB80000230422002342610122C2614FF48051C1
:100EC80007220383C0E90233C0E90933C0E90C12E1
:100ED8000361837680F8203080F82C30826380F8B4
:100EE8003C30C36401F02EFC18B1BDE8084000F0A6
:100EF80089BA08BD34010020002401400268084B6B
:100F08009A4282B00AD14FF0B0431A6E42F400728E
:100F18001A661B6E03F400730193019B02B07047BD
:100F2800002401400268054B9A4201BF4FF0B042CD
:100F3800136E23F400731366704700BF002401404A
:100F480030B585B000240546CDE901440394FFF788
:100F5800A9FF144801F096FF08B100F053FA1148B0
:100F6800039401A9CDE9015401F058FD08B100F03E
:100F780049FA0C4801F0B8FE08B100F043FA4FF006
:100F8800FF31084801F0ECFC064801F05DFF054818
:100F980001F041FD0446034801F008FF204605B072
:100FA80030BD00BF34010020014B024A1A6070476F
:100FB800340100200024014008B50948FFF7C0FFAC
:100FC80068B1084BB3F8AA304FF6FF72934216BFC8
:100FD80040F6E442044B5343B3FBF0F080B208BD43
:100FE800002000B40075FF1FD8084C0013B500237B
:100FF800ADF80630FFF7E0FF04461948FFF7A0FFF9
:101008001849B1F8C820B1F8A8108A4204FB00F0CA
:1010180018D040F6E443B0FBF3F364205B1A434373
:10102800521A93FBF2F31E331BB2ADF80630BDF82B
:1010380006305BB21B02ADF80630BDF8060000B200
:1010480002B010BD40F6FF73B0FBF3F34FF47A70B3
:101058004343A3F53923A3F50C6340F6C412E0E734
:10106800001000B00075FF1F4FF0B04307B59A6C31
:1010780042F004029A649A6C02F004020192019A06
:101088009A6C42F001029A649B6C03F0010300938E
:10109800002202210F20009B01F092FF0F2003B0D5
:1010A8005DF804EB01F0BEBFF8B50B4F04461646D9
:1010B8001D46D4E90023AB4208BFB24201D100204B
:1010C800F8BD3B691B03FCD432462B462146012060
:1010D80002F044FAEDE700BF00400058F7B522F0EF
:1010E8000705044605440E1AAC4206EB040101D17B
:1010F800002015E0082268460DF09CFADDE900237F
:10110800B3F1FF3F08BFB2F1FF3F04F1080701D177
:101118003C46E9E72046FFF7C7FF3C460028E3D0F6
:1011280003B0F0BD1FB50223CDE9013003915AB1D8
:1011380001A802F0A7FA20B102280CBF01206FF025
:10114800010005B05DF804FB694601A802F04CFAFD
:10115800F1E700002DE9F74F9A46474BD3F8E075C1
:10116800464B00F1784603EA8727B6FBF7F307FBFF
:10117800136602F17843013B03449146B3FBF7F24F
:1011880007FB1233DB0A0546F60A0193884621B9A4
:101198006FF0040003B0BDE8F08F40EA09035B0775
:1011A800F6D1374B5B69002B5FDB019B9E421ABF70
:1011B800C0F30A03C3F500674F46019B9E4201D95D
:1011C8000020E7E72C4607EB050B14F00700ABEB14
:1011D80004020CD14FEAD20C60452FD1A2EBC00219
:1011E8002244A24236D13A464146284620E014F825
:1011F800012BFF2AE9D0BAF1000FC9D0F40204F19B
:1012080000644FF40062214650460DF013FAC5F30E
:101218000A00BAB2414650440DF00CFA00220121EE
:101228003046FFF77FFF18BB4FF400625146204657
:10123800FFF754FF98B16FF00200ABE754F8083B92
:1012480054F8041CB1F1FF3F08BFB3F1FF3FD2D1FE
:101258000130C1E714F8011BFF29C2D0CBE7B8441D
:101268000136A9EB07075D46A7E76FF0030091E792
:101278006FF001008EE700BF0070FF1F00FCFF0346
:10128800004000584FF0B04382B0DA6C0243DA6491
:10129800DB6C18400190019B02B070472DE9F041CA
:1012A80086B01422002101A80DF00CFE0220FFF7E1
:1012B800E9FF294E0420FFF7E5FF0120FFF7E2FFD1
:1012C8004FF43A410022304602F02EFB01254FF43C
:1012D8000A430024CDE9013501A902233046CDE9AE
:1012E80003434FF0030802F0FFF94FF4041701A974
:1012F8004FF09040CDE90187039502F0F5F94FF4DE
:10130800405301A93046CDE90135CDE9034802F043
:10131800EBF9402301A911480395CDE9013702F003
:10132800E3F922462146062001F04AFE062001F094
:1013380079FE22462146072001F042FE072001F0EF
:1013480071FE22462146162001F03AFE162001F0D1
:1013580069FE06B0BDE8F0810004004800080048B6
:1013680000B59BB04822002108A80DF0ABFD18225B
:10137800002102A80DF0A6FD02F0F0FA4FF0B042ED
:101388000120D2F8903023F01803C2F89030D2F838
:10139800003423F4C06343F40073C2F80034D2F875
:1013A800003403F4C0630193019B24230893812331
:1013B8000B930023CDE91003B02208A8CDE912232E
:1013C80002F04AFC08B172B6FEE74F23CDE90230BD
:1013D800CDE90400CDE90600022102A802F0DCFEF6
:1013E80008B172B6FEE71BB05DF804FB08B501F062
:1013F80057F9FFF7B5FFFFF751FF00F07BFC00F04E
:1014080080FCFCE772B6FEE700B58DB02C22002107
:1014180001A80DF057FD1748174B03601F23836081
:101428004FF080420023C0E90433C0E907238361F9
:101438004FF48073436203F061F908B1FFF7E2FFEC
:101448000C4803F083FA08B1FFF7DCFF4FF00053B4
:1014580000220793074808924FF4807301A902926B
:1014680006920B9303F0A6F908B1FFF7CBFF0DB076
:101478005DF804FB980100200028004010B50446E0
:1014880090B03822002102A80DF01CFD2268194BEB
:101498009A422CD14FF48033029302A84FF4807300
:1014A8000F9302F09BFF08B1FFF7ACFF4FF0B0437A
:1014B8000220D3F8902042F40042C3F890209A6D9D
:1014C80042F480629A659B6D002203F480631146A2
:1014D8000193019B01F074FD022001F0A3FD00229D
:1014E8002A20114601F06CFD2A2001F09BFD10B066
:1014F80010BD00BF002800407047000008B501F08B
:10150800E5F8044B0120C3F88800BDE8084002F064
:101518007DBA00BF0004005801F0DFB808B501F03B
:10152800DCF8BDE8084000F0A5BB08B501F0CEF82E
:10153800BDE808400121002002F018BA7047704742
:10154800FEE7FEE7FEE7FEE7FEE7704770477047F5
:1015580070470000014803F01FBA00BF980100203F
:10156800012002F0EFB9022002F0ECB9014801F0C5
:101578003BBF00BFE4010020402002F0E3B90000B7
:10158800014803F0CFBD00BF44020020014803F02A
:1015980037B800BF98010020014803F01CBC00BF09
:1015A800D0010020054808B50823036003F03AFA83
:1015B80018B1BDE80840FFF725BF08BDD0010020DD
:1015C8004FF0B04307B55A6E42F001025A665B6E9F
:1015D800002203F00103019311463220019B01F020
:1015E800EFFC322003B05DF804EB01F01BBD0000F6
:1015F8000CB407B5054A05AB102101930DF026FB85
:1016080003B05DF804EB02B0704700BF84F0000837
:1016180030B585B0044602A80D460DF041F9BDF974
:101628000C30064A00931021029B2046FFF7E0FF8A
:101638002046FEF79DFD288005B030BD84F00008E7
:101648004FF0B04210B5936823F4004393600DF057
:10165800AFF90E4B01241C7000F0A2F80CF078FED4
:101668000B480CF08FFE0B4B4FF400421A6102201E
:101678000CF08EFEFFF798FC00F0EEF80CF084FFFB
:1016880021462046BDE810400CF09EBFDC0100203A
:1016980019160008004000580CF0ACBF08B5FFF759
:1016A8008BFC40F6B83398420CD8B0F5E16F0BD3F9
:1016B800FE23A0F5E16058434FF49663B0FBF3F0C6
:1016C800C0B208BDFE20FCE70020FAE77FB56846F7
:1016D80000F0A6F80198FFF71DFA00B207B05DF810
:1016E80004FB0000184A38B5D2F88035591C044666
:1016F80016D100F0F9FF054601F002F8054400F0A4
:10170800F9FF2B0EE3712B0CA3712B0A6371030EE7
:10171800E370030CA370030A25716370207038BD51
:10172800190AC3718171190C1B0E41710371D2F82A
:101738008435C370D2F884351A0A82701A0C1B0ECD
:1017480042700370EBE700BF0070FF1F074BD3F830
:101758008005431C10B508D100F0C6FF044600F010
:10176800C9FF444000F0CCFF604010BD0070FF1F6F
:10177800012102200CF012BF002102200CF00EBF44
:1017880000207047024B187808B100F09DB87047E8
:10179800DC01002082B00190019802B000F030B95D
:1017A800F0B589B000F0B2FF00F0B8FF00F0BEFF5E
:1017B800012304930323069300254FF0B0430595B6
:1017C8000795DA6C154C42F00202DA64DA6C02F022
:1017D80002020292029ADA6C42F00202DA64DB6CCC
:1017E80003F0020301934FF4805703A92046019B9D
:1017F80003974FF4005601F077FF03A9204603969C
:1018080001F072FF2A463946204602F08DF82A4632
:101818003146204602F088F809B0F0BD00040048BF
:1018280010B50446FFF7E2FB074BA36040F30F2017
:10183800FEF7CCFF054B064A2360064B6060C4E9FF
:101848000323002010BD00BF0000484200007A4476
:101858000D093E00AB03050000207047014B1868D6
:10186800704700BFE00100200320704708B501461B
:101878004FF47A7200238002890DFFF791F908BDB1
:101888004FF47A73A0FB03309B0A43EA80507047F9
:10189800034B98689A689042FBD1C043704700BFD9
:1018A8000028004008B5FFF7F3FF014B186008BD9A
:1018B800E001002008B5FFF7EBFF024B1B68C01AD8
:1018C80008BD00BFE0010020024B187808B1FFF7FF
:1018D800DFBF7047DD01002010B5074B074C012220
:1018E800DA654FF48071204602F04EFE4FF0FF3368
:1018F8002363002010BD00BF00280040980100208D
:1019080002460021014803F058B800BF98010020A2
:1019180002460121014803F050B800BF9801002099
:1019280010B58CB02C220021044601A80DF0CAFA8B
:10193800FFF7D2FF0C4B1868002304440893069362
:101948004FF00053E4430793084802944FF4807320
:10195800012201A90B9302F02DFF08B1FFF752FDF8
:1019680000200CB010BD00BFE0010020980100204D
:1019780038B50546FFF78CFF02210446074803F0F7
:1019880023F8C4F309024FF47A71A2FB0121920AE9
:10199800A30A2A8043EA805038BD00BF980100207E
:1019A8000148002103F010B89801002001480121E6
:1019B80003F00AB898010020F8B50F4D2E78CEB97B
:1019C8000E4C4FF0FF372763FFF71EFDFFF784FF2C
:1019D8004FF48071204602F0D7FD2046276302F0BD
:1019E80097FF32462046022102F0E7FFFFF75AFF31
:1019F80001232B700020F8BDDD0100209801002094
:101A0800014610B54FF47A7200238002890DFFF762
:101A1800C7F80146FFF73CFF0446FFF739FF031BF1
:101A28008B4200D310BD00BFF7E70DF0CBB8000024
:101A380010B5064C0221204602F0C6FF0221421CC6
:101A48002046BDE8104002F0B8BF00BF9801002052
:101A58001648174A08B54FF4E133C0E900230023BC
:101A68000C22C0E90233C0E90523C0E90733C0E905
:101A78000933036104F0E8F808B1FFF7C3FC0B4829
:101A8800002104F071FA08B1FFF7BCFC07480021F7
:101A980004F08EFA08B1FFF7B5FC044804F041FAE7
:101AA80018B1BDE80840FFF7ADBC08BD44020020EE
:101AB8000044004070B596B006461422002103A8E1
:101AC8000DF000FA3822002108A80DF0FBF9326861
:101AD800274B9A424AD10223089308A8254B0A9318
:101AE80002F07CFC08B1FFF78DFC4FF0B0430025F5
:101AF8009A6D214C42F400329A659A6D02F40032D4
:101B08000292029ADA6C42F00102DA64DB6C03F0AA
:101B180001030193019B0C220223CDE90323032334
:101B2800CDE9055303A907234FF09040079301F02F
:101B3800DBFD124925621423C4E900131023C4E90C
:101B4800023520468023C4E90435C4E9065501F06E
:101B5800CBFA08B1FFF756FC2520B4670022022112
:101B6800A66201F02DFA252001F05CFA16B070BDCE
:101B78000044004004000C00E4010020580002402A
:101B880002680C4B9A4210B5044612D14FF0B0428D
:101B98000C21936D23F4003393654FF0904001F0CE
:101BA8004FFEA06F01F016FBBDE81040252001F0A4
:101BB80047BA10BD0044004008B50A46014602482D
:101BC80003F002FA002008BD4402002013B5114BAF
:101BD800114C18604FF40013009302AB13E9060090
:101BE800204604F042F92368DA69D103FCD4DA69A3
:101BF8005202FCD59A68084842F480029A6004F0C0
:101C08007AF906490448012204F0E0F8002002B0FD
:101C180010BD00BFD402002044020020DC020020D6
:101C280008B5074B1860FFF71FFAFFF711FF054AC1
:101C3800D2F8803043F00063C2F88030002008BD3D
:101C4800D80200200008005808B54FF0B0430848F3
:101C58009A6B42F400329A639A6B22F400329A63C8
:101C6800FFF78EFF0F2001F0EBF9002008BD00BF41
:101C78004402002008B5074803F0E6FF08B1FFF763
:101C8800C1FB054801F030FA18B1BDE80840FFF77C
:101C9800B9BB08BD44020020E40100200268044BDF
:101CA8009A4203D1034B00201B681847704700BFB6
:101CB80000440040D802002002680B4B9A4210B53D
:101CC80004460FD1094B1B682BB1D0F88C2012B9F0
:101CD80007480121984720460549BDE810400122E0
:101CE80004F074B810BD00BF00440040D4020020C6
:101CF800DC02002008B5FFF7A3FCBDE8084000F0AF
:101D080047BB4FF0FF300CF0D9BC0000014BD87036
:101D1800704700BF58000020014B1873704700BF80
:101D28005800002007B5064B00221B5C00931146A3
:101D3800044B02200CF074FB03B05DF804FB00BFF9
:101D4800FAF00008E0F0000808B5022000210CF0C5
:101D58007DFCBDE8084001480CF0E2BE30040020DC
:101D6800002101200CF072BC10B5094C60B1206054
:101D780008480CF085FE216806480CF00BFFBDE80A
:101D8800104004480CF0CCBE42F210732360EFE719
:101D98006C0000203004002008B50E4B1B78022B85
:101DA80003D1002108200CF051FC0B4800224FF40D
:101DB800004101F0B9FD084800224FF4007101F01C
:101DC800B3FDBDE80840044800224FF4006101F06B
:101DD800ABBD00BF000000200004004802480022FC
:101DE8004FF4004101F0A0BD000400480248002261
:101DF8004FF4007101F098BD000400488AB201490F
:101E08000CF018BC00F0030870B51F4801224FF40D
:101E1800004101F089FD1C4801224FF4007101F0D6
:101E280083FD01224FF40061174801F07DFD17483A
:101E38000CF026FE04F046FD044650B10022144B77
:101E4800114602200CF0ECFABDE8704011480CF085
:101E580067BE114D114B0246014602200CF0E0FA14
:101E680001260F4B2E702246214602200CF0D8FA8C
:101E78000C4804F0B9FB2878314604F0D1F803483F
:101E88000CF04EFEE0E700BF0004004830040020DC
:101E9800FEF0000800040020000000201CF10008EB
:101EA80030F10008580000202DE9F04188B0FFF714
:101EB800F5FB044602A8FFF7B3FC534B009401223C
:101EC800002102200CF0ACFA0398504C504FFEF75A
:101ED80021FE00B201224F4B0090002102200CF09D
:101EE8009FFA4823049823704B49FEF7C3FCFEF77A
:101EF80037FE85B20398FEF70DFE484906B20298F0
:101F0800FEF7B8FC4449FEF769FDFEF729FE444A8E
:101F1800636812781A706368C0F307225A7063689E
:101F280098706368DE7063682A0A1A7163685D7165
:101F38003B78082B01D0012B37D8626800239371B6
:101F48006268D3716268137253720A236370354CE6
:101F5800637A63B104F038F9012808D120460CF0FF
:101F68008FFD314800224FF4006101F0DDFCF97863
:101F78002648002204F03CF9044678BB01220146B9
:101F88002A4B10460CF04CFA29480CF079FD294BE5
:101F980027481968A14238BF21460CF0FBFD2448A8
:101FA8000CF0BEFD08B0BDE8F081DDE90565D4F8A8
:101FB8000480FFF773FB88F8060063683214DA714F
:101FC800636832121A722A149A722A12DA7200227A
:101FD8005E721D735A739A730F23B7E7063410D1D4
:101FE80004F0ECF804460028CED001224FF47A73AE
:101FF8000021B0FBF3F3104600930F4B0CF010FADE
:10200800C2E70024C0E700BF4FF100080400002029
:10201800580000205AF10008000020410000C84282
:10202800CF030020D00300200004004865F1000819
:10203800300400206C00002074F1000802484FF4BE
:10204800006101F076BC00BF0004004800B50346FB
:102058008DB000282CD0407802280AD003282AD036
:10206800164B0022114602200DB05DF804EB0CF06F
:10207800D7B91A7F0B92DA7E0A929A7E09925A7E13
:1020880008921A7E0792DA7D06929A7D05925A681E
:102098000492DA68039293F914200292B3F9122099
:1020A80001921B7C00930022054B11460CF0B8F9F5
:1020B8000DB05DF804FB034BD3E700BF92F10008B5
:1020C800A9F100081BF2000801284FF000020CBF1C
:1020D800024B034B114602200CF0A2B93AF2000859
:1020E8004CF2000808B504F0F6FB80B904F06CF86F
:1020F80001280CD1BFF34F8F0549064BCA6802F47B
:10210800E0621343CB60BFF34F8F00BFFDE708BD0C
:1021180000ED00E00400FA051FB50446002837D09A
:102128000378002B34D001224FF400711E4801F0CF
:10213800FBFB1E480CF0F4FC002211461C4B02204D
:102148000CF06EF994F91830039394F90A3002935D
:10215800237C0193E368009300221146154B03206A
:102168000CF05EF90022144B114603200CF058F9CC
:10217800237A012B0ED1617A104A114B002908BF2E
:1021880013460022009311460E4B03200CF048F929
:1021980004B010BD00220C4B1146032004B0BDE86A
:1021A80010400CF03DB900BF00040048180400209E
:1021B80065F2000896F20008C7F2000860F200080D
:1021C80061F20008D4F20008E5F2000870B505468F
:1021D800F8B190F90540D4B90E480CF051FC0E48FE
:1021E80022464FF4006101F09FFB0C4B224621462A
:1021F80002200CF015F9AB79012B0CBF084B094BE9
:102208000022BDE87040114602200CF009B9064BC7
:10221800F6E770BDD003002000040048F3F2000880
:1022280008F3000825F3000842F30008F0B5054656
:1022380087B00C4661B32E4801224FF4004101F0EB
:1022480073FB2C480CF06CFC267846B1002D4CD062
:102258006B682E781BB1032E1CD0482E27D0237C08
:10226800052B15D894F90A20059294F909200492AF
:10227800214A52F82330039394F90830CDE90163D9
:102288000022E368009311461C4B03200CF0C8F8A9
:1022980007B0F0BD6A78012AE1D11878012803D087
:1022A800022801D00028DAD104F06AF8D7E76F785D
:1022B800012FD4D11D78124B05F001051D7065B9A9
:1022C8002A46104B294603200CF0AAF82A4608484B
:1022D8004FF4006101F028FBC1E7002211460A4BC8
:1022E80003200CF09DF83A46F1E72E46B7E700BF09
:1022F80000040048E80300209CF400086EF300087E
:10230800CF0300205BF3000865F3000838B50446E6
:102318000D4601F0D7F80246D8B90E4BD3F8E005C0
:102328000D4B03EA80204FF47C33B3FBF0F34343B7
:10233800C3F57C33D80A0121FEF7F4FE034620B921
:1023480006482A462146FEF705FFBDE8384001F059
:10235800CBB838BD0070FF1F00FCFF0300F0030876
:1023680010B504F0C1FA10F1080F07D1064B00228E
:10237800BDE81040114602200CF052B8013001D1DE
:10238800024BF4E710BD00BFB5F30008CBF300081B
:102398002DE9F04186B0002402250126CDE900652B
:1023A8002246214604274B4B0294284605940CF0FC
:1023B80037F8CDE9005722462146474B0294284674
:1023C8000CF02EF82246CDE90154444B00962146E4
:1023D80028460CF025F805A9204604F05FFA059B6D
:1023E800DFF8FC80C3F307220292C3F307421B0EF7
:1023F8000192009322463B4B214628460CF010F8E8
:1024080005A9304604F04AFA059BDAB20392C3F3F1
:1024180007220292C3F307421B0E01920093224641
:102428002146314B28460BF0FBFF22462F4B0094E8
:102438004FF4FA712E480CF0C5FA22462D4B009441
:102448004FF4FA712C480CF0BDFA32462B4B00942D
:102458004FF4FA7140460CF0B5FA294B0094224625
:102468004FF4FA6127480CF0ADFA21463046264A67
:102478000CF0A8F921462846244A254D0CF0A2F96B
:1024880021463846234A0CF09DF9234A2146082064
:102498000CF098F900F058F84FF081711F4804F0DB
:1024A800C3F91F4804F0A0F840460CF039FB1D4B57
:1024B8002146187803F0B4FD1B4900941B4B0968AA
:1024C800224628460CF07EFA28460CF029FB06B076
:1024D800BDE8F081E3F3000804F4000825F40008DF
:1024E800D003002046F4000867F40008F51D000832
:1024F80018040020E51D0008E80300204520000816
:10250800A11D00080004002025630008B11E000872
:102518003004002069230008111E00080C00002068
:1025280058000020000000206C000020511D000809
:10253800022804D0402806D10021042001E000210F
:1025480008200CF083B87047044B0022C3E902222C
:1025580001210322C3E90021704700BF480400207D
:1025680000487047480400204FF0B04382B0DA6C4E
:102578000243DA64DB6C18400190019B02B070479B
:102588002DE9F04186B01422002101A80CF09AFC34
:102598000220FFF7E9FF144D144F0420FFF7E4FF72
:1025A8004FF4807601230024CDE9016301A90323B8
:1025B8002846CDE903434FF4005801F095F801A9E6
:1025C8003846CDF8048001F08FF822464146384657
:1025D80001F0AAF928462246314601F0A5F920461D
:1025E80006B0BDE8F08100BF0004004800080048BC
:1025F800032810B50ED8012810D868B902460B4830
:102608004FF4807101F090F9002209484FF400510D
:1026180001F08AF9002010BD0122F0E700220348EA
:102628004FF4807101F080F90122EEE700040048C0
:1026380000080048022070470020704701207047BA
:1026480000280CBF0F201620704700000D48854653
:1026580000F025F80C480D490D4A002302E0D45833
:10266800C4500433C4188C42F9D30A4A0A4C0023D4
:1026780001E013600432A242FBD30CF0FFFBFEF72B
:10268800B5FEFEE7008000200000002018010020B1
:1026980070FE00081801002018160020FEE7704799
:1026A80010B5032000F07AFC01F0C6FA064B18605A
:1026B8000F20FFF765F8044618B9FEF740FF2046DB
:1026C80010BD0124FBE700BF700000204FF0E0229E
:1026D800136923F00203136170474FF0E022136976
:1026E80043F0020313617047014BD3F8900570471C
:1026F8000070FF1F014BD3F8940570470070FF1F4F
:10270800014BD3F8980570470070FF1F024A5368C1
:1027180023F0010353607047002004E0024A536825
:1027280023F0020353607047002004E0024A536814
:1027380023F0040353607047002004E08068C0F36E
:1027480080007047F7B5002301930446002800F085
:10275800F980856D25B9FEF7D1FBE56584F85450FD
:1027680020688368D90040F1A4808368DA0000F10A
:10277800B780A36D43F01003A365E36D43F0010335
:10278800E3650125FFF7DAFFA36D03F01003184393
:10279800A36D40F0D98023F4817343F002032168CC
:1027A800A3658B68DB0760D4E368A26894F818E037
:1027B80094F819C0276BA67E1A4342EA8E3343EA7F
:1027C800CC33226994F82CC0002F43EA463318BF53
:1027D8004FF4805743EA4C03002AB4BF22F000426A
:1027E8004FF400123B43134394F82020012A03D1ED
:1027F800002E77D143F48033626A22B1A66A02F4CC
:10280800E07232431343CA6822F4FE3222F4FF72A4
:1028180013436268CB60E36C02F0404C4CEA030758
:1028280094F83C30012B09D1D4E910363343A66C17
:102838003B43334343EA0C0343F001070B69444E1F
:102848001E4022F000433E43B3F1804F0E610CD08E
:10285800B2F1004F09D03F4ED6F8083702F4701293
:1028680023F470131A43C6F808274B69666BA26BEA
:1028780023F0070333434B614B6923F0700343EAAA
:1028880002134B612369002B35D18B6A63F00F0368
:102898008B624B6903F007039E4249D10023E3652D
:1028A800A36D23F0030343F00103A365284603B097
:1028B800F0BD8368284A23F0104323F0170343F040
:1028C80080538360254B1B68B3FBF2F301335B0035
:1028D8000193019B002B3FF448AF019B013BF7E7B5
:1028E80000254FE7A26D42F02002A265E26D42F09A
:1028F8000102E26580E7B3F5001FCAD1276E8200A6
:1029080027FA02F202F00F020F2A0ED0013008282F
:10291800F5D18B6AE369013B9B0003F01C036FF060
:102928000F0202FA03F33B43B2E70128ADD0F0E708
:10293800A36D23F0120343F01003A365E36D43F086
:102948000103E3650125B1E743F01003A365F9E747
:1029580002FCFF1F00200140400D03007000002012
:10296800F8B54569082D04460E460AD00368DB68A9
:10297800D90705D5836D43F0200383650120F8BD91
:102988000425FEF7FFFE0746206803682B4222D085
:10299800A36D43F40073A365C36813F4406F14D1A7
:1029A800A37E93B903681B070FD5FFF7C7FE38BB93
:1029B8002268536823F00C035360A36D23F48073DB
:1029C80023F0010343F00103A365207E08BB2368BD
:1029D8000C221A60D3E7721CD7D0FEF7D3FEC01BB7
:1029E800B04201D8002ECFD123681B682B40CBD131
:1029F800A26D84F8543042F00402A2650320BEE7B9
:102A0800A36D43F02003A365E36D43F00103E36581
:102A1800DBE70020B3E70368186C7047F7B50023BD
:102A2800019390F85430012B044600F0C78001232D
:102A380080F854300068FFF781FE002840F0B88025
:102A4800D1E900202369022823F0040300F08380E1
:102A5800B3F1004F2568C2F3110E13D1AB6A43EAF4
:102A68000E03AB628B68686903EA022323F07C4398
:102A780023F0FF0320EA02210B43002A6B6126DBC7
:102A8800002055E0236E00F01F074FF00F0C0CFAE2
:102A980007FC6FEA0C0623EA0C0CBEF1000F11D1FB
:102AA800C2F38463BB4043EA0C0323668008E369EE
:102AB80001309842D6D8A86AC2F38363BB40064067
:102AC8003343CEE792FAA2F3B3FA83F3EAE73C4939
:102AD8003C48D1F80837824203F0E07519D11B024F
:102AE800CED4D1F80837384A23F0E0732B4343F4A7
:102AF8000003C1F80837354B1B68B3FBF2F20C230F
:102B080002FB03330193019B002BB9D0019B013BCE
:102B1800F8E72F48824210D113F08070B0D1D1F875
:102B2800083723F0E0732B4343F08073C1F808376C
:102B3800002384F8543003B0F0BD264882429FD168
:102B480013F480009CD1D1F8083723F0E0732B43AD
:102B580043F48003EAE7B3F1004F06D121688B6A9A
:102B6800C2F3110023EA00038B62002A88DA1548B1
:102B780013498242D1F8083709D1D1F8082703F060
:102B8800A07322F0E0721343C1F8083778E71048C1
:102B9800824204D1D1F8082703F44003F1E70D4835
:102BA80082427FF46DAFD1F8082703F0C073E8E7DD
:102BB800A26D42F02002A2651846B9E70220BAE7E2
:102BC80000200140001000B0400D030070000020FC
:102BD800004000B8002000B438B504460068FFF78C
:102BE800ADFD08B9002038BD22689368990707D45D
:102BF800936823F0004323F0170343F01003936016
:102C0800FEF7C0FD054623689B685B07EAD5FEF71B
:102C1800B9FD401B0228F6D923689B685A07F2D5EC
:102C2800A36D43F01003A365E36D43F00103E3656F
:102C38000120D8E773B50023026801939368DD0784
:102C4800044602D5002002B070BD9168214B19429C
:102C580009D0A36D43F01003A365E36D43F00103AE
:102C6800E3650120EFE7936823F0004323F017039F
:102C780043F001039360184BD3F8083718021CD4AB
:102C8800637E012BDED0FEF77DFD144E05462268DB
:102C98001368DB07D6D49368D9075FBF93683340BE
:102CA80043F001039360FEF76DFD401B0228EED947
:102CB80023681B68DA07EAD4CBE7094B094A1B6883
:102CC800B3FBF2F301330193019B002BD8D0019B96
:102CD800013BF8E71700008000200140E8FFFF7F74
:102CE80070000020400D030038B504460068FFF767
:102CF80025FD054620BB94F85430012B20D0012334
:102D080084F854302046FFF795FFB0B9A36D2268C8
:102D180023F4706323F0010343F48073A3651C2339
:102D2800E065136084F85400936823F0004323F0AF
:102D3800170343F00403936038BD84F85450FBE74D
:102D48000220F9E7026838B5936891680446C80715
:102D580001D4002038BD9907FBD4936803F005031C
:102D6800012B19D1936823F0004323F0170343F094
:102D78000203936003231360FEF704FD05462368EE
:102D88009B68DB07E5D5FEF7FDFC401B0228F6D95A
:102D980023689B68DA07F2D5A36D43F01003A36597
:102DA800E36D43F00103E3650120D3E770B5044602
:102DB800002843D0836D43F002038365FFF70CFFBF
:102DC800054668B92046FFF7BDFF054608B9012347
:102DD800A3652268936823F0104323F017039360D8
:102DE80023685A6822F4677222F003025A6040F29C
:102DF8009F321A60D968124A0A40DA601A6922F0CA
:102E080040421A615A6922F007025A611A6A02F0AE
:102E1800F0221A629A6A0B4A00269E62D2F8083794
:102E280023F0FE73C2F808372046FEF77BF8E66504
:102E38002666A66584F85460284670BD0125FBE720
:102E480000023E830020014010B590F85430012B59
:102E5800044615D0012380F85430FFF7BDFE58B959
:102E68002046FFF76FFF38B9A36D23F4807323F072
:102E7800010343F00103A365002384F8543010BD17
:102E88000220FCE7F7B50023019390F85430012B9A
:102E980004467FD0012380F85430FFF753FF23689E
:102EA8009A6812F00102054670D1A16D3A4F21F4DB
:102EB800817141F00201A165DE68D96821F4004101
:102EC80021F00301D96008209968394041F0004198
:102ED80099609968002913DA0199013101910199E2
:102EE800B1F52E3FF5D3A36D23F0120343F0100381
:102EF800A365002384F854300125284603B0F0BDAB
:102F0800D3F8B410013801F07F010A44DCD1996884
:102F18002148014041F001019960D3F8B41021F033
:102F28007F0141EAD202C3F8B4209A68024042F015
:102F380002029A60FEF726FC074623689A68D207C1
:102F480012D426F4FF4626F07C06DA683604360CDE
:102F58001643DE60A36D23F0030343F00103A3656A
:102F6800002384F85430C8E7FEF70CFCC01B022885
:102F7800E3D923689B68D907DFD5A36D43F0100315
:102F8800A365E36D43F00103E365B5E7A36D43F083
:102F98001003E4E70225B0E7E8FFFF7F0749CA68A6
:102FA80022F4E0620302120403F4E063120C1343F8
:102FB80043F0BF6343F40033CB60704700ED00E09B
:102FC800164B30B5DC68C4F30224C4F10703251D91
:102FD800042B28BF0423062D4FF0FF3505FA03F311
:102FE8008CBF033C002421EA0303A34005FA04F440
:102FF80022EA0402002843EA0203ACBF00F1604061
:10300800074A4FEA0313B8BF00F00F00DBB2AABFAC
:1030180000F56140135480F8003330BD00ED00E046
:1030280014ED00E0002808DB0123420900F01F002E
:1030380003FA00F0014B43F82200704700E100E07A
:1030480000280DDB4309012200F01F0002FA00F0FE
:103058002033044A42F82300BFF34F8FBFF36F8F2A
:10306800704700BF00E100E070B5D0E91345656026
:10307800446D14B1D0E916456560D0E9105404F0E8
:103088001C060124B4406C60046863608368102BDC
:103098000BBFA260A160E160E26070BD0268416C94
:1030A800D3B210B5083B1424B3FBF4F30B4CA24283
:1030B80088BF0B4A21F0030199BF01F1804202F554
:1030C8000232521807338264064AC26403F01F03AF
:1030D800012202FA03F3036510BD00BF0704024092
:1030E8001C0802408008024010B5002861D0026820
:1030F800314B9A424FF014044ED830491144B1FB79
:10310800F4F189004164A3F207430364022380F8C1
:103118002530136823F4FF4323F070031360D0E9CC
:1031280002342343046911682343446923438469AF
:103138002343C4692343046A23430B431360FFF703
:10314800ADFF8368816CB3F5804F04BF00234360F3
:10315800426802F07F030B60D0E91314013A032A96
:103168004C6021D8164A174981651A44013B9200E0
:10317800012103F0030301FA03F300214265C3654B
:103188001160114A536400230122C36380F824307C
:1031980080F82520184610BD0C4B1344B3FBF4F3FC
:1031A8009B0043640A4BB0E70023C0E91533C365AD
:1031B800E9E70120EFE700BF07040240F8FFFDBF81
:1031C8003F8200104009024000090240F8FBFDBFA1
:1031D8000004024038B5002845D001680B6823F088
:1031E80001030B60214B99424FF0140433D8204A55
:1031F8000A44B2FBF4F292004264A3F20743036468
:10320800D0E91023012403F01C0304FA03F300257A
:103218000D605360FFF742FF836C41681D60D0E981
:1032280013325A604A1E032A06D8124B0B449B00DD
:1032380094401D60104B5C640023C363C0E91533E0
:10324800C0E90B33C0E90D33C36580F8253080F839
:103258002430184638BD094B0B44B3FBF4F39B00EC
:103268004364074BCBE70120F4E700BF07040240A3
:10327800F8FFFDBF3F82001000090240F8FBFDBFC8
:103288000004024070B590F82450012D04463CD04B
:1032980090F825600125AE4280F824504FF00006D2
:1032A8002DD1022580F82550C6630668356825F0BB
:1032B80001053560FFF7D8FE026B0368BAB11A68DA
:1032C80042F00E021A60A26C1168C90342BF11686D
:1032D80041F480711160626D1AB1116841F4807116
:1032E80011601A6842F001021A60002070BD1A6865
:1032F80022F004021A601A6842F00A02E2E7802308
:10330800C36380F824602846F0E70220EEE740B166
:1033180090F82530022B06D00423C363002380F8DD
:103328002430012070470368816C1A6822F00E026D
:103338001A600A6822F480720A601A6822F0010290
:103348001A60D0E9101303F01C02012393404B606C
:10335800D0E913325A60436D33B11A6822F480728F
:103368001A60D0E916325A60012380F8253000230C
:1033780080F824301846704710B590F82530022B95
:1033880003D00423C363012010BD03681A6822F028
:103398000E021A601A6822F001021A60826C136821
:1033A80023F480731360D0E9101303F01C02012387
:1033B80093404B60D0E913325A60436D33B11A68B9
:1033C80022F480721A60D0E916325A60012380F81C
:1033D8002530836B002480F8244013B19847204699
:1033E800D2E71846D0E7000070B4426C046C03685A
:1033F80026681D6802F01C020421914031420FD05A
:1034080015F0040F0CD01A6892065EBF1A6822F0F5
:1034180004021A60036B6160002B33D070BC18473C
:1034280002219140314217D015F0020F14D01A68CA
:10343800940606D41A6822F00A021A60012280F85B
:103448002520114A93428CBF104B114B5960002321
:1034580080F82430C36ADFE708219140314211D057
:1034680029070FD5196821F00E011960012303FA05
:1034780002F26260C36380F82530002380F82430AC
:10348800436BC9E770BC70478000024000040240EB
:10349800000002400A4A536943F4802330B553615F
:1034A800EFF3108472B60023CD58C5500433B3F53A
:1034B800807FF9D11369DB03FCD484F3108830BD15
:1034C80000400058064B5A69002ABFBF054A9A6057
:1034D80002F188329A60BABF5869C00F002070475D
:1034E8000040005823016745044B5A6942F00042E6
:1034F8005A615869C043C00F704700BF0040005868
:1035080070B50546FEF73EF9124E04463369D903F5
:1035180013D43369DA0744BF012232614CF2FA321C
:10352800134011D10B4E306910F480200BD0FEF7F8
:1035380029F9001BA842F6D304E0FEF723F9001B83
:10354800A842E3D3032070BD024A1361024A012056
:103558005360F8E700400058580400202DE9F04176
:10356800184D98462B78012B06460C46174626D050
:1035780001232B704FF47A7000236B60FFF7C0FFB4
:10358800A0B9012E16D1104A536943F001035361C3
:103598002760BFF36F8FC4F804804FF47A70FFF789
:1035A800AFFF094A536923EA0606566100232B70C8
:1035B800BDE8F08139462046FFF76CFFEDE70220B1
:1035C800F6E700BF5804002000400058054A536938
:1035D80023F47E7343EAC00040F4803040F00200D8
:1035E80050617047004000582DE9F041234F3B7867
:1035F800012B054688463FD001233B704FF47A7073
:1036080000237B60FFF77CFF044688B92B68042BF6
:1036180013D11B4A536943F4803343F004035361C5
:103628004FF47A70FFF76CFF0446154B1A681B6855
:1036380000233B702046BDE8F0814FF0FF33C8F807
:1036480000306E68D5E901321344B3420AD93046D6
:10365800FFF7BCFF4FF47A70FFF752FF50B1C8F87C
:1036680000600446064A536923F47E7323F002037C
:103678005361DAE70136E5E70224DBE75804002066
:103688000040005870B5164C2378012B054625D00C
:10369800012323700368A36000264FF47A706660E4
:1036A800FFF72EFF014610B12670084670BD0D4A7F
:1036B800536943F0407353612B68042B07D1206191
:1036C800536943F4803343F004035361EDE7AB6877
:1036D800686863612061FFF779FFE6E70221E4E7A4
:1036E80058040020004000582DE9F04F524C0023A8
:1036F8004FF00F090A6832FA03F501D1BDE8F08FDF
:10370800012505FA03F818EA020200F08E804E68D7
:10371800032706F003054FEA430E07FA0EFC6F1E57
:10372800012F6FEA0C0C32D8876807EA0C0ACF68B9
:1037380007FA0EF747EA0A078760476827EA080882
:10374800C6F300179F4047EA08074760C76807EABB
:103758000C088F6807FA0EF747EA0807022DC760BA
:1037680017D14FEAD30800EB880803F0070AD8F806
:1037780020704FEA8A0A09FA0AFB27EA0B0B0F693D
:1037880007FA0AF747EA0B07C8F8207001E0032D8B
:10379800DCD1076805FA0EF507EA0C072F4316F483
:1037A800403F076041D023F0030707F1804707F542
:1037B800803703F0030CBD684FEA8C0C4FF0070EFE
:1037C8000EFA0CFEB0F1904F25EA0E0E2FD01B4DCD
:1037D800A8422ED005F58065A8420CBF0225072512
:1037E80005FA0CF545EA0E05BD602568D74316F4C1
:1037F800801F0CBF3D4015432560656816F4001F07
:103808000CBF3D4015436560D4F8805016F4803FE6
:103818000CBF3D401543C4F88050D4F88450B6031B
:1038280054BF3D401543C4F88450013362E7002576
:10383800D6E70125D4E700BF000800580004004877
:10384800374A2DE9F04F00234FF0010A4FF0070BDC
:103858004FF00F0931FA03F401D1BDE8F08F0AFAED
:1038680003FC1CEA010654D023F0030404F180444D
:1038780004F5803403F00307A568BF000BFA07F8C6
:10388800B0F1904F08EA050E45D0264DA84244D025
:1038980005F58065A8420CBF02250725BD40754582
:1038A80017D1D2F8805025EA0605C2F88050D2F820
:1038B800845025EA0605C2F88450156825EA0605ED
:1038C8001560556825EA06055560A56825EA0805C6
:1038D800A560056803265C0006FA04F423FA06F6D8
:1038E800254300EB8606056003F00705376AAD003F
:1038F80009FA05F527EA05053562856825EA04050C
:103908008560456825EA0C054560C56825EA040414
:10391800C46001339EE70025C0E70125BEE700BF6C
:1039280000080058000400480AB1816170478162AC
:103938007047436901EA030221EA030141EA0241AF
:1039480081617047044AD168014208B502D0D0604D
:10395800FEF7EEFD08BD00BF00080058024A1368D4
:1039680043F4807313607047000400580D4B10B582
:103978005B690C4628B99A0507D500F027F820B1ED
:1039880010BD9B0501D400F019F8074A1369012CF2
:1039980023F00403136101D130BFF1E740BF20BF1A
:1039A80020BFEDE70004005800ED00E0024B186866
:1039B80000F4C060704700BF00040058024A136852
:1039C80043F4804313607047000400580C4A13689E
:1039D80023F4804313600B4B1B6832214B430A4985
:1039E800B3FBF1F35169890500D533B9536913F471
:1039F800007F14BF032000207047013BF2E700BF9F
:103A0800000400587000002040420F000B4A136861
:103A180023F0070343F002031360094B1A690128D6
:103A280042F004021A6105D130BF1A6922F004027B
:103A38001A61704740BF20BF20BFF6E70004005856
:103A480000ED00E04FF0B0431868C0F34040704705
:103A58004FF0B0431868C0F3802070474FF0B04370
:103A68001868C0F3400070474FF0B042536823F421
:103A78007F4343EA0023536070474FF0B043186810
:103A8800C0F34060704700007FB54FF0B0432C4A48
:103A9800D3F80831C0F3031003F00F0352F82040A5
:103AA800284A52F82330B4FBF3F4FFF77FFF264B84
:103AB800054693E80700B5F5007F04AB03E9070066
:103AC80010D0224B9C4218D303F5B70303F67F535B
:103AD8009C4229D903F5741303F510639C4225D839
:103AE80002230BE01A4B9C4207D91A4B9C421BD964
:103AF80003F5370303F5D853F0E7002304AA02EBD4
:103B0800830353F80C4C144D2B6823F0070323430D
:103B18002B60FDF737FE06462B6803F007039C422F
:103B280006D1002004B070BD0123E7E70024EAE7CE
:103B3800FDF728FE801B0228EED90320F2E700BF1C
:103B480014F50008B4F40008F8EF0008C0CF6A00C4
:103B5800BFEA21013F933402004000584FF0B043C0
:103B680010B59A68D96812F00C0205D00C2A4AD10F
:103B780001F00303012B50D14FF0B0412B480B68E3
:103B880013F0080306D00B6813F0080337D1D1F8F7
:103B9800941007E00C68240756BFD1F894300968E0
:103BA800C3F3032350F82330002A0CBF1846002023
:103BB8004FF0B0418A6802F00C020C2A1ED1CA6884
:103BC80002F00302022A2ED0032A06D10B68184AF3
:103BD80013F4801F174B18BF13464FF0B042D0683C
:103BE800D168D268C0F306205843C1F302130133E9
:103BF800B0FBF3F0530F0133B0FBF3F010BD0B68CB
:103C0800C3F30313CEE7042A0AD0082A05D11B6898
:103C180013F4801304D10748CAE700231846C7E7FE
:103C280003480023C4E7024BD7E700BF14F5000898
:103C38000024F4000048E80108B5FFF78FFF4FF0B3
:103C4800B043044A9B68C3F3031352F82330B0FB14
:103C5800F3F008BDB4F400082DE9F041044600284B
:103C680055D04FF0B0439D68DE680368990605F0AB
:103C78000C0506F003066BD51DB10C2D49D1012E9C
:103C880047D1FFF7EBFE10B1236A002B3FD04FF06E
:103C9800B043A06A1A68120756BFD3F894301B685D
:103CA8001B0903F0F00398421ED9FFF7EDFE002828
:103CB8002DD14FF0B042136843F008031360136826
:103CC800A16A23F0F0030B431360606AFFF7CCFE90
:103CD800FFF7B2FFAC4B1860AC4B1868FDF750FD0E
:103CE800002835D0BDE8F0814FF0B042136843F0AA
:103CF80008031360136823F0F00303431360606A3A
:103D0800FFF7B2FEA06AFFF7BFFE0028E0D001204F
:103D1800E8E7226A4FF0B043002A54D01A6842F00C
:103D280001021A60FDF72EFD0746FFF797FE0028EF
:103D380042D04FF0B042136843F008031360136891
:103D4800A16A23F0F0030B431360606AFFF78CFE4F
:103D58002368DB0748D423689F0700F19080236815
:103D68001E0740F1FC80A3694FF0B046002B00F01D
:103D7800E380D6F89430E16903F01002914200F034
:103D8800C68003F00302022AC1D0D80740F1B580EB
:103D9800D6F8943023F00103C6F89430FDF7F2FC0E
:103DA8000746D6F89430990740F1A780FDF7EAFC5A
:103DB800C31B112BF5D904E0FDF7E4FCC01B022856
:103DC800B3D903208EE71A6822F001021A60FDF7C2
:103DD800D9FC0746FFF742FE0028B9D0FDF7D2FC10
:103DE800C01B0228F6D9ECE7082D03D00C2D09D109
:103DF800032E07D1FFF726FE0028ACD06368002BFE
:103E0800A9D184E74FF0B043A1681A6822F4801260
:103E18000A431A606268B2F5803F10D11A6842F40A
:103E280080321A60FDF7AEFC0746FFF70BFE00284C
:103E380091D1FDF7A7FCC01B6428F6D9C1E7B2F5FC
:103E4800041F04D11A6842F400121A60E6E71968E0
:103E580021F480311960196821F400111960002AD1
:103E6800E0D1FDF78FFC0746FFF7ECFD00283FF493
:103E780072AFFDF787FCC01B6428F5D9A1E7042DB4
:103E880003D00C2D12D1022E10D1FFF7E1FD18B18D
:103E98002369002B3FF43BAF4FF0B0426169536890
:103EA80023F0FE4343EA0163536058E722694FF069
:103EB800B04382B11A6842F480721A60FDF762FC5E
:103EC8000646FFF7C5FD0028E6D1FDF75BFC801B21
:103ED8000228F6D975E71A6822F480721A60FDF78D
:103EE80051FC0646FFF7B4FD00283FF438AFFDF754
:103EF80049FC801B0228F5D963E74FF0B042E1691D
:103F0800D2F8943023F010030B43C2F894304FF0EA
:103F1800B047D7F8943043F00103C7F89430FDF761
:103F280031FC0646D7F894309A0718D4FDF72AFCD6
:103F3800831B112BF6D944E7D6F8943023F00103FC
:103F4800C6F89430FDF71EFC0746D6F894309B0758
:103F580005D5FDF717FCC31B112BF6D931E72368EC
:103F6800580753D50A4F3B68D90513D4FFF7F6FC19
:103F7800FDF708FC06463B68DA050BD4FDF702FCA2
:103F8800831B022BF7D91CE7700000207400002067
:103F980000040058E3684FF0B046002B58D023F0D7
:103FA8008003052B02BFD6F8903043F00403C6F80F
:103FB80090304FF0B046FDF7E5FBD6F8903043F06F
:103FC80001030746C6F8903041F28838D6F8903099
:103FD8009B0705D4FDF7D6FBC31B4345F6D9F0E68E
:103FE800E36823F00403812B1BD1FDF7CBFBD6F844
:103FF800903043F08003C6F8903007464FF0B04643
:1040080041F28838D6F89030180504D5E06A0028BF
:104018004AD1002066E6FDF7B5FBC01B4045F1D943
:10402800CFE6FDF7AFFBD6F8903023F08003C6F853
:10403800903007464FF0B04641F28838D6F89030B5
:104048001905E3D5FDF79EFBC01B4045F6D9B8E638
:10405800FDF798FBD6F8903023F080030746C6F8A2
:10406800903041F28838D6F890301A0516D4FDF70A
:1040780089FBD6F8903023F00103C6F89030074644
:104088004FF0B04841F28836D8F890309B07BDD53C
:10409800FDF778FBC31BB342F6D992E6FDF772FB36
:1040A800C01B4045DFD98CE60C2D53D04FF0B043F0
:1040B80002281A6822F080721A6033D1FDF762FB79
:1040C8000546FFF7DAFC38BBD4E90C314FF0B042B3
:1040D8000B43D0682F4901400B43E16B0B43216C24
:1040E8000B43616C0B43A16B43EA0123D360136854
:1040F80043F080731360D36843F08053D360FDF7B7
:1041080041FB0446FFF7B9FC002882D1FDF73AFBD2
:10411800001B0A28F6D954E6FDF734FB401B0A2891
:10412800CFD94EE6DA6822F00302DA60DA6822F0C4
:10413800885222F48032DA60FDF724FB0446FFF748
:104148009CFC00283FF465AFFDF71CFB001B0A2808
:10415800F5D936E601283FF4C5AD4FF0B043226BE0
:10416800DB6803F0030191427FF4D1AD616B03F08A
:1041780070028A427FF4CBADA16B03F4FE42B2EB2E
:10418800012F7FF4C4AD626C03F0604393423FF4A7
:1041980040AFBCE58C80C1112DE9F0410D460446C5
:1041A80010B90120BDE8F081674E336803F00703BA
:1041B8008B4216D32368980727D54FF0B047A268DB
:1041C800BB6823F0F0031343BB60FDF7DBFA064638
:1041D800BB68D90319D4FDF7D5FA831B022BF7D98D
:1041E80011E0336823F007030B433360FDF7CAFA85
:1041F8000746336803F00703AB42DBD0FDF7C2FA8A
:10420800C01B0228F5D90320CCE723685A0617D526
:104218004FF0B0476269D7F8083123F00F0343EA3B
:104228001213C7F80831FDF7ADFA0646D7F808317A
:10423800DB0305D4FDF7A6FA831B022BF6D9E2E7C8
:1042480023685E0713D54FF0B047E268BB6823F4D4
:10425800E0631343BB60FDF795FA0646BB68980315
:1042680005D4FDF78FFA831B022BF7D9CBE7236818
:10427800190714D54FF0B0472269BB6823F460537F
:1042880043EAC203BB60FDF77DFA0646BB685A03E2
:1042980005D4FDF777FA831B022BF7D9B3E7236818
:1042A800DB070FD4284C236803F00703AB4237D849
:1042B800FFF7C2FC254B1860254BBDE8F041186894
:1042C800FDF75EBA6368022B1ED1FFF7BBFB00281F
:1042D8003FF467AF4FF0B0466268B36823F003035A
:1042E8001343B360FDF74EFA41F288380746B368C6
:1042F800626803F00C03B3EB820FD3D0FDF742FAE8
:10430800C01B4045F3D97EE7032B02D1FFF7B5FB6D
:10431800DDE713B9FFF7A2FBD9E7FFF799FBD6E76B
:10432800236823F007032B432360FDF72BFA064687
:10433800236803F00703AB42BAD0FDF723FA801BCA
:104348000228F5D95FE700BF004000587000002040
:104358007400002008B5FFF76FFC4FF0B043044A23
:104368009B68C3F3022352F82330D84008BD00BF2E
:10437800F4F4000808B5FFF75FFC4FF0B043044AB7
:104388009B68C3F3C22352F82330D84008BD00BF4E
:10439800F4F400084FF0B043D3F89000C0F34000A5
:1043A80070474FF0B0410209D1F8883002F47F22FB
:1043B800000123EA020300F47F201843C1F88800B3
:1043C80070474FF0B041020CD1F88830120423EA4C
:1043D800020343EA0040C1F88800704770B50568D9
:1043E80015F48035044638D0FFF7B8FAFDF7CAF956
:1043F800644E05463368DB0529D54FF0B043616B41
:10440800D3F8902002F44072914214D0D3F890105F
:10441800D3F8902042F48032C3F89020D3F890204B
:1044280021F4407022F480328D07C3F89020C3F83D
:10443800900000F196804FF0B042616BD2F8903056
:1044480023F440730B43C2F89030002505E0FDF7D4
:1044580099F9401B0228CDD903252268D0070AD52F
:104468004FF0B0406168D0F8883023EA114389B230
:104478000B43C0F8883091070AD54FF0B040A168C7
:10448800D0F8883023EA114389B20B43C0F888304A
:10449800930609D54FF0B0412069D1F8883023F44C
:1044A80040630343C1F88830960502D5206AFFF7B8
:1044B80088FF2368580502D5606AFFF782FF2368E2
:1044C800190502D5A06AFFF77CFF23685A0602D5B2
:1044D8006069FFF766FF23681B0602D5A069FFF72E
:1044E80060FF2368DE0502D5E069FFF75AFF2168FF
:1044F800C80610D54FF0B042E068D2F8883023F4EF
:1045080040730343C2F88830B0F5807F02BFD36898
:1045180043F08073D3600A040ED54FF0B042206B8D
:10452800D2F8883023F040430343C2F8883018B9E2
:10453800D36843F08073D3604B0410D54FF0B0427A
:10454800E16AD2F8883023F040530B43B1F1005FA1
:10455800C2F8883003D1D36843F48033D360284647
:1045680070BDFDF70FF941F288360546FFF712FFD7
:1045780001283FF460AFFDF705F9401BB042F5D9BB
:104588006AE700BF0004005830B590F82C30012BC2
:104598004FF0020222D0194B80F82D20CA240125A1
:1045A80080F82C505C6253245C62B1F5807F046B08
:1045B80016D19A6922F488529A615A6C24F001043F
:1045C80022F000425A640463DD650C4BFF225A62F4
:1045D8000123002280F82D3080F82C20104630BDB1
:1045E800996921F408519961D96C24F0020421F0E9
:1045F8000041D9640463DA65E7E700BF002800409A
:1046080070B50B4E036B756D1D40EA07044603D564
:104618000123F365FDF709FAAB0704D50223F36517
:10462800204600F0C9F9012384F82D3070BD00BF81
:104638000028004038B50A4CE36823F02003E36003
:10464800FDF7A0F80546E3689B0601D5002038BDB4
:10465800FDF798F8401BB0F57A7FF4D90320F6E708
:10466800002800402DE9F041114DEC6814F0400499
:1046780007461AD1EB6843F08003EB60FDF782F838
:104688004FF003080646EB685B0601D4032C02D101
:104698002046BDE8F081FDF775F8801BB0F57A7FFC
:1046A80084BF87F82D800324EDE70024F0E700BFDE
:1046B80000280040104BDA6822F0800210B5DA605A
:1046C8009A699206044606D4FFF7B4FF10B1032096
:1046D80084F82D0010BD9A6922F020029A61FFF734
:1046E800A9FF10B1032084F82D00034A936943F011
:1046F80020039361EEE700BF0028004038B5044668
:10470800002847D090F82D3003F0FF021BB980F83D
:104718002C20FCF7B3FE204D022384F82D30CA2349
:104728006B6253236B622046FFF79CFF70BBAB693B
:1047380023F08E6323F04003AB6121696368AA69A3
:104748000B431343A2691343AB61D4E9022343EA41
:1047580002432B61D4E90931EA680B4322F4F85289
:104768001343EB602046FFF7A5FF78B9D4E9071398
:10477800AA690B4322F06042134362691343AB6199
:10478800FF236B62012384F82D3038BD024BFF22D2
:104798005A62FAE70120F8E70028004000230928B8
:1047A80003D840EA0310C0B270470A380133C0B2D8
:1047B800F5E700002DE9F04790F82C30012B05466D
:1047C8004FF0020069D0012385F82C304E4B85F854
:1047D8002D00DE6806F44076B6F5807F78D04C6907
:1047E800087891F8018091F802A091F82470002AC5
:1047F80055D19A6912F0400208BFCA70FFF7CEFF80
:1048080081464046FFF7CAFF80465046FFF7C6FF7D
:1048180082463846FFF7C2FF0A6ACB78224342EA4B
:10482800835242EA0A0343EA094343EA082343EA74
:104838000063354ACA205062532050628C6A8869E6
:10484800B4F5807F946945D124F488549461012497
:10485800D465B6F5807F09BFCB69136403435364FD
:1048680018BF5064284B4A681A672A6B42F0010245
:104878002A639A6942F488529A61244AD2F88030AD
:1048880043F40033C2F880301F4BFF225A620020E5
:10489800012385F82D3085F82C00BDE8F087B4F1A8
:1048A800803F07D0B4F5000F04D09A6912F0400297
:1048B80008BFCA700A6A144344EA0A0444EA004377
:1048C800C87843EA082343EA805343EA0763B0E71A
:1048D8000023AEE724F4085494610224D465B6F5A5
:1048E800807F09BFCB6993640343D36418BFD06446
:1048F800054B4A685A672A6B42F002022A639A6992
:1049080042F40852B8E700BF0028004000080058E9
:1049180090F82C20012A03464FF0020012D00A4AD0
:1049280083F82D00CA21516253215162916941F0E7
:1049380020019161FF2151620020012283F82D207E
:1049480083F82C00704700BF0028004090F82C2006
:10495800012A03464FF0020019D00D4A83F82D00B2
:10496800CA2151625321516291690A4841F080017C
:104978009161D0F8801041F48021C0F88010FF21A7
:1049880051620020012283F82D2083F82C00704703
:104998000028004000080058064B5A6D520610B512
:1049A800044603D54022DA65FDF742F8012384F86E
:1049B8002D3010BD002800407047890001F180416A
:1049C80001F531410A607047890001F1804101F524
:1049D8003141086870470000034AD2F8903043F428
:1049E8000043C2F89030704700040058034AD2F8D8
:1049F800903023F40043C2F8903070470004005808
:104A0800074B1A6822F040021A6040F441704FF4D4
:104A1800B85218605A601A6842F040021A6070472B
:104A28000000015813B50446002842D0837903F0EA
:104A3800FF0213B94271FCF7C3FD02234FF0B042E5
:104A4800A371D2F8943023F40043C2F894301A4B7F
:104A58001B681C214B43DB0C64214B430193019BD6
:104A6800F3B90121A160FFF7B7FF144AD2F89030DB
:104A780043F48053C2F89030114B9A6842F40062B4
:104A88009A604FF400629A6129B92068FFF7B8FF6D
:104A980001232371A1600123A371084602B010BD50
:104AA800019B013B0193D2F8941011F48041D6D1B7
:104AB800D9E70121F1E700BF700000200008005885
:104AC8000004005837B5174D2B6802461C20434395
:104AD800DB0C6420434314480193019B93B90120E4
:104AE8009060114C21732B681C214B43DB0C642113
:104AF8004B430193019B6BB9012090600A4BDB6823
:104B080003B030BD019B013B019383689C07E4D54A
:104B18000020E6E7019B013B0193A368DB07E9D589
:104B2800ECE700BF700000200000015837B5184DB1
:104B38002B6802461C204343DB0C64204343154882
:104B48000193019BA3B901209060124CFF232373AA
:104B58002B681C256B43DB0C64256B430193019B7D
:104B680073B9012090600B4BDB680B7003B030BD4C
:104B7800019B013B019383689C07E2D50020E4E791
:104B8800019B013B0193A368DB07E8D5EBE700BF76
:104B980070000020000001580F4B13B51B680F4C24
:104BA800182253431B0D6422534301460193626943
:104BB800019B02F0040223B902238B60012002B09A
:104BC80010BD019B013B0193606910F00200F6D013
:104BD800002AECD11046F2E77000002000040058CB
:104BE80007B50379012B0FD10A4B1B6818225343D1
:104BF8001B0C0193FFF7FAFE019B013B0193019BFC
:104C0800002BF9D1FFF7E8FE03B05DF804EBFFF7DE
:104C1800C3BF00BF70000020F8B51E468379012B82
:104C2800154604460F46DAB22DD14379012B2AD016
:104C3800022342718371FFF7D3FF0D212046FFF74E
:104C4800D5FEFFF73FFF390A2046FFF73BFFF9B2D1
:104C58002046FFF737FF2E44B5420ED12046FFF716
:104C6800BBFEFFF799FFA06801230038A3714FF03E
:104C7800000318BF01206371F8BD15F8011B204619
:104C8800FFF720FFE8E70220F6E7F8B51E4683792C
:104C9800012B154604460F46DAB22FD14379012B72
:104CA8002CD04271FFF79CFF1D212046FFF79EFE86
:104CB800FFF708FF390A2046FFF704FFF9B220463C
:104CC800FFF700FF00212046FFF7FCFE2E44B54207
:104CD8000ED12046FFF780FEFFF75EFFA068012394
:104CE8000038A3714FF0000318BF01206371F8BDAD
:104CF80029462046FFF71AFF0135E8E70220F6E7C4
:104D0800F8B51F468379012B154604460E46DAB2DC
:104D18002CD14379012B29D04271FFF761FF06F0AE
:104D2800EF03A3F1840253425341237131462046D5
:104D3800FFF75CFEFFF7C6FE2F44AF4210D1FFF726
:104D48004BFE842E02D02046FFF726FFA0680123E1
:104D58000038A3714FF0000318BF01206371F8BD3C
:104D680015F8011B2046FFF7ADFEE6E70220F6E73F
:104D7800F8B51E468379012B154604460F46DAB26C
:104D880027D14379012B24D04271FFF729FF3946F7
:104D98002046FFF72BFEFFF795FE00212046FFF780
:104DA80091FE2E44B5420ED12046FFF715FEFFF7BF
:104DB800F3FEA06801230038A3714FF0000318BF69
:104DC80001206371F8BD29462046FFF7AFFE013583
:104DD800E8E70220F6E737B50023ADF8043001AA6A
:104DE800022312210446FFF7C3FFBDF804305BBA63
:104DF800DA079DB202D5204609F0B4F9AB0702D50F
:104E0800204609F0B5F9680702D5204609F0DAF915
:104E1800290702D5204609F0DBF9EA0602D5204623
:104E280009F0DCF9AB0602D5204609F0C5F9680699
:104E380002D5204609F0A2F9290607D5EA05C5F3E7
:104E48000021204648BF012109F09EF9AB0502D593
:104E5800204609F0A9F9022301AA19462046FFF7BE
:104E68004FFF03B030BDF8B51E468379012B1546B8
:104E780004460F46DAB227D14379012B24D0427178
:104E8800FFF7AEFE0E212046FFF7B0FDFFF71AFE32
:104E980039462046FFF716FE2E44B5420ED120466D
:104EA800FFF79AFDFFF778FEA06801230038A37189
:104EB8004FF0000318BF01206371F8BD15F8011BFE
:104EC8002046FFF7FFFDE8E70220F6E7F8B51E46A3
:104ED8008379012B154604460F46DAB22BD1437964
:104EE800012B28D04271FFF77BFE1E212046FFF7D9
:104EF8007DFDFFF7E7FD39462046FFF7E3FD00217A
:104F08002046FFF7DFFD2E44B5420ED12046FFF7BD
:104F180063FDFFF741FEA06801230038A3714FF03D
:104F2800000318BF01206371F8BD29462046FFF72A
:104F3800FDFD0135E8E70220F6E7026852E8003F88
:104F480023F0C00342E8003102680029F5D102F1DC
:104F5800080353E8003F23F4000302F1080C4CE86F
:104F680000310029F3D12023C0F8843070470000B5
:104F780010B5026852E8003F23F4907342E800310C
:104F880002680029F5D10F4C02F1080353E8003FED
:104F9800234002F1080C4CE800310029F4D1C36E1B
:104FA800012B07D152E8003F23F0100342E80031FB
:104FB8000029F7D12023C0F888300023C36603678F
:104FC80010BD00BFFEFFFFEFF8B504461346D4F846
:104FD8008470202F43D161B35AB394F88020012AFA
:104FE8003DD0A06FA4F85630012500262122C4F830
:104FF8008C6084F880502165A4F85430C4F884206B
:10500800C8B1DFF860C02268C0F82CC0DFF858C00B
:10501800C0F830C0DFF854C02832C0E90DC6FEF72A
:1050280031F940B11023C4F88C3084F88060C4F89A
:105038008470012012E0236840221A62002322684B
:1050480084F8803002F1080353E8003F43F08003FE
:1050580002F1080141E800300028F3D1F8BD022030
:10506800FCE700BF79500008C1500008CD50000887
:1050780008B50346806A1B681B6813F0200317D124
:10508800A0F85630026802F1080353E8003F23F005
:105098008003083242E8003102680029F2D152E860
:1050A800003F43F0400342E800310029F7D108BD32
:1050B800FCF7F4FDFBE7704708B5806AFFF7FBFFD4
:1050C80008BD7047806A0268D0F8843010B5D0F8FF
:1050D80088409268120606D5212B04D10023A0F837
:1050E8005630FFF72AFF03689B685B0606D5222C1B
:1050F80004D10023A0F85E30FFF73AFFD0F88C30D7
:1051080043F01003C0F88C30FFF7DBFF10BD08B583
:10511800806A0023A0F85E30A0F85630FFF7D1FF70
:1051280008BD70470368DA6919682DE9F04140F64F
:105138000F0632429D68044610D1960640F19680CB
:1051480001F0200605F080573E4300F08F80036F82
:10515800002B00F08480BDE8F0411847A74EA8480E
:105168002E400840304300F08180D70709D5C80594
:1051780007D501201862D4F88C0040F00100C4F86B
:105188008C00970709D5E80707D502201862D4F8DC
:105198008C0040F00400C4F88C00570709D5E807D4
:1051A80007D504201862D4F88C0040F00200C4F837
:1051B8008C0017070BD501F02000304307D00820DA
:1051C8001862D4F88C0040F00800C4F88C0016056A
:1051D8000AD5480108D54FF400601862D4F88C301D
:1051E80043F02003C4F88C30D4F88C30002B36D030
:1051F80093060AD501F0200105F0805551EA050310
:1052080003D0236F0BB1204698472368D4F88C50FD
:105218009B6805F0280503F040031D43204620D075
:10522800FFF7A6FE226893685F0615D502F108030A
:1052380053E8003F23F0400302F1080040E8003142
:105248000029F3D1E06F38B16E4B8363FEF794F811
:1052580028B1E06F836B7EE72046FFF732FFBDE899
:10526800F081FFF72EFFC4F88C50F8E7E06E0128B4
:1052780040F08180D6067ED5C8067CD510221A62F9
:105288009A68510647D5E26F11684A6892B2002AB7
:10529800E5D0B4F85C009042E1D9A4F85E200A6831
:1052A80092062ED453E8002F22F4807243E800219E
:1052B8000029F7D103F1080252E8002F22F0010279
:1052C80003F1080040E800210029F3D103F10802A6
:1052D80052E8002F22F0400203F1080040E80021C4
:1052E8000029F3D12022C4F88820E16653E8002F72
:1052F80022F0100243E800210029F7D1E06FFEF701
:1053080006F8B4F85E30B4F85C10C91A89B22046C1
:10531800FFF707FFA3E7B4F85E108AB2B4F85E108F
:1053280089B200299BD0B4F85C10891A89B2002987
:1053380095D053E8002F22F4907243E8002000280B
:10534800F7D1314D03F1080252E8002F2A4003F14A
:10535800080646E800200028F4D12022C4F8882056
:105368002067E06653E8002F22F0100243E800208F
:105378000028F7D1CBE7D70209D56E0207D54FF43D
:10538800801220461A62BDE8F04100F06BBD10069D
:105398000BD501F0800005F40005284305D0636FA4
:1053A800002B3FF45CAF2046D5E6570611D54E06D4
:1053B8000FD553E8002F22F0400243E800210029CE
:1053C800F7D12023C4F8843061672046FCF766FCD7
:1053D80045E7150206D5480004D52046BDE8F0414A
:1053E80000F042BDD3017FF53AAF0029BFF637AFD1
:1053F8002046BDE8F04100F036BD00BF01000010B6
:105408002001000417510008FEFFFFEFD0F88820A4
:10541800222A08B5036845D15B6AB0F86010826D2E
:105428000B401370836D01338365B0F85E30013B28
:105438009BB2A0F85E30B0F85E309BB273BB0268D6
:1054480052E8003F23F4907342E8003103680029D2
:10545800F5D103F1080252E8002F22F0010203F10E
:10546800080C4CE800210029F3D12022C0F888203C
:10547800C26E0167012A12D1C16653E8002F22F0DB
:10548800100243E800210029F7D1DA69B0F85C106E
:10549800D20644BF10221A62FFF743FE08BDFCF78C
:1054A8000BFCFBE79A6942F008029A61F6E7D0F82C
:1054B8008820222A08B5036842D1596AB0F86020CA
:1054C8001140826D22F8021B8265B0F85E20013A15
:1054D80092B2A0F85E20B0F85E2092B262BB53E8A8
:1054E800002F22F4907243E800210029F7D103F13C
:1054F800080252E8002F22F0010203F1080C4CE8E0
:1055080000210029F3D12022C0F88820C26E01674B
:10551800012A12D1C16653E8002F22F0100243E895
:1055280000210029F7D1DA69B0F85C10D20644BF2F
:1055380010221A62FFF7F5FD08BDFCF7BDFBFBE77B
:105548009A6942F008029A61F6E700002DE9F84FDF
:105558000368DD69D3F800809E68D0F88820222A85
:10556800044640F0A780B0F86070B0F86890DFF8A3
:1055780050B14FF0000A06F00106B9F1000F01D052
:10558800AB0620D4B4F85E309BB2D3B1B4F868202F
:105598009A4216D9226802F1080353E8003F23F023
:1055A8008053083242E8003122680029F2D1454B85
:1055B800236752E8003F43F0200342E80031002906
:1055C800F7D1BDE8F88F2368A26D5B6A3B40137082
:1055D800A36D0133A365B4F85E30013B9BB2A4F818
:1055E8005E302368DD6969072AD0EA070AD518F40E
:1055F800807F07D001221A62D4F88C2042F0010281
:10560800C4F88C20A80708D53EB102221A62D4F843
:105618008C2042F00402C4F88C20690708D53EB1FA
:1056280004221A62D4F88C3043F00203C4F88C3098
:10563800D4F88C3023B12046FFF743FDC4F88CA082
:10564800B4F85E309BB2002B97D1226852E8003F35
:1056580023F4807342E8003123680029F5D103F16F
:10566800080252E8002F02EA0B0203F1080040E8A2
:1056780000210029F3D12022C4F88820E26E216796
:10568800012A13D1E16653E8002F22F0100243E803
:1056980000210029F7D1DA69B4F85C10D20644BFBA
:1056A80010221A622046FFF73CFD66E72046FCF709
:1056B80003FB62E79A6942F008029A6181E700BF3A
:1056C800FEFFFFEF155400082DE9F84F0368DD6968
:1056D800D3F800809E68D0F88820222A044640F03B
:1056E800A580B0F86070B0F86890DFF84CB14FF062
:1056F800000A06F00106B9F1000F01D0AB0620D46C
:10570800B4F85E309BB2D3B1B4F868209A4216D987
:10571800226802F1080353E8003F23F0805308325F
:1057280042E8003122680029F2D1444B236752E84D
:10573800003F43F0200342E800310029F7D1BDE8DB
:10574800F88F2368A26D596A394022F8021BA265B6
:10575800B4F85E20013A92B2A4F85E20DD696907C8
:105768002AD0EA070AD518F4807F07D001221A62E6
:10577800D4F88C2042F00102C4F88C20A80708D580
:105788003EB102221A62D4F88C2042F00402C4F816
:105798008C20690708D53EB104221A62D4F88C30EF
:1057A80043F00203C4F88C30D4F88C3023B120467F
:1057B800FFF787FCC4F88CA0B4F85E309BB2002BCE
:1057C80099D1226852E8003F23F4807342E80031FF
:1057D80023680029F5D103F1080252E8002F02EAF4
:1057E8000B0203F1080040E800210029F3D1202230
:1057F800C4F88820E26E2167012A13D1E16653E8D4
:10580800002F22F0100243E800210029F7D1DA69BD
:10581800B4F85C10D20644BF10221A622046FFF783
:1058280080FC68E72046FCF747FA64E79A6942F08B
:1058380008029A6183E700BFFEFFFFEFB754000834
:1058480038B5044603682169A2681D68C0690A431F
:1058580061690A437E49024329400A431A605A682B
:10586800E16822F440520A435A607A4AA169934295
:105878001CBF226A11439A6822F06E4222F43062F9
:105888000A439A60DA6A616A22F00F020A43DA620E
:10589800714A93421CD14FF0B043D3F8883003F0DB
:1058A800030343F44033A3F54033013B022B00F2DA
:1058B800C8806A4A9B5CB0F5004F40F08A80082B8C
:1058C80024D8DFE803F061C1842381232323650002
:1058D800634A934209D14FF0B043624AD3F8883003
:1058E80003F00C0343F44023E4E75A4A93420DD1F2
:1058F8004FF0B043D3F8883003F44063B3F5006F3A
:105908001AD005D853B1B3F5806F12D0012009E041
:10591800B3F5406FFAD14FF400400EE0FEF71AFDE0
:1059280058B900204FF00113A3660023C4E91C33C3
:1059380038BDFEF713F9F3E74B4865684B4B626ACD
:1059480005EB450133F81220B0FBF2F39942DDD89C
:10595800B3EB053FDAD800231946FBF721F9090212
:1059680041EA10616B080002C0182A464FF0000394
:1059780041F10001FBF714F93D4BA0F540729A4242
:10598800C4D82368D860CCE7FEF7E4FC0028C8D068
:105998006268616A354B33F81130B0FBF3F3500895
:1059A80000EB4300B0FBF2F083B2A3F110014FF615
:1059B800EF729142AAD820F00F00226880B2C3F398
:1059C80042031843D060ACE7FEF7C8F8DEE7264884
:1059D800DEE7082B9AD801A252F823F02F5A0008C4
:1059E8003B5A0008475A000815590008415A000850
:1059F800155900081559000815590008095A0008D2
:105A08004FF400406368616A184A32F81120B0FB0D
:105A1800F2F000EB5300B0FBF3F080B2A0F11002FB
:105A28004FF6EF73ABE7FEF795FC00283FF479AF2C
:105A3800E8E7FEF79FFCF8E7FEF790F8F5E70A4875
:105A4800E0E7B0F5004FF4D1FEF794FC9EE700BF05
:105A5800F369FFCF008000400038014054F500088A
:105A68000044004057F5F4070024F40064F50008EA
:105A7800FFFC0F00836ADA0710B506D50168C46A0F
:105A88004A6822F4003222434A609C0706D501681E
:105A9800046B4A6822F4803222434A60590706D5CB
:105AA8000168446B4A6822F4802222434A601A073C
:105AB80006D50168846B4A6822F4004222434A6092
:105AC800DC0606D50168C46B8A6822F4805222433A
:105AD8008A60990606D50168046C8A6822F4005227
:105AE80022438A605A060FD50168446C4A6822F43A
:105AF80080122243B4F5801F4A6005D14A68846C3D
:105B080022F4C00222434A601B0606D50268C16C13
:105B1800536823F400230B43536010BD2DE9F04173
:105B2800DDF8188004460E4615461F462268D369DC
:105B380036EA03030CBF01230023AB4201D0002047
:105B480027E0B8F1FF3FF2D0FBF71CFEC01B404531
:105B5800206802D8B8F1000F1DD150E8003F23F4A7
:105B6800D07340E80032002AF7D100F1080353E867
:105B7800003F23F0010300F1080141E80032002A48
:105B8800F3D12023C4F88430C4F8883084F8802006
:105B98000320BDE8F08103685A07C7D5C3691B0510
:105BA800C4D54FF40063036250E8003F23F4D07378
:105BB80040E80032002AF7D100F1080353E8003F1B
:105BC80023F0010300F1080141E80032002AF3D173
:105BD8002023C4F88430C4F88830C4F88C30D5E762
:105BE80073B504460026C0F88C60FBF7CBFD23682C
:105BF8001B681A07054618D423681B685B070AD573
:105C08006FF07E43009300222B464FF4800120461C
:105C1800FFF784FFA8B920230020C4F8843084F853
:105C28008000C4F88830E0660CE06FF07E43009393
:105C3800324603464FF400112046FFF76FFF002855
:105C4800DAD0032002B070BD10B5044650B3D0F8C6
:105C580084301BB980F88030FBF72CFF226824239E
:105C6800C4F88430136823F0010313602046FFF75B
:105C7800E7FD012816D0A36A13B12046FFF7FAFE04
:105C880023685A6822F490425A609A6822F02A02DD
:105C98009A601A6842F0010220461A60BDE8104076
:105CA800FFF79EBF012010BD836830B5B3F5805F54
:105CB80081654FF00001A0F85C20A0F85E20016724
:105CC80039D10369002B34D140F2FF13A0F86030BA
:105CD8000023C0F88C302223C0F88830016801F115
:105CE800080353E8003F43F00103083141E800345A
:105CF8000368002CF2D1456E84680169B5F1005F34
:105D08003AD1B0F86850954236D8B4F5805F23D1BF
:105D18002A4A2B4C002918BF22460267002280F825
:105D28008020D9B153E8002F42F4807243E8002163
:105D3800F7E7FF23CAE723B90369002BF9D07F23CC
:105D4800C4E7B3F1805F04D10369002BF7D03F2388
:105D5800BCE7A0F86010BBE7194ADEE703F10802C8
:105D680052E8002F42F0805203F1080040E8002179
:105D78000029F3D1002030BDB4F5805F12D1114A5B
:105D8800114C002918BF22460267002280F88020A3
:105D980051B153E8002F42F4907243E800210029E2
:105DA800F7D1E7E7084AEFE753E8002F42F020026F
:105DB80043E800210029F7D1DCE700BFD1560008ED
:105DC80055550008B754000815540008D0F8883015
:105DD800202B30B41FD1D9B1D2B190F88030012B2B
:105DE80019D0012380F8803000230468C3660B4B68
:105DF8009C420AD063681B0207D554E8003F43F071
:105E0800806344E80035002DF7D130BCFFF74CBF64
:105E1800012030BC70470220FBE700BF0080004033
:105E2800436E30B51BB94FF00113836630BD03686C
:105E38000A4D9A6899680A4C490FC2F342626B5C32
:105E4800615CDB00B3FBF1F3A0F86A30AB5CA25CE9
:105E5800DB00B3FBF2F3A0F86830E7E784F500084D
:105E68007CF500087047704770471FB504AB03E91D
:105E7800060090F88030012B04463AD0012380F8C0
:105E880080302423C0F8843003681A6822F00102A5
:105E98001A609A6822F440120A439A6071B95968E4
:105EA800BDF80C209DF80E0021F010011143596037
:105EB8005A6822F07F4242EA00625A601A6842F049
:105EC80001021A60FBF75EFC6FF07E420346009207
:105ED8004FF4800100222046FFF720FE38B9202326
:105EE800C4F88430002384F8803004B010BD032047
:105EF800F8E70220F9E790F88020012A03460ED03F
:105F0800012280F88020196851E8002F42F002022F
:105F180041E800200028F6D183F88000704702206D
:105F2800704710B590F88030012B04461AD0012331
:105F380080F880302423C0F8843003681A68196810
:105F480021F00101196042F000524FF00051416602
:105F58001A60FFF765FF2023C0F88430002084F81A
:105F6800800010BD0220FCE738B590F88030012B86
:105F780004461BD0012380F880302423C0F88430E5
:105F880003681D681A6822F001021A609A6822F0F4
:105F9800604211439960FFF743FF03681D602023A7
:105FA800C0F88430002084F8800038BD0220FCE767
:105FB80038B590F88030012B04461BD0012380F8B7
:105FC80080302423C0F8843003681D681A6822F0E2
:105FD80001021A609A6822F0606211439960FFF723
:105FE8001FFF03681D602023C0F88430002084F858
:105FF800800038BD0220FCE738B5084D052455F867
:10600800043B2BB9013C14F0FF04F8D1204638BDFD
:10601800DB6898470028F5D0F9E700BF7005002035
:1060280070B5264E264B96F90420264D8EB00C46A8
:1060380002284FF001018DF800108DF8052010D1CD
:106048008DF804009871DC7102F02CFD2B7803B1F7
:1060580014B1684603F0DEF81B4B049A1A600EB0C0
:1060680070BD99718DF8041000211A715971DC7195
:106078002B78C3B91F2305A88DF814308DF8182084
:1060880002F090FE20238DF8143005A833798DF89E
:10609800183002F087FE29238DF8143005A80B4B21
:1060A800069302F07FFE02F0FDFC012305A88DF89F
:1060B80014308DF8183002F075FEC7E7840500200B
:1060C8009000002062050020640500200004000103
:1060D8007FB5092301A88DF8043003F09BF8003838
:1060E800044B059A1A6018BF0120404207B05DF8BA
:1060F80004FB00BF6405002070B504460B46164932
:1061080062784A700020A2780A7208701A884A7267
:106118009A788A72DB780B746368CB60237803F013
:10612800FB030A2B03D00D4B1B68DB6A98470C4E08
:10613800052556F8043B1BB15B6A0BB1204698470E
:10614800013D15F0FF05F4D12378062B02BF054B5E
:1061580001221A7070BD00BF980000206C05002055
:10616800700500206805002070B504461048114EDF
:106178000123037063784370A3788372E368C36074
:10618800E378037623694376237943720A4B1B68C5
:106198009B6A9847052556F8043B1BB19B690BB1D0
:1061A80020469847013D15F0FF05F4D170BD00BFAA
:1061B800AC000020700500206C050020014B186819
:1061C800704700BF6405002000B58BB0012301A80B
:1061D8008DF8043002F00EFD38B99DF8080000383B
:1061E80018BF01200BB05DF804FB0020FAE700009F
:1061F8002DE9F04186B005460E46174601F036FEF9
:10620800044600287BD1FFF7DFFF01280AD03D4B69
:10621800D9799879FFF704FF6FF00204204606B099
:10622800BDE8F081DFF8E08088F80860003E18BF1C
:1062380001268DF80460354E687833798DF8123070
:10624800694602F079FC00283ED08DF8044003949A
:10625800ADF810406FF0060495E803002C4B83E876
:106268000300337988F80A30394601A803F0D8F8D2
:10627800284B059A1A6011283ED801A353F820F03C
:10628800E76200080763000801630008016300086B
:106298000163000801630008016300082162000827
:1062A800016300080163000801630008FB6200083D
:1062B800016300080163000807630008076300081A
:1062C80007630008F56200082B788DF808306B78B2
:1062D800ADF810306B6803934FF0FF34BCE70E4BFA
:1062E80000221A70E31D18BF144697E76FF00404E4
:1062F80094E76FF0050491E74FF0FF348EE76FF0F5
:1063080001048BE790000020AC00002084050020E9
:10631800BC000020640500206805002037B501F0A6
:10632800B9FD144D052455F8043B5BB11B694BB10D
:1063380055F8043C9B682BB1984718B155F8043CB4
:106348001B699847013C14F0FF04ECD1FFF754FE99
:1063580068B9094D2B7853B1084BADF80040D9788E
:10636800019422466846FFF743FF00B92C7003B03A
:1063780030BD00BF7005002068050020840500209E
:1063880030B58BB0054601F071FD0446002839D1BF
:10639800FFF71AFF012838D101A88DF8044002F050
:1063A80029FC10B14FF0FF3004E09DF80830AB42F3
:1063B80002D100200BB030BD012DF3D0022D11D039
:1063C800002DF7D1002BF4D001A88DF8085002F069
:1063D800E9FC0028E6D10E4B1B681B6B002BE8D0AC
:1063E8009847E6E7002BDDD101A88DF8085002F0A8
:1063F800D9FC0028D6D1064B1B681B6B002BD8D0C4
:106408002846EDE76FF00100D4E76FF00200D1E70E
:106418006C05002010B504468AB018B94FF0FF305B
:106428000AB010BD002301A88DF8043002F0E2FB89
:106438000028F3D19DF808302370F1E77FB50022DA
:106448000B4621498DF8072001220A7042784A70CC
:106458000446002A35D102790A721A884A729A7853
:106468008A72DB780B740369CB60C378174D8DF89B
:106478000830037B8DF80930836803932B6802A8E2
:10648800DB6A98472B689B6B13B1227E02B1984751
:106498000F4E052556F8043B1BB1DB690BB12046AE
:1064A8009847013D15F0FF05F4D10DF10700FFF7FE
:1064B800B1FF6379012B04D19DF807200AB9054A79
:1064C800137004B070BD00BF980000206C05002058
:1064D800700500206805002010B504468AB018B978
:1064E8004FF0FF300AB010BD202301A88DF804300A
:1064F80002F080FB0028F3D1024A9DF9083023708E
:106508001371EFE784050020F0B504462748284FAB
:10651800284E00230370637843703B688BB09B6AF6
:106528009847052556F8043B1BB11B6A0BB120465A
:106538009847013D15F0FF05F4D12378042B24D0AA
:106548000B2B2AD0012B1BD106231B4E8DF80430B0
:1065580001A802F04FFB194B029A5A61301DFFF750
:10656800BBFF637873B9164B75715878FFF708FF4E
:106578003B6811485B6A984763780BB905F010FED1
:106588000BB0F0BDFF237371F2E70E4B01225A7472
:10659800227A9A74627ADA74F2E76378002BEFD081
:1065A8000BB0BDE8F040FFF793BD00BFAC00002082
:1065B8006C05002070050020900000207800002065
:1065C800840500209800002000B58BB0232302909A
:1065D80001A88DF8043002F0E5FB003818BF01204F
:1065E80040420BB05DF804FBF0B5704C014691B029
:1065F8001422204608F01EF86D4B00221A70FBF793
:10660800AFFF23784068012202FA03F1014004D168
:10661800684B084607F004FFFEE7674967481A46D3
:1066280002F080F8002840F0BE80272307A88DF8E4
:106638001C3002F0B7FB624F624E634D00287AD1DE
:1066480001233B703368DB690BB1002098470623B0
:1066580007A88DF81C3002F0CDFA089B6B6107A8DB
:1066680027238DF81C3002F0C5FA089B93F84020C8
:10667800227093F8042193F806316270A370022601
:1066880007A88DF81C6002F0B5FA08994E48082250
:1066980005F0CAFE032307A88DF81C3002F0AAFAF9
:1066A80008994A48082205F0BFFE05F01BFD2B7D1E
:1066B80003936B7D0293AB7D01930022EB7D0093E6
:1066C8001146434B304607F0ABFE0F26012307A8BF
:1066D80000258DF820308DF81C6002F063FB102334
:1066E80007A88DF81C308DF8205002F05BFB0423BE
:1066F8008DF81C3007A8A3788DF8203002F052FBE3
:1067080038238DF81C3007A82369089302F04AFB48
:1067180005A920788DF8146003F094FF401B18BF7A
:106728000120A0711420FFF74FFFA07903F03EF875
:10673800284611B0F0BD28238DF81C3033681B693A
:1067480043B107A802F056FA336808981B6940F26B
:106758007C519847272307A88DF81C3002F022FBAC
:1067680050B9012307A88DF81C3002F043FA9DF8B0
:106778002030002B7FF464AF3B78002B7FF462AFAE
:10678800052207A88DF81C20089302F00BFB33683C
:10679800DB68984706236861089007A88DF81C30C5
:1067A80002F000FB6BE74FF0FF30C2E784050020E2
:1067B800680500208CF50008A8050020BC0500200D
:1067C800620500206C050020780000208000002071
:1067D800D5F5000838B50D46044610B14FF0FF3026
:1067E80038BD00F0FDFA0028F8D00A4B0A491860B5
:1067F8000A4B83620A4B1B689A6B02639A6C42636A
:106808009B69084AC2624361F22243682846984756
:106818002046E5E770050020700400202960000884
:106828006C050020D960000808B5134B134A18609E
:10683800134B1A60134A5A60134A9A60134ADA6073
:10684800134B02681A6042685A6082689A60114A5B
:10685800DA6082691A61104BC26B5A60026C196067
:106868009A601946426CDA600020FFF7B3FF0038DF
:1068780018BF0120404208BD6C0500207161000866
:10688800BC05002045640008116500080161000886
:10689800A8050020FDA500089805002051B118B1F1
:1068A800012804D000207047044B0B607047044B4C
:1068B8000B60F7E74FF0FF30704700BF000400019E
:1068C8000100010208B502F083FF002814BF6FF031
:1068D8000100002008BD08B502F0FEF8002814BF2A
:1068E8006FF00100002008BD30B58BB0FFF7F3FF53
:1068F8000446F0B903F086FE831C1DD0F8B9134D89
:106908002B685B69DBB1272301A88DF8043002F0FE
:1069180071F92B6802985B694FF4B061984703F0EE
:1069280083FE78B92CB9094B1B68DB690BB10120D0
:10693800984720460BB030BD6FF00704EFE74FF0E3
:10694800FF34ECE74FF0FF34F3E700BF6C0500209D
:10695800014B1878704700BFD0050020014B5878CC
:10696800704700BFD005002070470000024B01228D
:106978005A70024B5B691847D0050020C8000020F8
:1069880073B5234C6378002B35D008F035F866686A
:106998000546FFF713FC0644AE421BD2A37ACBB1DF
:1069A800E0228DF800208DF80130217AE368019308
:1069B80001226846FFF71CFC20F004035BB2063393
:1069C80015D114484FF47A7108F0E4F8114808F02A
:1069D800A7F8656094F83430C3B1002384F83430E4
:1069E8000D4B5B6B93B102B0BDE8704018470023B4
:1069F8006370A372EDE794F83520002AEAD094F882
:106A0800360084F83530FFF7BBFCE3E702B070BD11
:106A1800D005002008060020C800002037B5104D1A
:106A2800104CC8B1C1B10123627200222860E16034
:106A380023700D480D4B00924FF0FF3107F0C2FF55
:106A480000250B4825822022294605F001FD6570A6
:106A5800A574A58603B030BD00232B602370EFE733
:106A6800CC050020D0050020080600207569000824
:106A7800E40500202DE9F0478C4C23788CB0002BDE
:106A880053D0C2780AB9837B13B1238A0133238296
:106A9800437B002B49D0E02A47D10023A3728768A3
:106AA80097F80080B8F1220F27D8B8F1220F30D814
:106AB800DFE818F03E00F8004F0055005C00690060
:106AC800700089009800AF00C2002F002F002F002F
:106AD8002F002F002F002F002F002F002F002F0036
:106AE8002F002F002F002F002F002F002F002F0026
:106AF8002F002F00C400CC00D000B8F17E0F00F0AA
:106B0800C980B8F17F0F00F0DB80B8F17D0F00F08D
:106B1800A780A57A002D00F0578165484FF47A7157
:106B280008F038F8624807F0FBFF0CB0BDE8F087C2
:106B3800E36801220021A2721970A37AE16898180B
:106B4800A0720620C854A37AE1689818A072CA54A3
:106B5800DFE7584B01219B6A02209847D9E77B78E9
:106B680084F83630012384F83530D2E704238DF8D1
:106B780004307B78003B18BF012301A88DF808304A
:106B880002F010F9C5E77878003818BF012002F044
:106B98000DFEBEE7484E0FCE01AD0FC50FCE0FC597
:106BA80096E8070085E807007B780A2BB1D8434AA6
:106BB80012685268002AACD00CA901EB830353F881
:106BC8002C0C9047A5E77878431E012BA1D83B4BA6
:106BD80001381B6818BF012020729B68002B98D0D1
:106BE800984796E7E26801230821A3721170627A38
:106BF800057BA17AAA4228BF2A46934289D2856892
:106C08005A1CEB5CE56801334E1CA6726B54D3B278
:106C1800EDE7E3680122A27209221A70A37AE268FA
:106C2800218A581CA072D154A27A238AE1681B0ACF
:106C3800501CA0728B546CE723826AE704238DF8FA
:106C480004300DEB030002F0E5FA62E7194BDB6A4A
:106C580098475EE7194B78781B686075DB68BDE775
:106C6800037B072B7FF455AF05238DF80430B7F865
:106C78000130ADF808307B793A791B0443EA0223E6
:106C8800FA781343642253430393BB798DF8103089
:106C980001A8D8E7392201A88DF804208DF808301A
:106CA80002F080F8012384F8343032E7D005002060
:106CB80008060020C800002004F00008CC050020C9
:106CC8002A2301A88DF8043001F094FF94F80A9063
:106CD800E6689DF808009DF809509DF80A709DF82F
:106CE8000BC09DF80D309DF80E209DF80F109DF8F3
:106CF8000CE009F1010A84F80AA006F80980354E6B
:106D080094F80A903668D4F80C8009F1010A84F8DE
:106D18000AA096F803A008F809A094F80A90D4F8F5
:106D28000C8009F1010A84F80AA096F802A008F874
:106D380009A094F80A90D4F80C8009F1010A84F8A3
:106D48000AA096F801A008F809A094F80A9009F199
:106D5800010A84F80AA096F80080E66806F8098017
:106D680094F80A80E66808F1010984F80A9006F8A0
:106D780008C094F80AC0E6680CF1010884F80A8093
:106D880006F80C70A77AE66807F1010C84F80AC0C7
:106D9800F555A57AE6686F1CA7727055A07AE56864
:106DA800461CA6722954A17AE0684D1CA57242546B
:106DB800A27AE168501CA0728B54A37AE268591C2D
:106DC800A17202F803E0A4E6034807F059FE6570D3
:106DD800ABE600BFCC050020080600207047000085
:106DE80000487047C8000020064A137843F004039F
:106DF8001370054BD3F8483313B11B6903B1184717
:106E0800704700BF2006002024060020044B054AD6
:106E180093F80431022B18BF062382F89434704784
:106E280000800020240600201FB50C4B8DF80900B7
:106E380093F874208DF80A200D228DF8082093F815
:106E4800802012B10E228DF8082093F8400002A984
:106E580003F0F8FBC0B205B05DF804FB0080002029
:106E680010B50A4C04F2044007F00AFE94F81E34E8
:106E780013B1012384F81D34D4F8483323B11B69B6
:106E880013B1BDE81040184710BD00BF240600200C
:106E980010B50C4CD4F8403343F08003C4F84033A9
:106EA80094F81E3413B10020FFF7DAFF94F89534F4
:106EB80023F0220343F0220384F89534BDE8104000
:106EC800FFF7A4BF240600202DE9F041DFF8AC80CD
:106ED80098F80431022B06460D4602D0284BDB6A8F
:106EE800984702F00FFD044628B1022002F000FD89
:106EF800002002F002FD98F80431012B17D102F0AE
:106F080003FD074630B1002002F0F3FC002002F038
:106F1800F5FC3C4602F0FAFC48B1002002F0EAFC1D
:106F2800002002F0ECFCBDE8F041FFF76FBF002C39
:106F3800F9D1144C94F8942494F81E34BAB90BB1CE
:106F480084F84564304602F091FED8F82C0007F02A
:106F58005DFDD4F8B4339842E5D30B4807F090FDB3
:106F680094F8953443F0200384F89534DBE70BB1AB
:106F780084F84554284602F079FEF1E700800020A5
:106F8800C0FC000824060020BC09002073B5164C7C
:106F9800164D04F57A766B6C95F8482095F97010C3
:106FA80095F84000009603F073FB95F81C3184F8BF
:106FB800FC3395F8400040F2012304F58562314620
:106FC800A4F8FA3303F070FB58B194F8283484F825
:106FD8006E34074B00205B6B984794F8FB3384F8BA
:106FE800943402B070BD00BF240600200080002049
:106FF800C0FC00080A4A137843F0020310B5137066
:10700800084BD3F8483313B11B6903B19847BDE85F
:107018001040054B01220021022007F001BA00BFF1
:107028002006002024060020FFF500080A4A1378ED
:1070380043F0080310B51370084BD3F8483313B165
:107048001B6903B19847BDE81040054B0122002198
:10705800022007F0E5B900BF200600202406002022
:107068000FF600082DE9F04116461D4680460F46EA
:1070780007F0C2FC0D4A0E4C1378278123F0110348
:1070880043F0110313700B4B6681D3F84833257313
:10709800C4E9000813B11B6903B19847BDE8F04182
:1070A800054B01220021022007F0BAB92006002072
:1070B800D40B0020240600201FF6000837B507F07F
:1070C8009BFC104B104D18606C46204607F0E8FBFF
:1070D80094E803000D4A05F54E7383E8030013781E
:1070E80043F020031370D5F8483313B11B6903B17B
:1070F8009847074B01220021022003B0BDE8304029
:1071080007F08EB9E40B002024060020200600209A
:107118002CF60008F0B5484C484DB4F8CC2022872E
:10712800D4E92A0194F8A52084F8612004F16402C6
:1071380082E80300D4E92C0191B0012304F16C0228
:1071480082E80300A4F80C31B4F8B8208DF81830A0
:1071580004F5F273A4F874200393D4F8BC20A26752
:1071680004F5F4730026D4F8C0200493344BE26786
:1071780084F81C61A66284F8076184F83A6084F890
:10718800096184F80A6103A9C5F89C64A5F81C6420
:1071980085F81E64059394F8400003F061FA636E65
:1071A800C5F8D43394F8753085F8E03394F8803016
:1071B80085F8E1334FF48073A5F8E23385F8D0639E
:1071C80094F81C3185F8E43305F574770FCF05F58D
:1071D8007A740FC497E8030040F2012384E803009F
:1071E800A5F8FA33D5F8483385F81F64CDE9016668
:1071F8001BB15A681B6901920293124B0793A3F1C2
:1072080048020892A3F1140209920F4A0B922933FB
:107218000A93A2F194030C93A2F190030D93131D0A
:107228000E9301A902F1480307A802F592620F9391
:1072380002F05DFB11B0F0BD0080002024060020A4
:10724800440B0020900A0020D4800020F8B52F4D70
:1072580095F80441012C064646D0022C4CD034B98E
:1072680038B9D5E9190105F16C0383E80300032453
:1072780038E0012838D00228F9D1254F85F80401D3
:1072880007F5747EBEE80F0007F57A7CACE80F00BE
:107298009EE8030095F8DA308CE8030087F8FB6372
:1072A800C3B1D5F8F030EB66C7F8EC3395F8753014
:1072B80095F8F42087F8F83395F8803085F8702031
:1072C80087F8F93397F81F2487F8E82340F2013349
:1072D800A7F8FA33002387F81E340E4BDB6A984769
:1072E800FFF754FE2046F8BD02F017FB04460028BD
:1072F800F8D185F80461F5E70028B8D1054B85F881
:107308000401DB6A98473446ECE700BF00800020A0
:1073180024060020C0FC00082DE9F04192B0074681
:1073280002F0F0FA002840F05781AC4D95F804318E
:10733800012B09D02B6BAA4C9BB194F80431C3B133
:10734800042B71D0032603E002F0DEFA20B10F26E9
:10735800304612B0BDE8F08102F0D8FA0028E9D032
:10736800F5E7B5F80C31D4F82024013B53432B63DF
:10737800E3E79C4803F09DF8002840F0298194F841
:107388000C3123802B6B0C930DF1180895F83930CC
:107398008DF83830404695F808318DF83A3007F0C6
:1073A800A5FAD5F81431009302AE98E80600D5F88E
:1073B8001031304607F031FA96E803000FAB83E846
:1073C8000300EB6A0D9300238DF844302388ADF851
:1073D800463095F81C3101228DF839201BB98DF8FB
:1073E80044208DF83930804B0093804B95F840004D
:1073F800A3F179020CA903F09AF90646C0B10B284B
:10740800A6D1002FA4D0D4F8981459B1D4F8403399
:10741800774843F02003C4F8403307F0BBFB7448B7
:1074280007F07EFB002693E76E4803F076F8A3E7A3
:1074380095F8408095F9613095F9392095F87510DF
:107448006C4F404603F080F9009741B26B6C95F899
:1074580048204046183703F01BF900976B6C95F9E4
:10746800681095F8400095F8482003F011F9D4F811
:10747800DC03696DD4F8C4732B6D0144C4F8B413EC
:1074880095F81C113B44C4F8B03339B9AA6DEB6DBB
:107498003A440344C4F8B023C4F8B433002308932F
:1074A80081B108A802F0FEFA00284CD195F93900FC
:1074B80094F837729DF82080FFF7B6FC474480B2F5
:1074C800B8423ED300238DF8133095F839308DF843
:1074D800213095F838308DF82230AB6F0993EB6F77
:1074E8000A932388ADF82C3095F81C3194F81F7452
:1074F8008DF82E3095F840003F4B8DF820700DF137
:10750800130208A903F0D8F8012384F8453495F844
:10751800393084F846349DF8133084F84734D4F869
:107528002034C4F85474C4F84C34C4F85C3402F001
:10753800EFF950B1D4F8200402F0FCF928B1102674
:1075480006E7082604E7132602E795F80431012B1D
:1075580001D102F0F1F902F0DEF90023059394F865
:10756800043195F9395094F81F749BB1042B7FF4BA
:10757800E9AE05A802F00EFD60BB94F81C3413B107
:10758800059B013B0593174B05983A46E9B202F073
:1075980061FD02E0134802F039FDC8B994F80C31D6
:1075A8002380D4F840332178144843F00203C4F808
:1075B800403394F81C340133DBB284F81C3484F86B
:1075C80049340023C4F89C340D4B9B6A9847BFE6A6
:1075D8001126BDE61226BBE60E26B9E6008000207D
:1075E800240600202C07002030800020BC0A002040
:1075F8008C090020DC090020440A0020260600200F
:10760800C0FC0008F8B50D4F0D4C0E4E0D4607F0A6
:1076180037FA3B6B984796F8400004F5856229468F
:1076280003F042F848B194F8283484F86E34F06CCA
:107638007B6B9847EB7C84F89434F8BDC0FC000859
:1076480024060020008000200F4890F81F3480F89E
:10765800B8330E4B93F8612080F8BB2393F875205C
:1076680080F8C82393F8802080F8C92393F81C3148
:1076780080F8CC330022A0F8CA2300F56E7100F51B
:107688006070FFF7BFBF00BF240600200080002005
:10769800114890F89434EBB190F81F3480F8D03347
:1076A8000E4B5A6EC0F8D42393F8752080F8E02367
:1076B80093F8802080F8E12393F81C3180F8E433B4
:1076C8004FF48072A0F8E22300F5747100F566703B
:1076D800FFF798BF704700BF2406002000800020F5
:1076E80070B5344C2421204604F0B4FE636A9842F5
:1076F80018BF60624FF014012F4814BF0125002500
:1077080004F0A8FEE36B984218BFE0634FF0E00175
:107718002A4818BF45F0020504F09CFED4F8203131
:10772800984218BFC4F820014FF0BC01244818BF84
:1077380045F0040504F08EFED4F8E031984218BFF5
:10774800C4F8E0014FF000011E4818BF45F00805D5
:1077580004F080FED4F8E431984218BFC4F8E4017C
:107768004FF45E71184818BF45F0100504F072FE1A
:10777800D4F86035984218BFC4F860054FF014017A
:10778800124818BF45F0200504F064FED4F8783597
:1077980098420F4B18BFC4F87805D3F8483318BF80
:1077A80045F040052BB1DB681BB12846BDE87040A9
:1077B800184770BD008000202880002040800020ED
:1077C80024810020E4810020E881002064850020D5
:1077D800240600202DE9F04F91B04FF00008012B4E
:1077E80005460F4602928DF81580ADF8188003D82B
:1077F800C94EC146B94502D311B0BDE8F08F15F89E
:10780800090002F0A1F94844B842F5DC15F809303E
:1078180009F10104023BE4B2112BEDD801A252F8A0
:1078280023F000BF75780008A7780008AB79000836
:10783800D57900085D7A0008857A0008F77A00088B
:10784800297B0008B57B000801780008017800084A
:10785800137C00080178000801780008D17C000832
:10786800F97C00083D7D00087B7D0008042002F0BB
:1078780017FA90B10421002002F0D6F92A5DA74B2F
:1078880009F1030409F102095FFA89F983F8602410
:1078980015F8092083F86124E4B2A146AAE7002379
:1078A8008DF816308DF817308DF81C308DF8203093
:1078B800B8F1000F70D14FF0050896F874208DF8D4
:1078C8003920631E96F839208DF83B202B4496F812
:1078D80038200D938DF83C2096F8063196F86020F4
:1078E8008DF83D20D6F818218DF83A300C9273B3F4
:1078F8007B1C1B1BDBB28DF8383008AB019307AB40
:10790800009396F840000DF117030DF116020CA92B
:1079180002F0DEFE8DF8150000F00700072813D1ED
:1079280096F939209DF9163086F839309A429DF833
:10793800173086F83830B8BF01229DF81C30B8BF20
:1079480086F8092186F860304FF0000909E0052320
:10795800D1E701220DF11501032001F0FFFF09F124
:1079680001095FFA89F29DF82030B3FBF8F19142E2
:10797800EFD81C44E4B204F1FF395FFA89F94F45A6
:1079880006D915F80930032B97D0A74298BFA1460E
:107998004C464FF0010880E709F105095FFA89F9BB
:1079A800F6E72B5D012203F00F0309F1020986F8BF
:1079B800073102FA03F35FFA89F9A6F80C310022BD
:1079C80006A9042001F0CAFF4C4666E707238DF894
:1079D80015302B5D96F84000C3F3021203F00F0335
:1079E8008DF831208DF8303009F1040209F10303D4
:1079F800DBB2D2B209F1050409F10209E95CAB5C1A
:107A08005FFA89F91B0415F8092043EA0123134397
:107A1800642253430CA90D9302F069FE00F007039A
:107A2800072BE4B28DF815000CD19DF8303086F89C
:107A3800683086F870300D9B7366F3669DF83130B8
:107A480086F861308DF81800012206A9052001F09A
:107A580085FF22E7314BD3F848336BB11B685BB124
:107A68009847029B8DF8180003F03F038DF81930F2
:107A7800022206A90620EAE7FF20F2E703238DF891
:107A880015302B5D8DF824300CAB089309F10402F6
:107A980009F10303DBB2D2B2E95CAB5C96F84000B3
:107AA80009F10202D2B21B04AA5C43EA0123134380
:107AB80009F10604642209F1050953435FFA89F9BB
:107AC8000C9300230D9308A915F809308DF8383068
:107AD80002F013FEC3B20028E4B28DF81530FFF6A9
:107AE800DCAE8DF81830012206A90720AFE72B5D20
:107AF80003F00F03012B4FF47A7238BF012353436D
:107B080009F10209336513445FFA89F973650022A4
:107B180006A9082056E700BF0080002024060020A0
:107B28002B5D96F8400000228DF81C2013F02002EF
:107B380018BF01228DF81D20DA0648BF012203F084
:107B48000F0307A948BF8DF81C208DF81E3002F0DE
:107B5800DAFD09F1020901305FFA89F93FF434AF1F
:107B68009DF81D30914A86F875309DF81E309DF8B5
:107B78001C40D05C86F87440F8F724FE0223B067F6
:107B88000CA996F840008DF830308DF8324002F09C
:107B980059FD96F93930089040B29842B8BF184656
:107BA80086F83900002206A909200BE703238DF87F
:107BB80015302B5D8DF8303009F1040209F103030B
:107BC800DBB2D2B209F1050409F10209E95CAB5C48
:107BD80096F840005FFA89F91B0415F8092043EA72
:107BE80001231343642253430CA90D9302F091FD22
:107BF800C3B20028E4B28DF81530FFF64EAE8DF80A
:107C08001830012206A90A2021E7092002F048F8C5
:107C1800DFF89CA1002854D00921002002F004F8C4
:107C28000023ADF8263009F1030209F10203DBB2A3
:107C3800D2B2E95CAB5C2A5D1B0443EA012313431F
:107C480009F10402D2B209F1060409F10509AA5C96
:107C58005FFA89F943EA026315F8092003934FF4A0
:107C68007A714A430DF1300B12125846ADF82420B0
:107C780006F016FE039B03F1965303F5A91303F5CB
:107C8800EC530893DAF83C3300930DF1200999E896
:107C98000600DAF838330AA806F0BFFD0B9B0093FC
:107CA8009BE806000A9B484606F09CFD99E80300FD
:107CB80006F0CEFD01F03BFE0123E4B28AF83C3425
:107CC800EBE58AF83C04E8E50C2001F0E9FF002820
:107CD8003FF4E3AD0C21002001F0A6FF344B93F8EC
:107CE8009434043B012B7FF6D8AD01F01CFED4E59B
:107CF80009F10202D2B2295DA85C09F10302D2B2ED
:107D080009F10504AB5C09F104095FFA89F91B0460
:107D180043EA002315F809000B436421594300F096
:107D28000F0001F001FEE4B28DF81800012206A947
:107D380011208CE60D2001F0B3FF00283FF4ADAD13
:107D48000D21002001F070FF09F10203DBB2194A8E
:107D5800E85C2B5D126809F1040409F103095FFA74
:107D680089F943EA002015F80910E4B201F0DEFDB4
:107D780093E5285D09F1020309F1040409F10309F7
:107D8800DBB25FFA89F9EA5C15F809301B0443EAAB
:107D9800022303436420584301F0CAFDE4B28DF87E
:107DA8001800012206A9132051E600BF39F6000881
:107DB80024060020D40B00200E4B93F8952492073C
:107DC80003D593F89324012A08D90B4991F8062181
:107DD80022B18A6A501C18BF01328A620022A3F8B5
:107DE8001C2483F81E24D3F8402322F00202C3F88F
:107DF80040237047240600200080002070B5194CED
:107E080004F55A7006F03CFED4F84033D4F89C04CC
:107E180023F02003C4F8403350B1134DD5F88460E3
:107E280006F0F4FD864203D2002385F83A3070BD8F
:107E38000120FFF771FA0028F9D00B28F7D00A4B78
:107E480093F8393084F84634092094F81C3484F8BF
:107E5800493484F8450401F009FFBDE87040FFF794
:107E6800ABBF00BF2406002000800020074B1B7812
:107E7800DB0709D4064BD3F840232AB993F89604B4
:107E8800013818BF012070470120704720060020E4
:107E9800240600202DE9F04FA9B0EFF3108272B646
:107EA800DFF8F0820021D8F80030C8F8001082F31B
:107EB8001088B94C002B00F0D980DAB29E060392E4
:107EC80059D5B64D95F80431022B02D0B44BDB6A74
:107ED8009847D4F8B013B34806F05CFEB14806F0F2
:107EE8001FFED4F8B413B04806F054FEAE4806F0AE
:107EF80017FE94F81E34002B00F07781152312A981
:107F080095F840008DF8483002F09CFBD4F8B41383
:107F18000F900144A54806F03DFEA44806F000FE77
:107F2800A34B94F81F241B68EB620DAF38468DF8FD
:107F380070201D9306F0DAFCD5F81431009306AED4
:107F480097E80600D5F81031304606F066FC96E84A
:107F580003001FAB83E80300D4F820341E9395F880
:107F68001C3195F84000002B18BF01231CA98DF87F
:107F7800713002F070FB039BDD064BD5874DDFF8AF
:107F880034A2D5F8D420BAF90A30059298F800201E
:107F98000493002363F300020A9388F8002084F80E
:107FA8004834049AA4F8263484F82934C4F82C34C4
:107FB800A4F8303484F83234C4F8343484F82434DF
:107FC800C4F8383484F83C34C4F84034744B9AF913
:107FD8000C90A4F8902494F89424DB6A84F8929482
:107FE80084F89324DAF80470BAF80860984794F88B
:107FF800933413B96C4806F043FD3146384601F016
:108008007FFC8346002800F0F380049BA4F88234A8
:1080180084F88494039B19071AD5604B93F80431AC
:10802800022B02D05E4BDB6A98470220FEF7EEFE79
:1080380084F8450401F01AFE94F81E3413B10123A4
:1080480084F81D3494F8953443F0200384F895346B
:10805800039B5A0703D506210520FEF735FF039B2E
:108068009B0703D504210320FEF72EFF01F066FCD1
:1080780094F89524970668D5002384F89634D4F8A4
:1080880040331E0644BF23F08203C4F8403312F085
:10809800050F00F0E0820B2001F002FE002800F03E
:1080A800DA8294F89534DD0700F1D582580740F15B
:1080B800EE82D4F8403323F00203C4F84033D4F8F6
:1080C8004023002A38D194F8955415F001011EBFB9
:1080D8002B4662F3000384F8953494F895345E07D0
:1080E80044BF6FF3820384F89534012384F89634EF
:1080F80021B1D4F8443330481B6898476D070BD535
:108108002E4801F0D9FD01F001FE28B194F895340C
:1081180043F0040384F8953401F0FEFB94F8953499
:108128006FF3451384F89534D4F8403323B91CA869
:108138008DF8703001F0F4FC012384F8963494F83B
:10814800953443F0400384F8953494F8953418072F
:108158000AD56FF3C3031A4984F89534D4F8443325
:10816800A1F12400DB68984794F8953499070AD55B
:108178006FF34103124984F89534D4F84433A1F1DC
:108188006C005B68984794F89434022B1AD1FEF778
:10819800FDFE17E0200600202406002000800020B5
:1081A800C0FC0008A4090020BC090020280A0020FF
:1081B800E40B0020D40B0020680A00207C0A002071
:1081C800B40A002094F895345A0640F1A3826FF35C
:1081D800861384F89534D4F84033002B40F09A8203
:1081E80029B0BDE8F04FFFF77BBA84F8453497E62D
:1081F80095F80421012A0CD101F086FB8046C0B114
:10820800584601F076FB584601F078FB042384F8C1
:1082180093343B7804935B09013B062B00F20782F9
:10822800DFE813F01300050294000502910005022F
:10823800F60101F06BFB0028EBD0404601F05AFB39
:10824800404601F05CFB0523E1E7102E03D801232B
:1082580084F8253420E195F81C311297F6B28DF890
:108268004C60002BF3D104F0B7F812AA0146FF20A6
:1082780002F004F800285ED19DF853309DF8522092
:108288001B0443EA02239DF851201343C5F8D0305C
:10829800159BC5F8D4309DF85830C3F30212C3F3C8
:1082A800030385F8683085F870309DF8593085F8F3
:1082B8006120002B3DD02B652B6D95F840004FF4C5
:1082C8007A7253432B6513446B650DF15A0310936F
:1082D800002794F81F348DF83C30113E0FA985F81B
:1082E8001A718DF8446002F0C8F90223012085F85C
:1082F8001C3101F0D5FC18B10121384601F094FC7D
:1083080094F8953443F0080384F8953494F893343A
:10831800012B00F29A8194F81E34002B40F08D81D5
:1083280094F8953443F0200384F89534FEF76EFDF5
:1083380070E60123BFE7012001F0B2FC0028DFD07E
:1083480001210720DAE7012384F8243495F87530F1
:108358008DF82E3094F828348DF82D300D238DF8B3
:108368002C3095F8803013B10E238DF82C3095F809
:1083780040000BA902F066F9A6F10D031BB20990A3
:1083880023EAE37300B283423FF761AF0B2E7FF617
:108398005EAFBB4B25931CA8FF238DF874601C9718
:1083A8008DF8983002F02AF8064600287FF44FAF7F
:1083B80095F80431012B13D101F0A6FA00286ED0EC
:1083C800304601F096FA304601F098FA04239DF8F9
:1083D8007C101E9884F89334C1F3001101F0ADFAB3
:1083E8009DF87C301E99C4F8381413F00F0203D09E
:1083F8009DF8900000285ED19DF8980000285CD078
:10840800002A7FF424AF9DF89020002A0CBF022791
:10841800032700220A92D5F8DC2091424FD195F823
:10842800DA1000294BD0D5F8F81095F8DBB00968B8
:108438000A9195F80411022902D1032184F89314B2
:10844800032F7FF404AF13F0600F7FF400AF0592A1
:10845800012695F81A81BBF1000F33D0BBF1010F4B
:1084680039D1B8F1010F30D197B3032F14BFD846D3
:108478004FF00208BDF87E100AAA404601F096FDAA
:1084880058B307280CBF0823012384F825340A9B16
:10849800C4F83434C4F87034FEF7FAFCBAE501F0D5
:1084A80035FA00289CD0304601F024FA304601F015
:1084B80026FA05238BE70027ABE70127A9E74FF04A
:1084C800010BC6E74FF00408D4E74FF00308D1E7E3
:1084D8004FF00208CEE70123D7E71CAB00930599BC
:1084E8000A9B4246584601F027FE20B102280CBFDD
:1084F8000A230B23ACE69DF87C3084F82504C3F3EB
:108508000012C3F3401384F8323484F8483494F8E2
:10851800933484F82924012B0A9AC4F83424C4F823
:1085280070249EBF0122A86285F80A21012E84F8D2
:108538002664C4F82C0484F8300484F8450403D174
:10854800022284F8242418E0049A02F0E002A02A07
:108558003ED195F81A11012285F83A2009B92799D0
:108568006963012B84F8242407D9D5F88420C4F83A
:108578004024DAF80020C4F89C24012B94F8441411
:108588009DF87C2005D8012901D1900601D501F07C
:1085980071FA022F94F893341ED0032F09D09DF856
:1085A8007C10012F4A4601F00F0120A818D0FFF7D0
:1085B80011F99DF8903084F82734259BC4F82C34A1
:1085C8009DF8983084F83034012384F831340DE074
:1085D800002285F83A20B4E79DF8981025984A4675
:1085E800FFF7F8F89DF8903084F827349DF890202C
:1085F800E02A08D195F80B312BB984F82724C4F860
:108608002C34A4F8303494F8953443F002037BE614
:108618001B4D013EB2B2791C284603F005FF032327
:10862800A4F82434C4F82C5484F83064EBE701230C
:1086380084F82534FEF72CFC68E694F84834002BBF
:108648003FF46EAE0020FEF70BFC94F89334022B37
:108658003FF46CAE64E694F89534590717D50120B9
:1086680001F01EFB70B1012001F0F0FA08B984F89E
:108678001C04D4F8403323F00203C4F8403306E066
:108688005C080020052001F00BFB0028F1D194F8CC
:108698009534DA077FF513AD94F844240AB1032A18
:1086A80018D11E4A94F81C1492F86020914205D201
:1086B8009B0723D594F89334012B1FD8184806F04C
:1086C800DFF9D4F8403323F02003C4F84033FFF730
:1086D80073FBF4E4012A11D194F81D24002A3FF415
:1086E800EEAC0E4A94F81C1492F860209142E5D240
:1086F8009F0703D594F84834002BDFD194F89534BC
:1087080000206FF3451384F8953484F81D04FFF7AF
:1087180075FBD4E429B0BDE8F08F00BF00800020CD
:108728008C0900202DE9F04F88468DB09146074608
:10873800002800F09181002900F08E810368002B49
:1087480000F08A814368002B00F086818368002B43
:1087580000F08281C368002B00F07E81104601F092
:108768006DFF002800F07A81BE4CBF4D384601F0FD
:1087780011FA40F27C520021204603F069FE4FF4C2
:10878800A4620021284603F063FEB84BC4F81831F0
:1087980004F5F273089304F5F47300264846099328
:1087A80008A9B34B84F840900A9384F8046184F8CC
:1087B80080608DF82C6001F053FF0F2306A994F810
:1087C80040008DF8183001F03DFF801B18BF0120D4
:1087D8004FF00A0B84F8080106A994F840008DF8B8
:1087E80018B001F02FFF4FF0060A84F8CC0006A954
:1087F80094F840008DF818A001F024FF102384F8A5
:10880800CD0006A994F840008DF8183001F01AFF41
:108818001123C4F8900006A994F840008DF8183088
:1088280001F010FF1223C4F8940006A994F8400040
:108838008DF8183001F006FF1323C4F8980006A934
:1088480094F840008DF8183001F0FCFE1423C4F8A9
:108858009C0006A994F840008DF8183001F0F2FE4B
:108868001623C4F8A00006A994F840008DF8183023
:1088780001F0E8FE172384F8A50006A994F8400043
:108888008DF8183001F0DEFE18230DEB0301C4F853
:10889800A800C4F8B00094F840008DF8183001F032
:1088A800D1FEC0B21D2384F8AC0084F8B40006A938
:1088B80094F840008DF8183001F0C4FE1E2384F8A7
:1088C800B80006A994F840008DF8183001F0BAFEF7
:1088D8001F2384F8B90006A994F840008DF81830D1
:1088E80001F0B0FE2023C4F8BC0006A994F84000AB
:1088F8008DF8183001F0A6FE0B23C4F8C00006A9B5
:1089080094F840008DF8183001F09CFE0C2306A95D
:10891800A5F8000494F840008DF8183001F092FE94
:10892800D4F89030E364D4F894302365D4F89830C0
:108938006365D4F89C30A3654FF00109D4F8A030E2
:108948000590A5F80204E36584F8A490C4F888B0FB
:1089580084F88CA0C4F844B084F848A084F86090E7
:1089680084F80B91C5F84883FEF7D4FB414B009679
:1089780032464FF0FF3105F55A70C5F84473C4E923
:108988000B6684F8059185F89564C5F8409306F060
:1089980019F8394B009632464FF0FF3105F56070F3
:1089A80006F010F8354B009632464FF0FF3105F5CA
:1089B800667006F007F802AF314B009632464FF06A
:1089C800FF3105F2044005F0FDFF384605F08EFF43
:1089D80097E8030004F5887383E80300294B2A4FBE
:1089E8001E602A4BC5F84C33294BC5F85433294B24
:1089F800C5F85C33284BC5F85033284BC5F85833B5
:108A080005F553703B689847D8F8081004F592703C
:108A180003F0AAFA20B1112630460DB0BDE8F08F58
:108A2800204601F093FA0028F5D100F089FFB8B983
:108A38001B4801F0DFFA06460028ECD17B6998470D
:108A480003F0D0FCBB6D94F805019847FB6A984782
:108A5800012385F89634DFE70326DDE70926DBE7FF
:108A68001326D9E700800020240600200004000116
:108A7800440B0020057E000851760008997600080E
:108A8800696E000820060020C0FC0008C5700008B8
:108A98006D700008F16D000835700008FD6F000862
:108AA800D8800020024B0020C3F84003704700BF65
:108AB8002406002008B5FFF7D9F9064B18B901229A
:108AC800C3F8402308BDD3F84003013818BF01207C
:108AD800F8E700BF2406002038B5134C04F55A7097
:108AE80005F0CEFF04F5607005F0CAFF04F5667066
:108AF80005F0C6FF04F2044005F0C2FF00F00BFFCA
:108B08000A4B0025DB6A9847C4F84053FEF7E8FD96
:108B18000749084840F27C5203F086FC0123C4F858
:108B28004033284638BD00BF24060020C0FC00089A
:108B3800008000207C850020F0B52C4B8BB093F88A
:108B4800CD208DF8092093F8CC208DF80A20284AEA
:108B58009E6A03960546002792F81C048DF80B00C0
:108B680004970C4600293DD0D2F8002407921A8FAA
:108B780093F806118DF8151052BAADF8202093F825
:108B8800742093F840308DF8243003AB8DF8220020
:108B98008DF8232000930DF10A020DF10B030DF15E
:108BA800090105A88DF81470069600F033FE9DF9AA
:108BB8000900FEF739F9607004A800F073FF98B94E
:108BC800049B0F2B0AD86278934207D8D11A2B44FA
:108BD80021709A4238BF08200BB0F0BD00232370E3
:108BE8000820F9E70320F7E71320F5E700800020C5
:108BF800240600201FB50446002800F0C480007831
:108C0800392800F2BA80DFE800F01D23282D30341F
:108C180039B8B8B8B8B8B8B8B83D41454F56595C36
:108C2800615F63676A6D7073768589918D95989C8D
:108C3800A4A0A2B8A8B8B8B8B8B8B8B8B8B8B8B8FE
:108C4800B8B8B0B4514B93F80431237104B010BDD7
:108C58004E4B93F81C31237102E003F0A7FB6060D0
:108C68000020F3E703F0B8FBF9E7484B93F8063127
:108C7800F1E7464BD3F8D0306360F1E7434BD3F8C4
:108C8800D430F9E7414B93F80531E4E73F4B93F8CB
:108C98008030E0E71C238DF808303C4B02A993F89C
:108CA800400001F0CFFCDAE7394B043493E80300C5
:108CB80084E80300D4E7374B0434F7E7364B043431
:108CC800F4E7364B0434F1E71A23E4E71923E2E723
:108CD8002E4B93F86030BEE72C4BDB6CCCE72B4B6C
:108CE8001B6DC9E7294B5B6DC6E7284B9B6DC3E736
:108CF800264BDB6DC0E702238DF80830234B02A911
:108D080093F8742093F840008DF80A2001F09AFC3B
:108D18002071A5E71D4B93F8CD309CE71B4B93F8CA
:108D2800393098E7194B93F8CC3094E7174B93F800
:108D3800383090E7154B5B6C9EE7144B93F848303E
:108D480089E7124BDB6F63608AE7104B94E7144B9B
:108D580092E70E4BD3F8C030F5E70C4BD3F8183137
:108D6800636001F0FDFCA0607AE7084BD3F884301B
:108D780082E7064B93F80B316DE7204604B0BDE857
:108D8800104000F0CCBD032060E700BF0080002049
:108D980064800020A88000206C800020B080002023
:108DA8007C8500207FB5044610B9032004B070BD4F
:108DB800A44DD5F840339A0700F126820278392A63
:108DC80000F21F82DFE812F03A0040004E00540023
:108DD80058005D0062006700710077007D00830025
:108DE80089008F0095009B00A5001D02AA00CC00F9
:108DF800DF000601280119012C0135013901440160
:108E080048014C011D02500162018A0178019C0150
:108E1800A201A901AD01B2011D0207021D021D0236
:108E28001D021D021D021D021D021D021D021D0242
:108E38001D021D021D021D02130218020079FEF711
:108E480005FA0028B2D105E00379022BADD07E4A9D
:108E580082F81C3195F8953443F0400385F8953431
:108E68000020A3E7406803F093FA0028F2D09CE7BB
:108E7800406803F0A1FAF8E7734B027983F80621FA
:108E8800E8E7714B4268C3F8D020E3E76E4B4268CD
:108E9800C3F8D420DEE74168002986D0002001F01D
:108EA800D7F90028D6D0112080E7416800293FF47F
:108EB8007CAF0120F3E7416800293FF476AF022038
:108EC800EDE7416800293FF470AF0320E7E7416808
:108ED80000293FF46AAF7F20E1E7416800293FF4A9
:108EE80064AF8020DBE7416800293FF45EAF812052
:108EF800D5E7416800293FF458AF8220CFE7534CAB
:108F0800514B007983F80501A36D9847E36A9847A8
:108F1800A0E74D4B027983F880209BE74A4E037AFD
:108F28008DF8043096F8400096F875308DF80530C5
:108F3800072201A901F099FB00283FF436AF6368C6
:108F480096F840000193002201A901F08EFB002849
:108F58003FF42BAF6436D4E9010186E8030079E7D2
:108F6800394E037A8DF8043096F8400096F875303B
:108F78008DF80530072201A901F077FB00283FF49E
:108F880014AFA836E7E7304E037A8DF8043096F828
:108F9800400096F875308DF80530072201A901F0D8
:108FA80064FB00283FF401AFD4E9010106F16C032A
:108FB80083E8030096F80431022B7FF44BAF96F850
:108FC8001C31002B3FF446AF204BDB6A9847FDF776
:108FD800DDFF3FE71C4E037A8DF8043096F8400019
:108FE80096F875308DF80530072201A901F03DFB90
:108FF80000283FF4DAAEB036ADE7436802930123A8
:109008008DF80C30104B02A993F8400001F03AFBA0
:1090180000287FF41FAFC8E6436802930023EFE7F8
:1090280003795A1E0E2A3FF6C0AE074A82F860300E
:1090380010E7054B4268DA640CE7034B42681A658F
:1090480008E700BF2406002000800020C0FC0008BC
:109058006E4B42685A65FDE66C4B42689A65F9E6C4
:109068006A4B4268DA65F5E6684C037994F8400083
:109078008DF80430062201A901F0F7FA00283FF420
:1090880094AE9DF8043084F8CD30E3E65F4C037964
:109098008DF8043094F8400094F874308DF8063058
:1090A800052201A901F0E1FA00283FF47EAE9DF8FF
:1090B800043084F83930CDE6544C037994F84000F4
:1090C8008DF804300A2201A901F0CFFA00283FF4F4
:1090D8006CAE9DF8043084F8CC30BBE64B4C037979
:1090E80094F840008DF80430092201A901F0BDFA76
:1090F80000283FF45AAE9DF8043084F83830A9E6C9
:10910800424B4268C3F888205A64A3E63F4B027971
:1091180083F88C2083F848209CE63C4B4268DA6749
:1091280098E63A4B4268C3F8C02093E6012B6BD10E
:10913800374C2421204603F08DF9636A984201D008
:10914800172033E6142104F1280003F083F9E36BB8
:109158009842F5D1E02104F1400003F07BF9D4F8FE
:1091680020319842ECD1BC2104F5927003F072F9D9
:10917800D4F8E0319842E3D1002104F5F27003F00D
:1091880069F9D4F8E4319842DAD1142104F2645030
:1091980003F060F9D4F878359842D1D11B4E40F2EB
:1091A8007C522146304603F03FF940F27C520021C0
:1091B800204603F04DF995F81F3485F8E833F36E2F
:1091C800C5F8EC3396F8753085F8F83340F201238A
:1091D800A5F8FA333EE68379012B3FF6E6AD0B4B53
:1091E80042684068C3F8182100F0CCFE59E6074BE6
:1091F8004268C3F884202DE6044B027983F80B21DA
:1092080028E600F08EFB1CE60120CFE50080002058
:109218007C8500202DE9F04387B00023ADF80030AD
:109228000646002800F0F0800361FEF71FFE20B11B
:109238000124204607B0BDE8F08300F06DFD00284A
:10924800F6D100F063FD014618B97048142203F006
:10925800FFF86F4D95F89534012243F0040385F823
:10926800592485F8953433788DF804300021013B72
:109278008DF805208DF807108DF806100C2B00F2DC
:10928800BB80DFE803F007B9B97F88B9B9B996B9E7
:10929800AD9AA900D5F8404314F02007C8D196F834
:1092A8000480B8F1020F4AD1DFF868815A4CFDF703
:1092B80031FF96F9051098F840003A4601F02FFA68
:1092C800072388F8390038468DF80530FDF7BEFFCA
:1092D800FF23A5F80C31C5F8084185F8047103F09F
:1092E8007BF80822014604F5867003F09DF803F028
:1092F8005DF80822014604F58A7003F095F83846AF
:10930800FEF70AF8044640B196F9051098F84000AF
:10931800012201F004FA88F83900D5F8983433614D
:10932800002C6DD000F0F2FC002882D195F895341D
:1093380085F81E0460F3820385F8953479E7B8F15F
:10934800010F4FF00204E8D1DFF8C8908DF81440FF
:1093580099F8400089F8097102A901F081F9337977
:1093680089F81C31D5F848338DF805701B698DF8DC
:109378000680984795F8953443F0200385F895348E
:109388000024CAE700226946022000F0E7FA002814
:10939800F6D01324C1E7214BB288DB6B96F90C1089
:1093A800B0689847D5F8403343F00203C5F8403316
:1093B800E6E7002269460D20E7E7164B93F80431EB
:1093C800D3B9347904F0070000F0A4FA8DF800400E
:1093D800012269461020D8E7002269461220D4E706
:1093E8008DF8072000F087FA044638B900F080FAB3
:1093F800204600F082FA90E702248EE701248CE7E9
:1094080001A800F0DBFB14E7032412E77C0A002024
:10941800240600200080002026060020C0FC00084A
:109428002DE9F04F9BB08046079118B903201BB077
:10943800BDE8F08F00230361FEF718FD04460028FD
:1094480040F0AA8046460FCE10AD0FC55A4D98F889
:1094580000A0B8F80C7098F90EB0142205F2444038
:10946800214602F0F5FF012285F84524534D95F871
:109478001C21022A26460BD195F80421022A07D17D
:1094880095F80A2122B9BAF1010F38BF4FF0010A45
:10949800BAF1010F2CD0BAF1030F2BD0BAF1000F9B
:1094A80034D102229DF84430DDF84890029362F3EB
:1094B8004716012495F874108DF83A1002220EA967
:1094C80095F840008DF8382001F0BCF895F80611A1
:1094D80040B20222002973D095F81C31012B67D1C4
:1094E80095F80931002B63D1002C6ED1104627E086
:1094F8000422D7E70023DDF84490BDF848709DF9B1
:109508004AB0029366F01F060124D3E74FF0000B20
:10951800D946CDF808B0CDE74FF0010184F81E1404
:10952800E0E007F29E420DA900F0C8FA002800F01A
:1095380023811320059B33871F4B002283F81E24A9
:109548001D4BD3F89834C8F8103070E707F29E47DF
:109558003A460DA900F0B2FA0028EAD10D9B84F82A
:109568002801C4F82C7184F8303105E1B9F1000FF5
:1095780000F00281002A00F0FF804946E01C02F05A
:1095880053FF94F8373201332380F5E01220D1E7F6
:109598000220CFE70720CFE7012048E7064B93F8E2
:1095A800952483F844A442F0010283F89524C7E780
:1095B800F4B90220C4E700BF240600200080002080
:1095C800002C93D05845B8BF584695F874308DF89C
:1095D8002800052295F840008DF82A300AA901F0E4
:1095E80044F800283FF422AF9DF8283085F8393038
:1095F8006A4BD3F89C0440B1D5F8844005F006FACC
:1096080084423CBF002385F83A302A8F2B8F95F887
:109618001C110592AA6A0B925BBA0029BAD095F878
:10962800071101B9296395F80611039195F80411FA
:10963800ADF86030481E95F860308DF862304142D0
:1096480095F87430554C8DF86330414195F84030A9
:1096580006918DF8643095F83A1004910BAB4FF0F1
:1096680001011692D4F8002400934D4B8DF8541044
:1096780003998DF855101792A3F12701A3F1280239
:1096880015A800F0C7F8069B049A4FF0000B1B01C1
:10969800D94543EA4213039AA4F800B008BF5F46CD
:1096A80043EA801343EAC21349463A4604F59C70DC
:1096B8001D460393CDE90CBB84F81EB402F0B4FE3A
:1096C800C6F34211FAB20429F0B2A670039B354ED4
:1096D80084F837223FF420AF07293FF447AF022927
:1096E8007FF456AF0421304F84F80411FF2184F829
:1096F8000C11029984F80D0184F8281184F81431AA
:10970800D6F8D410C4F8087107F59B730CA8C4F8F0
:10971800101184F83021C4F82C3100F03BFC0028EB
:109728007FF434AF0C9BA4F848040DA8A4F81631B4
:10973800C4F8503400F0B6F900287FF4FAAE0D9B57
:10974800D3B196F93900FDF76FFB94F83732002B47
:109758003FF4FCAE0D9B0F2B3FF6E3AE07F58B7283
:109768000DA90F2000F0AAF900287FF4E2AE0D9BA6
:1097780063F3030584F814510798FDF7CDFD00281D
:109788007FF4D8AE0B9B86F83A00B36200F064F918
:1097980000283FF403AF1320CEE600BF24060020C4
:1097A80060800020008000202606002037B5074D85
:1097B8008DF8040004460F2295F8400001A900F036
:1097C80054FF08B185F8084103B030BD008000207F
:1097D80010B5FFF76FF9044688B90A4805F050F943
:1097E800094805F04DF9094805F04AF900F093F8E1
:1097F800FDF790FC064BDB6A9847204610BD012414
:10980800FBE700BF8C090020A4090020BC09002048
:10981800C0FC00082DE9F04F8BB047780093149BEB
:1098280090F90C8090F90D6090F80E908B46416885
:10983800196004469246002F57D002238DF8103045
:1098480004A9C37B007C8DF8123000F0FBFEB4F84D
:1098580008C0618943B26068984545466144B8BF0D
:109868001D46604534BF00270127884209D30A21D5
:109878008DF81010207C019304A900F0E3FE019BF1
:1098880046B2B4F808C0608961680CEB400E7145B7
:1098980020D3A1EB0C01B1FBF0FC00FB1C11C9B9F2
:1098A80098450ADC237833B10223207C8DF82430D4
:1098B80006A900F0D5FE4FF0010921238DF81030DC
:1098C800207CE37B8DF8115004A98DF8123000F04C
:1098D800B9FE45B2009B8BF8005038468AF8006004
:1098E80083F800900BB0BDE8F08F4546F2E770476B
:1098F800704770477047002070477047704770473F
:1099080000207047002070470020704700207047F3
:109918000020704770477047704702207047022048
:1099280070470220704770470020704770477047A3
:10993800002070470020704770477047704700004C
:1099480010B5054C4FF403722046002102F080FD4B
:109958000020C4E9000010BDE80B00202DE9F84301
:1099680080461646002940D0234B002403F1010C01
:1099780018462201103310F8017FC7BB9842FAD16C
:109988001E4D2B680BB9C5F800C06B680BB1C3F846
:1099980000C0AB184FF000090134C3F8089083F8F1
:1099A8000C8002F10D002301B2B22844EE50C5F834
:1099B80004C002F039FDB8F1110F14D8104B012082
:1099C80000FA08F818EA030F14BF03464B4605EBE4
:1099D80004142371D5F8083201331E44C5F808620F
:1099E8003846BDE8F8834B46F1E70127F8E701342C
:1099F800202CBBD10227F3E7EF0B0020E80B002057
:109A08002007020010B510B3124A1368984204D117
:109A180003681360002304E00B4613B119688842F9
:109A2800FAD15168884208BF53600BB101681960C8
:109A3800D2F808328168013B00245B1A0460214691
:109A4800C2F80832102202F003FD204610BD0120A2
:109A5800FCE700BFE80B002010B5054B186800B9FB
:109A680010BD037B04680BB9FFF7CCFF2046F6E76F
:109A7800E80B0020094B70B51868094D012400B99E
:109A880070BD03790668112B05D804FA03F32B423D
:109A980001D0FFF7B7FF3046F1E700BFE80B002021
:109AA8002007020028B1044BD3F8083203600020D5
:109AB80070470120704700BFE80B00202DE9F041F6
:109AC80007460E46154632B329B3144B1C680023CB
:109AD8002CB93046FFF7E6FF0020BDE8F081A26808
:109AE800F91A013291420FD32279EA54581C22897B
:109AF8005FFA80F8611D55FA80F002F095FCA368C2
:109B080024684344DBB2E3E720462468FFF77AFF82
:109B1800002CF9D1DDE70120DFE700BFE80B0020CA
:109B2800034668B1074A106800221A7000B97047E6
:109B3800027B1AB101221A70002070470068F5E70D
:109B480001207047E80B00200238C0B211289ABFE4
:109B5800014B185C0020704749F6000830B50B4BE4
:109B680093F820200446084672B100211C3305787A
:109B7800A54208D001319842CDB20CBF0448043048
:109B8800AA42F4D8002030BD1046FCE7F40D0020AE
:109B9800000E002010B5084C00232060142204F1A8
:109BA8000C00FF2184F82030C4E9010002F050FCC9
:109BB800012384F8213010BDF40D002010B50E4AA1
:109BC80092F82010042915D8936804781C704478FA
:109BD8005C70C478807898700131DC7082F820104D
:109BE80002F11C018B4214BF043302F10C03936091
:109BF800012010BD0020FCE7F40D0020094B93F86C
:109C0800200068B15A6803F11C018A4200F1FF3054
:109C180014BF043203F10C0283F820005A600120BB
:109C2800704700BFF40D002010B5074B93F82020B3
:109C38000446084632B15968FFF790FF10B1012376
:109C48004470837010BD00BFF40D002008B5064BAA
:109C580093F820202AB15968FFF780FF08B14078AF
:109C680008BD0120FCE700BFF40D002030B50A4A0A
:109C780092F82010536882F8210061B1916801249C
:109C88001C32DD78587005B99C7093420CBF034BA9
:109C980004339942F5D130BDF40D0020000E0020A8
:109CA80008B5044B5968FFF759FF003818BF012061
:109CB80008BD00BFF40D00202DE9F341124E96F8BF
:109CC800208004460025EBB2984502D802B0BDE8D2
:109CD800F0817368197821705A7862709F785FB143
:109CE800336820469B689847FFF788FF17B901A893
:109CF800FFF764FF0135E6E7DB788DF804108DF88F
:109D080005208DF80730EFE7F40D0020014B93F89C
:109D180020007047F40D0020034B93F8200004281E
:109D280094BF002001207047F40D00201FB50024C7
:109D3800CDE90244441E8DF800408DF801100C0A4C
:109D4800090C8DF803108DF80420110A120C8DF8F7
:109D580005108DF806208DF8073002461B0A0121F0
:109D680068468DF802408DF8083002F0B2FA0028F3
:109D780018BF0E2004B010BD2DE9F04188B0174679
:109D88000D460F9A0646002853D000240121CDE93C
:109D980004448DF810109DF838108DF81510190A24
:109DA8008DF816308DF81710190C1B0E8DF8193018
:109DB800CDE90044130ACDE902448DF81A208DF844
:109DC8001B30130C120E07948DF818108DF81C30E8
:109DD8008DF81D20E3B24FEA0318002D5FFA88F8CA
:109DE80003DC002008B0BDE8F081013310218DF8B4
:109DF8001F303A466B460DEB010002F0FFF90346AF
:109E0800C8B9102DAC46A8BF4FF0100CDAB26245A5
:109E180003F1010303DB103D2DB20134DAE708EB4F
:109E2800020020326A44315C12F8202C4A40325435
:109E3800ECE70920D6E70E20D4E71FB500237F22E0
:109E480004216846CDE90033CDE9023302F041FA36
:109E5800002818BF0E2005B05DF804FB0138032860
:109E68001CD8DFE800F0020A10160D4B1B681A69AF
:109E78000A601A691A6200207047094B1B685A6900
:109E88000A605A69F6E7064B1B689A690A609A697C
:109E9800F0E7034B1B68DB690B60ECE705207047B4
:109EA800180E00202DE9F043C5B00C464C9E904694
:109EB8001D468146002845D0B1F5807F44D84FF42F
:109EC80088720021684602F0C3FA49238DF80030F1
:109ED80001238DF805302B0A8DF807302B0C8DF8EF
:109EE80006508DF808302D0E330A00278DF80950DA
:109EF8008DF80B302246330C494604A8350E8DF8F0
:109F08000C308DF801708DF802708DF803708DF8A3
:109F180004708DF80A608DF80D508DF80E708DF86C
:109F28000F4002F081FA04F110014D9A434689B2BC
:109F3800684602F04DF910B1012818BF0E2045B04F
:109F4800BDE8F0830920FAE70D20F8E710B590B1D5
:109F58000A4C28220021206002F07AFA2368084A75
:109F68001A6000204FF0FF32C3E90302C3E905225B
:109F7800C3E9072210BD0820FCE700BF180E002027
:109F880000010101024B1B6818600020704700BFE8
:109F9800180E002030B1044B1B68DB6801330360E6
:109FA8000020704709207047180E002037B500239D
:109FB8000D4601931446D2B101A9FFF74FFF18B916
:109FC800019B5A1C02D1256003B030BD9AB2AA1A6F
:109FD800002A02DD13442360F6E702D1236007203C
:109FE800F2E71B0C1B0403F580332B44F3E709202D
:109FF800EAE7000028B1044B1B681C330362002009
:10A0080070470920704700BF180E002013B504469A
:10A01800C8B10F4B1A68938801339BB29380C382EF
:10A0280000F047FA60B904F118030093216801238E
:10A03800132202F0C4F840B9204600F03AFA00B101
:10A04800102002B010BD0920FBE70E20F9E700BF81
:10A05800180E0020F0B5054687B01C4623B3354ED0
:10A068003368DB68834263D894F82020002A14BF41
:10A0780003220222834205D3204600F04EFA70B133
:10A0880010200AE0002301900093A36894F8281098
:10A09800606AFFF771FE0028EED007B0F0BD27799F
:10A0A8002168043FBAB209B90920F6E7B2F5807F02
:10A0B8003CD8A3688DF80E304FF0490C8DF808C0D5
:10A0C8004FEA132C8DF80FC04FEA134C1B0E8DF876
:10A0D80011302B0A8DF813302B0C8DF814302B0E01
:10A0E8008DF8153004F12C038DF809008DF80A005D
:10A0F8008DF80B008DF80C008DF80D008DF816000A
:10A10800009302A802238DF810C08DF812508DF824
:10A11800177002F054F808B10E20BEE7204600F090
:10A12800FCF90028ACD13368DD60B6E70D20B4E750
:10A138000620B2E7180E00202DE9FF410A9D80464F
:10A148000F4616461C46002D59D0002303A9104679
:10A158000393FFF783FE18B1062004B0BDE8F08131
:10A16800039B9C4201D80133F6D1284600F046F9FA
:10A17800002846D1264B1A78424503D01A79424521
:10A1880041D10120AA68BA423FD103EB8000EB6AB3
:10A1980090F801802979CDE900430439827828684C
:10A1A8003B4689B2FFF77EFE0028D6D195F82030CD
:10A1B8000194002B4FF00103009314BF4246022282
:10A1C80095F82810686A3B46FFF7D6FD0028C4D1E9
:10A1D800013E032EC1D8DFE806F002060A0E0D4B39
:10A1E8001B681C61B9E70B4B1B685C61B5E7094B41
:10A1F8001B689C61B1E7074B1B68DC61ADE7092070
:10A20800ABE70F20A9E70B20A7E70220A5E700BFCF
:10A2180000010020180E00201FB5B1B90128CDE9B2
:10A22800001108BF2023CDE902114FF004024FF0BE
:10A238000001684608BF8DF8003002F04AF800288F
:10A2480018BF0E2005B05DF804FB0A20FAE70000ED
:10A2580038B5054602F038F8044650B955B9064BEA
:10A268001B6801469878FFF7D7FF10B9FFF7E5FD9F
:10A2780000B10E24204638BD180E00202DE9F04309
:10A2880080468FB00D461446002A5FD000295DD065
:10A29800002631461D2206A8059604F013FE8DF807
:10A2A80013602E4E33680DF114099F88CDF8049081
:10A2B8000DF1130302932379009323683A46294644
:10A2C800404602F022F8002842D149462279206807
:10A2D80002F0AAF8204600F043F80146002839D1D8
:10A2E800257AE279A3792D0445EA02251D433368CE
:10A2F8009A68AA4230D09DF813009D60FFF78CFF42
:10A3080008BBFFF79AFDF0B9627AA37AE47A2404CD
:10A3180044EA032414433B46224629460320FFF718
:10A3280005FD80B93B46224629460220FFF7FEFC80
:10A3380048B933689DF813209A704FF0FF32C3E98B
:10A348000422D8609A610FB0BDE8F0830920FAE7CB
:10A358000E20F8E70F20F6E70320F4E7180E002098
:10A3680010B50446002845D00168002942D011F8EC
:10A37800013B43710322063002F056F820460322BF
:10A3880050F8091B043102F04FF82168CB79E360DB
:10A398000A7A43EA0223E3604A7A43EA0243E36023
:10A3A8008A7A43EA0263E360CB7A23740B7B637493
:10A3B8002379212B1AD110220D3104F1120002F059
:10A3C80033F81D222168501C8B5C6362085C43EAE9
:10A3D8000023901C6362085C033243EA0043636213
:10A3E8008A5C43EA02636362002010BD112B03DC20
:10A3F8000D22E7E70220F8E70120F6E710B504464A
:10A40800002854D00168002951D00B7843714B784B
:10A4180083608A7843EA02238360CA7843EA024366
:10A4280083600A7943EA026383604B7903738B790B
:10A43800C381CA7943EA0223027BC38102F00F0277
:10A448000831103001F0F0FF237B002203F00F03E6
:10A4580084F8202084F82820227903F10800111AB2
:10A4680004290DDD21680933043AD21A085C84F8FE
:10A478002000D2B2606A84F82820194401F0D4FF81
:10A48800237922681A44002012F8043CE36212F887
:10A49800031C43EA0123E36212F8021C43EA014366
:10A4A800E36212F8012C43EA0263E36210BD022062
:10A4B800FCE710B5044660B3036853B30279162A63
:10A4C80029D942791A700146082251F8060B013041
:10A4D80001F0B4FF2146082251F80E0B093001F0B3
:10A4E800ADFF2368E28A5A74E38A22681B0A9374D0
:10A4F8002368A269DA74A36922681B0A13752368A2
:10A50800628B5A752368E27E9A751723237100209F
:10A5180010BD0120FCE70220FAE738B50446002800
:10A5280063D00168002960D0037B90F8282003F0ED
:10A538000F03002A57D10833207904321344984274
:10A5480055D363790B702368A2685A70A368226890
:10A558001B0A937023686289DA702368E27A1A7199
:10A568002368227B5A712368E2899A71E3892268F9
:10A578001B0A2146D371227B51F8100B02F00F02FF
:10A58800083001F051FF237B94F8282003F00F03D3
:10A5980003F108052AB1226894F82010515503F1F7
:10A5A8000905206894F82820616A284401F03CFFD6
:10A5B80094F828302268E16A2B44D1545A1CE16A85
:10A5C800206892B2090A81549A1C2168E08D92B2DF
:10A5D8008854DA1C216894F82F0092B20433885406
:10A5E8002371002038BD0933A6E70120FAE70220CD
:10A5F800F8E70000024B1A8810431880704700BF24
:10A608001C0E002008B5074B1B883BB1FEF752FA19
:10A6180000280CBF00206FF0020008BD6FF0010099
:10A62800FBE700BF1C0E002010B5034B00241C8064
:10A63800FEF738FA204610BD1C0E0020B0FA80F054
:10A648004009704782B018B9084602B000F0CAB88D
:10A65800002002B0704710B9084600F079B9704779
:10A6680010B9084600F090B97047034608461146ED
:10A678000BB900F0DDB90020704710B9084600F0AA
:10A6880041BD704710B9084600F0FEB90020704778
:10A6980010B40446084611461A46019B14B910BC6A
:10A6A80000F010BA10BC70470346084611460BB9B3
:10A6B80000F03ABA0020704710B404460846114624
:10A6C8001A4614B910BC00F0ADBA002010BC70478F
:10A6D80030B40546084611461A46DDE902341DB96C
:10A6E800029430BC00F02CBB002030BC704710B97D
:10A6F800084600F0DDBB0020704710B9084600F09E
:10A708003FBD0020704710B9084600F0EFBB00209D
:10A71800704710B9084600F0EBBB002070470346AD
:10A72800084611460BB900F001BC0020704710B470
:10A738000446084611461A46019B14B910BC00F09D
:10A74800F7BB092010BC704710B4044608461146F0
:10A758001A4614B910BC00F033BDC8B210BC70471B
:10A768000048704701000102064B10B51B6A0446F9
:10A77800984730B10448054B204498428CBF0020CC
:10A78800012010BDC0FC0008403576C9405DC600F8
:10A79800F0B5114B85B00C4610491F56054601F01F
:10A7A8001DF80F4BE4B25E6A072D4FF00103CDE9A7
:10A7B800024301460AD105220023CDE900234FF4C4
:10A7C8007A727A431846B04705B0F0BD08220020D7
:10A7D800CDE900203A46F5E783F600085CF6000864
:10A7E800C0FC00081FB5002300930378013B372BFA
:10A7F80000F28180DFE803F01C227F7F7F1F7F7FCC
:10A808007F7F3F41434A7F5255585B5E617F691F96
:10A818006B7075777A7F7C83247F7F7F7F7F7F7FD4
:10A828007F7F7F7F7F7F85878C7F7F858C7F8E92E0
:10A83800C378002B5FD0022300935CE08378F8E7AD
:10A8480043788DF8043007238DF805308378002B82
:10A858000CBF002302238DF8063010238DF8073033
:10A86800314B1B6801A803F55872CDE9022300F0AB
:10A8780096FF00903FE04023DEE72023DCE7827864
:10A8880090F9013042B9294AD35CD5E7827890F92A
:10A8980001300AB9264AF7E7264AF5E740F6B83301
:10A8A800CAE74FF47A73C7E74FF4FA63C4E741F293
:10A8B8008833C1E741F27073BEE71F484FF47A71DD
:10A8C80001F096FD00F5FA60D3E71C4BB4E7164B90
:10A8D8001B6803F55873AFE7134B1B6803F55B73ED
:10A8E800AAE71023A8E7104B1B68A5E70123A3E7F5
:10A8F8004FF083430093009805B05DF804FB104BBC
:10A90800F8E7104B98E740F21113ADF80030F2E782
:10A91800032391E790F901300B4AB5E70B4990F909
:10A92800010000F05BFFA4E7240E00200BF70008ED
:10A938001BF7000813F7000818FCFFFF00EA0637AA
:10A948009A99094040F7093783F600085CF6000831
:10A9580037B50B4B02781B680C2101FB02335B7A7D
:10A9680003EB4304074B1D6803690093C3684278EF
:10A97800816805EBC40000F0B2FC03B030BD00BF35
:10A98800240E0020200E002030B587B0027B6423FF
:10A99800ADF80030012A4FF00003CDE90133CDE9CD
:10A9A80003338DF802308DF8143028D0022A2FD0C6
:10A9B8001ABB03680BB34368FBB11A4C8068236069
:10A9C800194B18226946186001F02EFD174B2468B0
:10A9D80093E807000C3384E8070093E8070004F1C4
:10A9E8000C05032385E80700A4F86C33012204F55D
:10A9F8005B7104F5587000F063FC07B030BD09497D
:10AA080008684360036100F55B7100F55870F2E770
:10AA1800044B1B68B3F86023B3F86C130A43A3F81C
:10AA28006023EAE7240E0020200E002030F0000802
:10AA380008B503460A2924D8DFE801F006232323B2
:10AA4800230B161B23212100BDE808400068FFF7EF
:10AA58008BBE90F900009978072271B900F0F0FBDD
:10AA6800003818BF012008BD052293F90000002115
:10AA7800F4E790F900005978EEE70221EEE70722A3
:10AA8800F3E70020EFE7000010B504791CB1012CB2
:10AA98000BD0002010BD0A4B01681B68012203F58A
:10AAA800587000F00DFC0120F4E7054B01681B68A5
:10AAB800224603F55B7000F003FC2046EAE700BF7E
:10AAC800240E0020F7B50728144D1C46A8BF072000
:10AAD80058700E462946174600F080FE94F901305A
:10AAE800A070072B13D1322000F078FD0C4BDB6DE2
:10AAF8000546984704F10C02083403460192009475
:10AB08003A463146284600F06EFD03B0F0BD054ACE
:10AB180055F82310D05C00F059FDE7E75CF6000813
:10AB2800C0FC000883F600082DE9F04FDFF8DC9040
:10AB380090F90160D9F80430D0F804808BB004464D
:10AB48008A469847054600285DD1E37C63B9304AB8
:10AB58002378126803EB430302EB830152F8238046
:10AB68004B68002B18BF98462A4B404613F906B08D
:10AB7800D9F80C309847D9F81830A1689C46072EA8
:10AB8800A37C09932BD189B2002302912249069311
:10AB98000522CDE90733CDE9001201204FF47A727E
:10ABA800CDE90430039302FB0BF24CF25031184606
:10ABB8006746B847637C23B3184B995DD9F854307E
:10ABC8000D31C9B228469847E07C3246414600F02C
:10ABD80017FE8AF8006001200BB0BDE8F08F00274F
:10ABE800012589B20823CDE900730291CDE90775E3
:10ABF800CDE90577CDE90377A1782B465A46284653
:10AC0800D6E7074BD9E70020E6E700BFC0FC0008FD
:10AC1800240E002083F60008854501001BF7000874
:10AC28000BF700082DE9F04F8DB090F90130DFF8EF
:10AC3800FCA0DFF8FC90CDE90A123E4A12F903B0F5
:10AC48000278DAF800300C2505FB02333A4A5B7AC1
:10AC5800126803EB430302EBC303044693F90210A3
:10AC680090F9020000F0B6FD3449064694F9010057
:10AC780000F0B4FDA26861688046304600F0DCFC54
:10AC88002378DAF800205D430746D9F80C3050598C
:10AC98009847D9F81C309C4694F901300025072BB9
:10ACA8004FF47A63CDE90753CDE905552DD101233A
:10ACB800CDE903530523CDE901534FF47A7303FB20
:10ACC8000BF300933946434646F2A81228466746D6
:10ACD800B8472378DAF800200C214B4394F9011087
:10ACE800D05800F0AFFDA18994F90100FFF750FD9D
:10ACF8000B9B217B1860D9F85430284698470A9B4B
:10AD080001201E700DB0BDE8F08F01200823CDE9A9
:10AD18000350CDE901032A46CDF800B06546434605
:10AD28003946A84701200546D3E700BF240E002076
:10AD3800C0FC000883F60008200E00205CF600081E
:10AD48002DE9F04F8FB0002405468A469146984673
:10AD58000494ADF81440ADF8024007264FF0010BFB
:10AD68002B7AA34206D9686804A9204400F0C8FBDE
:10AD780000285DD102238DF8083002A86B7A8DF87F
:10AD88000A30FFF72FFDAB7A8DF81D309DF8113092
:10AD98008DF81E309DF812308DF81F309DF8103058
:10ADA8008DF82030EB7A8DF821302B7B8DF822300E
:10ADB8006B7B8DF8233010238DF81C608DF82430C0
:10ADC8003A4E8DF82C000DF102030A9307233268DE
:10ADD8008DF82D30ADF834302B680C9206930DF1B8
:10ADE800120204AB0DF1110106A800F0A3FB07281D
:10ADF80005460BD130680C22002100F5587001F08F
:10AE080027FB3368BDF80220A3F860239DF81130B2
:10AE18008AF800309DF8123089F800309DF810301B
:10AE280088F80030189B28461C700FB0BDE8F08FDA
:10AE38009DF81330BDF81470ADF802700444E4B204
:10AE4800F3B917B3194A00201168072602464FF0D4
:10AE58000C0C062B1BD10CFB00FE51F80EE0BEF1CA
:10AE6800000F04D00BFA00F21743BFB201220130E1
:10AE78001028EED1002A3FF473AFADF802706FE7E7
:10AE88005A1E042A01D9062BDCD0062668E747FAA1
:10AE980000FE1EF0010FEAD00CFB00FE51F80EE098
:10AEA800BEF1000F08BF0626E1E700BF240E002010
:10AEB80038B505464068FFF757FC072200284FF0D1
:10AEC800000195F9000014BF0724062400F0B8F922
:10AED80008B904F0050495F901000722002100F0E3
:10AEE800AFF908B904F0FB04204638BD00207047CC
:10AEF80010B504464068FFF737FC23780A4A03EB8D
:10AF08004303126802EB830152F82330002814BF70
:10AF18000320022013B900F0010010BD032806BF6A
:10AF280063684B600220F8E7240E00200220704777
:10AF38002DE9F0413A4D0446286896B00E469046F1
:10AF480000211F460122032300F55870CDE90411A2
:10AF5800CDE906118DF80C108DF80D10ADF80E30F6
:10AF680000F090F930B92A68B2F8603343F003036F
:10AF7800A2F860332A68637A8DF8203002F5587198
:10AF8800CDE90912274A94F9083012680B92102269
:10AF9800ADF830200DF10E020D9222680E92626813
:10AFA8000F92D4E90301A27A8DF8402001228DF88E
:10AFB800412011AA82E80300227DE18A8DF8213020
:10AFC80018468DF84C20FFF7E3FB08AB15930DF1FD
:10AFD8000D0314900093CDF8048003AB04AA3946FE
:10AFE8000EA800F098FB044678B99DF80C100139BA
:10AFF80001F0FEF900F158030DEB030010F8483C8E
:10B008003370204616B0BDE8F0810C2801BF2A68CD
:10B01800B2F8603343F00303A2F86033F1E700BFEE
:10B02800240E0020200E0020F8B50679012E0546D2
:10B0380001D80620F8BD0F2E2BD80368187A40F3E4
:10B0480003000722002140B200F0FAF82B680446FA
:10B05800187A40F303100722002140B200F0F0F8FC
:10B06800A8B1B4FA84F4640929680B7A086843F330
:10B07800030243F3031352B25BB29A42C8BF0124DE
:10B08800FFF772FB48B9002CD3D10420D2E7012482
:10B09800EAE70320CEE70520CCE7002CFBD10C4FD4
:10B0A80029683B6806EB460003EB80000C2201F0A0
:10B0B800BBF93A680C2303FB062320465C72012384
:10B0C80003FA06F6B2F860331E43A2F86063B1E7EC
:10B0D800240E002010B4017801290ED9084B1868F5
:10B0E8000C234B43C4180022C250C4E9012200F5C6
:10B0F800587010BC102200F0ACB8002010BC70478B
:10B10800240E00202DE9F04186B050238DF814302C
:10B11800037A102B074630D14368DD7B6DBB0224D0
:10B12800A8466426062C14D87A68535D03932A44EB
:10B13800517843EA01230393927843EA0243734325
:10B14800CDE9033863B968468DF80040FFF7C2FFC0
:10B158000DE0CDF80C808DF81480CDF81080F2E762
:10B1680003AB01A801938DF80840FFF75DFF013498
:10B17800E4B2102C05F10305D4D106B0BDE8F08186
:10B188001FB502680379116851B901A88DF8043018
:10B19800FFF7A0FF78B9002040B205B05DF804FBC6
:10B1A80002A802928DF80C30FFF73EFF0628F2D86D
:10B1B800024B185CF0E70320EEE700BF7CF60008BE
:10B1C800C90020B9034B19448856C0B27047024BD6
:10B1D800F9E700BF8BF60008CBF60008F0B59A42F5
:10B1E800069E03DB9DF914309A4225DD0020F0BD50
:10B1F80003EB430331F814E006EB830300274EFA10
:10B2080007F5ED070CD593F808C04CF303150CF0BF
:10B218000F0C62456DB203DB05F00F05AA420DDD88
:10B228000137102F03F10C03E9D10134E4B22301F3
:10B23800DBB29842DCD8D9E70024F8E70120D6E74A
:10B24800884204DB9042CCBF0020012070470020D8
:10B25800704710B51409B4EB111F03464FEA1110DB
:10B268000ED391420CD202B201F00F0133F8124012
:10B27800012000FA01F124EA010123F8121010BD9F
:10B288000020FCE7F0B528B100EB410501260020BD
:10B29800914200D3F0BD002435F8027B234606FA1C
:10B2A80004FC3CEA070C08BF013304F1010408BFA1
:10B2B800DBB2102CF3D118440131C0B2C9B2E7E7B0
:10B2C80010B500B149B910BD31F8134020F813404A
:10B2D8000133DCB2A242F7D8F5E70023F9E782B0E0
:10B2E80030B5048804936AB9B3F5616F18D349F689
:10B2F800AF2542F21072AB4298BF4FF47A72944273
:10B3080038BF1446012CC36838BF01244C43A342FC
:10B318008CBF1C1B0024C460BDE8304002B07047DD
:10B328006422ECE72DE9F04F91B01546DDF86C800A
:10B3380004939DF8683009930C46064603F05CFBBD
:10B34800684ADFF8A4B10590A8F5F633303BB3FBA3
:10B35800F2F3534303F5F632303203F5A83303F51D
:10B36800C07306921822039312FB05430893002525
:10B378004FF0FF3A089BA34207D1002D14BF504657
:10B388004FF0FF3011B0BDE8F08FBDF97030ADF867
:10B398002C300B99CDF86C804046CDF8288003F00E
:10B3A800BBFAB4F800906EB9B8F5616F5BD349F693
:10B3B800AF2242F21073904598BF4FF47A739945C3
:10B3C80038BF99464B46012B38BF01230793002EFF
:10B3D80052D1B9F1640F48D1A0605F46A1680EA8A8
:10B3E80003F0BCFA0F9B0093DDE90A120E9B0CA830
:10B3F80003F013FA049B0BB9099B33B12369BB42D1
:10B4080003D13A4B0C9A9A420DD9394BE7609845CB
:10B4180009D90023ADF83430069B0D990C931846D2
:10B4280003F07AFAA060606800B9E760276126B186
:10B4380003F0ECFAE3680344E360D4E9033293428F
:10B44800059B1D996360079B88BFE2604B43E168D9
:10B45800994202D80498A8B9A6B101231D442375BE
:10B46800EDB2183486E76423A9E7B9F57A7F0ABFF5
:10B47800204F214FA060B1E7049B0BB9C4F80CB072
:10B488005F46D0E700209342207506D25B1A9A45A2
:10B4980005F1010528BF9A46EDB2002EE1D1B9F1B8
:10B4A800640F164AADF8346019D049F6B023B9F5DF
:10B4B8007A7F18BF1346904584BF039A9B180C9354
:10B4C8001C9B00930CAF97E806001B9B384603F0C3
:10B4D800A4F997E8030003F01FFA8246C1E74FF486
:10B4E8006163E8E78051010040771B007F5101004C
:10B4F8002FEC010080A81201002E930230EC01000D
:10B508000378032B14D1437803F00F021B098A70C8
:10B518004B7083788B80C27843EA02238B8003794F
:10B52800C3F3021203F00F03CA700B7005207047B3
:10B53800002070472DE9F34798464379057990F93B
:10B548000770067A9146044690F906208A467BB130
:10B5580076B275B30F2A12D194F909200F2F1ED194
:10B5680094F90A70072D24D1002E08BF012620E087
:10B5780090F90B6090F9092090F90A70E9E7A3693E
:10B58800019394F915300093216994F91430207BC4
:10B59800FFF724FE0028E1D105F0FD05DEE794F968
:10B5A8001D3094F91C10BB420DDCB942DADA05F003
:10B5B800FB0528468AF8002089F8007088F80060A2
:10B5C80002B0BDE8F0871F46CCE70000024B03FA43
:10B5D80000F0B0FBF1F0704740420F004FF4FA530F
:10B5E800B3FBF0F0704730B54FF47A750C1F6A431F
:10B5F80000FB042252001EBF00F1FF341219B2FBF7
:10B60800F0F28A4238BF0A468400504318BF01301E
:10B61800039918BF40080A60201A4FF47A7202FB97
:10B6280013000028049BD2BF90FBF2F000F2E73031
:10B63800B0FBF2F0186030BD38B5400014460D4636
:10B64800F5F7C0F801462846F5F70AF82146F5F758
:10B6580007F8F4F7F9FE03F03FFCF4F7D5FF40B222
:10B6680038BD2DE9F74F019300231F469C461C0166
:10B67800058A5FFA84FE04F0F004A54206D8019B0F
:10B6880082F800C01F7003B0BDE8F08F0EEB4E05C6
:10B698004FEA4309AD000024466836F809602641A0
:10B6A800F60727D5866806EB050A765916B3067895
:10B6B80036B9466926B136F809602641F60719D524
:10B6C8009AF8086090F901B046F303084FFA88F831
:10B6D800D8450FDC46F3031676B25E450ADB9AF8C6
:10B6E800096006EB4608C66806EBC806367D4EB903
:10B6F8000137FFB20134102C05F10C05CCD1013310
:10B70800DBB2B4E70CF101060EEB040801F80C807B
:10B718005FFA86FCEEE72DE9FF4704464068DDE95D
:10B728000C671D468A46914603F070F923681B1A78
:10B738003B604FF000080123337085F80080636890
:10B7480013B12368834224D8CAF80080D4F81CC0F7
:10B75800A3699CF800E00393D4E9030101AB83E8F3
:10B768000300237D0093DCF80C10237A627A70467C
:10B77800FFF7D8FD334638602A46E0694946FFF7A7
:10B7880070FF2B782BB1C7F80080002004B0BDE80B
:10B79800F0873378002B14BF0B200C20F6E737B561
:10B7A80090F9002090F90250954204460FD0013AD2
:10B7B80052B295420BD0A368019394F901300093DB
:10B7C8006168E0782B46FFF709FD0028EFD01046A6
:10B7D80003B030BD8842B8BF0846704751F8200012
:10B7E800054B984205D0054B98420CBF022000201B
:10B7F80070470120704700BF90D0030020A10700C8
:10B8080005281FB50ED80C4B53F820300093CDE90E
:10B8180001120A4B01220021022002F001FE05B0AC
:10B828005DF804FBCDE90012054B0122002102203E
:10B8380002F0F6FDF3E700BF8CF7000823F70008D5
:10B8480042F7000807B5054BCDE9000101220021A8
:10B85800022002F0E5FD03B05DF804FB5EF7000886
:10B8680010B5102204460021F13000F0F1FD00214E
:10B87800C4F814112046F022BDE8104000F0E8BDDD
:10B8880002460846102100F09DB92DE9F043044610
:10B89800D0F8140185B00E46154604F2011788B396
:10B8A800C0F110099145C84628BF90461FFA88F292
:10B8B800384400F0B9FDD4F8143143440F2BC4F8D0
:10B8C800143128D9A94526D204F1F103994613F871
:10B8D800012BD97BBB4282EA010203F8012CF6D185
:10B8E80010224946684600F09FFD22466946684690
:10B8F80000F0E4F910226946484600F095FD4644F8
:10B90800A5EB0805102D09D8AAB23146384600F033
:10B918008BFDC4F8145105B0BDE8F08304F1F103C0
:10B92800711E98461A7811F8010F424003F8012B4E
:10B93800BB42F7D110224146684600F075FD224609
:10B948006946684600F0BAF910226946404600F098
:10B958006BFD1036103DD5E7F0B589B00C461022C6
:10B9680000210646684600F073FD2246694668468F
:10B9780000F0A4F99DF90030002B6A464FF0000151
:10B9880041DA137812F8010F01315B0043EAD01352
:10B998000F2902F8013CF4D19DF80F305B0083F0C9
:10B9A80087038DF80F30D4F81431102B3AD104F2F4
:10B9B8000113694604F211101A7811F8015B6A4004
:10B9C80003F8012B9842F7D104F1F10304F20110B6
:10B9D800194613F8012BDD7B834282EA050203F83E
:10B9E800012CF6D110220DEB020000F01DFD2246BD
:10B9F800314604A800F062F910220021684600F0E0
:10BA080027FD09B0F0BD137812F8010F01315B0072
:10BA180043EAD0130F2902F8013CF4D19DF80F3006
:10BA28005B00BEE79DF90020002A69464FF0000040
:10BA380035DA0A7811F8015F0130520042EAD5126E
:10BA48000F2801F8012CF4D19DF80F20520082F044
:10BA580087025F1C8DF80F20102F04EB0302C3F13F
:10BA68000F054FF0800188BF002503F5817382F828
:10BA78000111E0182A4600213D4403F023FAC4F8D6
:10BA8800145104F20113694604F211101A7811F8DE
:10BA9800015B6A4003F8012B9842F7D194E70A78D2
:10BAA80011F8015F0130520042EAD5120F2801F85F
:10BAB800012CF4D19DF80F205200CAE70A780378C8
:10BAC800534003704A784378534043708A788378A8
:10BAD80053408370CA78C3785340C3700A79037996
:10BAE800534003714A794379534043718A79837982
:10BAF80053408371CA79C3795340C3710A7A037A70
:10BB0800534003724A7A437A534043728A7A837A5B
:10BB180053408372CA7AC37A5340C3720A7B037B49
:10BB2800534003734A7B437B534043738A7B837B35
:10BB380053408373CA7BC37B5340C373704710B5AC
:10BB48000B7814786340037054784B7863404370E3
:10BB580094788B7863408370D478CB786340C370D3
:10BB680014790B796340037154794B7963404371BD
:10BB780094798B7963408371D479CB796340C371AD
:10BB8800147A0B7A63400372547A4B7A6340437297
:10BB98008B7A947A63408372D47ACB7A6340C37287
:10BBA800147B0B7B63400373547B4B7B6340437371
:10BBB800947B8B7B63408373CB7BD27B5340C37373
:10BBC80010BD0000A1F110032DE9F047DCB2102CE4
:10BBD80006D80123A34003F0013323F080732BB967
:10BBE800002382F8F030FF20BDE8F087531E441888
:10BBF800A04252D101F11C039B005FFA83F8C3F302
:10BC08000313013B2C4C82F8F0304FF001090B462E
:10BC180002EB030CB3FBF1F001FB103010F0FF0056
:10BC28001CF804AC1CF8037C1CF8026C1CF8015CC2
:10BC380038D14FEAD91014F807E0A75D665D14F80B
:10BC48000A5000EB400000EBC00089EA0E0E80EAC3
:10BC580049005FFA80F9F246581AC0B212F800E0BB
:10BC68008AEA0E0A02F803A0104403F1010E90F8C4
:10BC780001A05FFA8EFE87EA0A0702F80E7087783D
:10BC88007E408CF80260C0780433DBB245409845AA
:10BC98008CF80350BCD80020A6E710F8015B03F825
:10BCA800015FA5E71829D7D9102801BF14F80AA001
:10BCB800E75DA65D655DCFE7A4F900082DE9F04FC3
:10BCC80093B092F8F0300D910B92002B00F0448164
:10BCD80001460EA8FFF733FFA04CA14DA14E01234A
:10BCE8000193019A0B9BDDF804909DF838809DF82C
:10BCF8003CE09DF83DC09DF841709DF842009DF8DC
:10BD0800461003EB02130C939DF8393002939DF80B
:10BD18003A3003939DF83B3004939DF83E300593E9
:10BD28009DF83F3006939DF8403007939DF84330C7
:10BD380008939DF8443009939DF845300A930B9B6E
:10BD48009DF8472093F8F0304B4544D814F8083054
:10BD58008DF8383014F80E308DF83C30079BE35CD2
:10BD68008DF84030099BE35C8DF8443014F80C30B2
:10BD78008DF83930E35D8DF83D300A9BE35C8DF832
:10BD88004130029BE35C8DF84530235C8DF83A30F6
:10BD9800039BE35C8DF84230635C8DF83E30059B75
:10BDA800E35C8DF84630089BE35C8DF84730069BD2
:10BDB8000D98E35C8DF84330049BE35C8DF83F30CD
:10BDC8000EA9A35C0C9A8DF83B30FFF7B8FE002053
:10BDD80013B0BDE8F08F16F80CB015F8089014F8F9
:10BDE80000A0A35C89EA0B098AEA090983EA090920
:10BDF8008DF8389014F8089015F80CB083EA090308
:10BE08008BEA030316F800B0285C83EA0B038DF86D
:10BE1800393014F80C3016F807C089EA03098AEAA1
:10BE2800030316F808A08AEA030AAB5C89EA00094A
:10BE38008AEA0303B05C8DF83B3015F80E20049BAA
:10BE480089EA0009605CE35C8DF83A9082EA0C02AA
:10BE580042405A408DF83C2014F80E2015F807C0CF
:10BE680053408CEA030316F801C0695C83EA0C03AB
:10BE78008DF83D30E35D5A404A400499715C434077
:10BE880016F80E004A4058408DF83E20049B079A49
:10BE9800EB5CAA5C43408DF83F300A98039B305C0A
:10BEA800E15C069B4240E35C0A984A405A408DF8A0
:10BEB8004020079A285CA25C534043400398305CBA
:10BEC80043408DF841300A9B0398E35C285C5A4054
:10BED80042400698305C42408DF84220079A4B4019
:10BEE800B15C069A4B40A95C4B408DF84330059BEA
:10BEF800E35C089A0298A15C099A305CAA5C42400B
:10BF08005A404A408DF84420099A0298A25C285C5D
:10BF1800514041400598305C41408DF845100299E8
:10BF28000598615C285C4A4042400898305C424071
:10BF38008DF84620099AB25C4B405340089A0C99F8
:10BF4800AA5C0EA853408DF84730FFF7B7FD019B58
:10BF58000133DBB20193C4E6FF2039E7A4F90008F6
:10BF6800A4F70008A4F8000838B50C4650B1074DEE
:10BF780007492860C02200F057FA2CB12868A0476A
:10BF8800002038BD0220FCE72046FAE7280E0020F2
:10BF980000E503080A4B1A6870B5002302F1100582
:10BFA80003EB03142E5D864204D1103422440A6048
:10BFB800002070BD01330A2BF2D10320F9E700BF3E
:10BFC800280E00202DE9F041CCB00646DDF8488166
:10BFD80017461C460D4631B3B8F1000F23D006A80A
:10BFE800FFF73EFC204601A9FFF7D4FF0446B0B98D
:10BFF800019906A80131FFF743FC26B1102231460A
:10C0080006A8FFF742FC3A46294606A8FFF73DFC7A
:10C0180006A902A8FFF7A0FC029BC8F8003020463A
:10C028004CB0BDE8F0810224F9E7000010B592B0E9
:10C0380011A90446FFF7AEFF024600282ED1002CB6
:10C048002ED1214B22461146022002F0E9F9119B1C
:10C058001A7C0F92DA7B0E929A7B0D925A7B0C9285
:10C068001A7B0B92DA7A0A929A7A09925A7A089289
:10C078001A7A0792DA7906929A7905925A7904928D
:10C088001A790392DA7802929A7801925B7800938F
:10C0980000220E4B1146022002F0C2F912B010BD68
:10C0A800012C01D10A4BCEE7032C01D1094BCAE779
:10C0B800022C01D1084BC6E7042C01D1074BC2E77B
:10C0C8007F2CC4D1064BBEE7A4FA000822FB000867
:10C0D800B9FA0008CEFA0008E3FA0008F8FA0008EE
:10C0E8000DFB000810B5002288B01146264B274CDE
:10C0F800022002F095F90020FFF798FF0120FFF7D2
:10C1080095FF00221146224B022002F089F90320F4
:10C11800FFF78CFF0220FFF789FF002211461D4B15
:10C12800022002F07DF92368DA7907929A7906925B
:10C138005A7905921A790492DA7803929A780292D7
:10C148005A7801921B78009300221146124B022064
:10C1580002F066F92368DA7B07929A7B06925A7B8B
:10C1680005921A7B0492DA7A03929A7A02925A7AA0
:10C1780001921B7A00930022084B1146022002F01C
:10C188004FF9002008B010BD74FB0008280E0020ED
:10C1980089FB00089EFB0008B3FB0008F1FB0008C0
:10C1A80008B50420FFF742FF7F20FFF73FFF02207A
:10C1B800FFF73CFF0320FFF739FF002008BD7E2B67
:10C1C80010B402D810BCFFF7FDBE032010BC7047A6
:10C1D80030B50D4685B01446014668B103AA002063
:10C1E80000922A460390FFF7EDFE18B90398001B4A
:10C1F80018BF012005B030BD0220FBE72DE9F04350
:10C208000E46BFB014469946804628B323B311F0B2
:10C218000F0123D1F02201A800F01AF9204669463F
:10C22800FFF7B8FE044648B9009801AA102101306A
:10C23800FFF7C8FC3546771BFFB21DB920463FB053
:10C24800BDE8F08301AA09EB070108EB0700103DE0
:10C25800FFF734FDADB2EEE70224EFE70524EDE782
:10C268007FB5184E356802460023084605F11001CF
:10C2780003EB031401330C5D94421ED1802A03EBB7
:10C28800031413D10023CDE90033CDE902337F2213
:10C2980010216B46FFF7B2FF054630681022694649
:10C2A800204400F0C1F8284604B070BD01461022B1
:10C2B800281900F0B9F80025F5E70A2BD8D103258D
:10C2C800F1E700BF280E002009B1FFF7C9BF02201F
:10C2D80070471FB51446A0B17F2A01D1042912D195
:10C2E8000023CDE90033CDE902330A466B4610211D
:10C2F800FFF784FF18B969462046FFF7B1FF04B07D
:10C3080010BD0220FBE70320F9E72DE9F0411F46A5
:10C31800DDE907589DF8184093B38DB3B8F1000FC5
:10C328002ED0212C2ED8A6B219463246284600F027
:10C338007BF8711E01226B1C89B2B818FFF75EFFEB
:10C3480010BBEB7ADB0988F80030FBB92B19311FD9
:10C3580013F8010C13F8022C000640EA024013F807
:10C36800042C104313F8032C89B240EA022201235B
:10C378002846FFF72DFF003818BF0120BDE8F081DF
:10C388000220FBE70520F9E70720F7E70420F5E797
:10C3980008B5014630B1044B0822186800F044F88B
:10C3A800002008BD0220FCE7280E0020014B186879
:10C3B800704700BF280E002008B5014638B1054B6C
:10C3C80018680822104400F02FF8002008BD022049
:10C3D800FCE700BF280E0020014B186808307047A2
:10C3E800280E0020014B1860704700BF080100208C
:10C3F8000B4A30B514680B4D43F2390305FB04337F
:10C408001360091A6FF00042B3FBF2F2C2EBC2727A
:10C4180001319B1A93FBF1F201FB1233184430BD32
:10C42800080100206D4EC64101380A44914200D1EE
:10C43800704711F8013B00F8013FF7E710440A4440
:10C44800914200D1704711F8013B00F8013DF7E730
:10C4580002F038BD30B530B10A4D01444FF0FF331A
:10C46800814201D1D84330BD10F8012B5340082236
:10C4780043F30004013A2C4092B284EA5303002AA1
:10C48800F6D1EDE72083B8ED01207047054B4FF456
:10C4980000529A62044B1B6813B15B6803B11847DA
:10C4A800704700BF000400482C0F0020054B4FF4D4
:10C4B80080529A62044B1B6813B1DB6803B11847BA
:10C4C800704700BF000400482C0F002001F0B0BBEB
:10C4D80001F0DEBA08B501F02EFE012101F015FECB
:10C4E800BDE8084001F0A2B970B50C4E01EB40035D
:10C4F8000D46B3654FF6FF71002304461A460846F9
:10C5080001F018FA96F85600002101F0FEFD2946C0
:10C518002046BDE8704001F05FB900BF480F002019
:10C5280010B5044601F0BEFE01281CD101F0C2FE80
:10C5380034B11248214602F02DFB104802F0F0FAFF
:10C548000F4C104B00214FF48052A1659A6194F86A
:10C55800560001F0DAFD63786BB16FF07F40BDE8FB
:10C56800104001F0A5BA002340F262211A4608469D
:10C5780001F0E0F9DCE7A0688001F0E7300F002067
:10C58800480F002000040048002001F0E3B8000034
:10C5980008B501F0D9F80438C0B2032896BF024B99
:10C5A8000020185C08BD00BFBCFC000808B501F0FD
:10C5B800D7FD033008BD01F01DBD01F067BC08B50B
:10C5C80001F01DFA00B208BD38B50D46144601F059
:10C5D800E3F9284601F0AFFD084D012101F095FD72
:10C5E80001F024F94FF47A716143284602F0D2FA37
:10C5F8002846BDE8384002F093BA00BFA40F0020D7
:10C6080001F0CAB908B5084B002193F8560001F0AB
:10C618007CFD00234FF4C0711A46084601F08AF9E0
:10C62800BDE8084001F0F6B8480F002010B50446F0
:10C6380001F038FE01281CD101F03CFE34B112484B
:10C64800214602F0A7FA104802F06AFA0F4C104B84
:10C6580000214FF48052A1659A6194F8560001F0C8
:10C6680054FD63786BB16FF07F40BDE8104001F076
:10C678009DB8002340F262211A46084601F05AF993
:10C68800DCE7A0688001F0E7300F0020480F0020A9
:10C698000004004808B54FF0040001F025FBBDE890
:10C6A80008400220F5F776B808B500231A4619465F
:10C6B800184601F03FF9BDE8084001F0ABBC0000A6
:10C6C8001D4B73B51D4D186000241D486C70C5E9DD
:10C6D8000144AC6501F0D0FAAC8101F0BDF8214607
:10C6E800204601F07FF921460422012001F032FBA7
:10C6F800144E154D4FF6FF7123462246084601F0A9
:10C7080019F9FFF7C7FF2246104B00944FF0FF318D
:10C71800304602F057F90E4B009422464FF0FF3195
:10C72800284602F04FF9304602F0AAF9284602B02E
:10C73800BDE8704002F0A4B92C0F0020480F00207B
:10C7480001D70008A40F0020300F002095C400086E
:10C75800B5C400080128084805D1084BC1771970ED
:10C768000E3001F0D5BB437D012B03D1034B8175FE
:10C778001970F5E7704700BF480F00200C01002032
:10C788000D4B10B5044618735873012000F016F8C5
:10C798005CB134214FF4E86001F07AF94421BDE836
:10C7A800104040F2417001F073B914214FF4E86071
:10C7B80001F06EF92421F2E7480F002038B5114C3A
:10C7C8000546207001F07BFD052D04D8DFE805F053
:10C7D800090B03171709032001F09EF9002363735F
:10C7E80038BD0020F8E7012001F096F9207B637B33
:10C7F8008342F5D06073BDE83840FFF7C1BF02201F
:10C80800EAE700BF480F00202DE9F0431E4687B035
:10C8180000230546CDE901330C46174601F041FDDA
:10C82800032D61D8DFE815F07B00C3000E0104007A
:10C83800A27C082A04D94FF0FF3007B0BDE8F08386
:10C84800A16801A801F0F6FE21680029F3D042F2A0
:10C8580010729142E37C864D51D80322AA7385F861
:10C868003820E96385F844304FF002086368A17DF9
:10C87800DB002B820423AB74A37CDB00EB7402295E
:10C888004FF000032B75637D02D0227D022A42D12E
:10C8980003F10F02D2B2012A01D9012BCBD1754B7A
:10C8A800754A196803944FF0010903A88DF814908C
:10C8B80001F0F4FC0028BED1287685F81790687539
:10C8C800FFF762FE4046FFF779FF6C4801F03AF93E
:10C8D8006B4801F01DFB01A801F0E8FA208A01F07D
:10C8E8001DFAA08901F000FB384601F024FC604CD9
:10C8F80084F8560001F0DAFC666000209DE74FF0EE
:10C908000008E963890885F80E8085F8388085F87D
:10C9180044302964AAE7EB7529766A75D0E723685D
:10C92800002B88D0A27C082A85D8514DA16801A87F
:10C9380001F080FE002385F838302268EA63E27C43
:10C9480085F84420A269AB732A646268A17DD2008D
:10C958002A820422AA74A27C2B75D2000229637D44
:10C96800EA7402D0227D022A1DD103F10F02D2B24D
:10C97800012A02D9012B7FF45EAF3E4B3E4A19686B
:10C9880003944FF0010803A88DF8148001F086FC89
:10C9980000287FF450AF287685F817806875FFF770
:10C9A800F3FD00208FE7EB7529766A75F7E7304DC0
:10C9B800012185F83810227885F85020637885F8A9
:10C9C8005130A37885F85230E3788B4202D0022B9D
:10C9D80003D03BB985F8533004E00B3A012A29D833
:10C9E80085F853104FF0010885F80E80A388AB83B3
:10C9F800A379AB77E37985F82030237A85F821305D
:10CA0800FFF7C2FD4046FFF7D9FE1C4801F09AF82F
:10CA18001B4801F07DFA95F85130062B40F6890045
:10CA28000AD101F005F900F0FB0140F6890001F098
:10CA38002FF859E70023CDE701F0FAF840F0040198
:10CA4800C9B2F2E72368013BB3F57A7FBFF4F3AECE
:10CA58000320FFF7B3FE0648022380F83830236826
:10CA68008364162380F84C30383001F06BF83BE7CC
:10CA7800480F00202C0F0020A40F0020800F00205A
:10CA8800560F00202DE9F041002686B01F461446B7
:10CA9800CDE9016680460D4601F003FCB442774CAF
:10CAA80016BF0123334637466370B8F1000F06D02E
:10CAB800B8F1010F7CD0002006B0BDE8F081AB686A
:10CAC800002B00F0D780EB68002B00F0D380AA7F02
:10CAD800082A00F2CF80296901A801F0ABFD286877
:10CAE800003818BF012000F0ABFE84F83880AB682E
:10CAF800E36395F8203084F84430686801F074FBEB
:10CB080084F80E8084F84500EB68DB002382EB7F15
:10CB1800A374AB7FDB00E37495F82130237595F897
:10CB28002230002B3ED16A6995F82410A27502299B
:10CB380095F8232001D0022B36D102F10F03DBB286
:10CB4800012B02D9012A40F0958000238DF814307A
:10CB58004B4B4C4A1968049503A801F09FFB002829
:10CB680040F0888001232076E3756075FFF70CFD9F
:10CB78000020FFF723FE444800F0E4FF434801F09B
:10CB8800C7F901A801F092F9A88B01F0C7F8288B22
:10CB980001F0AAF94FF4FA535F43AB68B7FBF3F718
:10CBA800A76088E7FF22BFE7E27521766375DDE7B6
:10CBB8002B8E002B5ED095F83230A86A012B0CBF63
:10CBC80095F814804FF0FF08003818BF012000F0D6
:10CBD80037FEF8B200F088FF012184F8381095F884
:10CBE8002C2084F8502095F82D3084F8513095F891
:10CBF8002E3084F8523095F82F308B4202D0022B19
:10CC080003D03BB984F8533004E00B3A012A29D801
:10CC180084F853102B8EA38395F83230A377AB8E0C
:10CC280023840126A67384F81F80FFF7ADFC3046E5
:10CC3800FFF7C4FD144800F085FF144801F068F9B7
:10CC480094F82130B34240F236700DD100F0F0FF75
:10CC580000F0FB0140F2367000F01AFF4FF6FF7348
:10CC6800A36028E70023CDE700F0E2FF40F00401CD
:10CC7800C9B2EFE74FF0FF301EE700BF480F0020B2
:10CC88002C0F0020300F0020800F0020560F0020AE
:10CC98002DE9F04F85B082460E9DBDF840B09DF855
:10CCA80044709DF84890019288461E4601F0F9FAB2
:10CCB800BAF1010F4F4C4DD0BAF1040F00F08B8040
:10CCC800BAF1000F3AD10B22304684F8442084F898
:10CCD80038A0E56301F088FA019B23644FEACB038F
:10CCE800B9F1000F238241F60403638214BFF223D3
:10CCF8000123E37587F001070123237684F84500B3
:10CD080084F80EA084F814A06775FFF73DFC504620
:10CD1800FFF754FD04F1380000F014FF04F10E0091
:10CD280001F0F6F8344A1068516802AB03C302A850
:10CD380001F0BCF840F2FF1000F0F0FF404601F0AF
:10CD4800FAF984F8560001F0B1FA169B636005B051
:10CD5800BDE8F08F294984F838A0895D84F851101E
:10CD6800EAB29DF83C1084F8502084F8521036BB83
:10CD78000B3D012D8CBF002501250121053A8A4272
:10CD880084F85350A17323D8BBF10B0F20D80C2380
:10CD9800A3831B4BA7771B78E3779DF8543084F85F
:10CDA800213084F82090FFF7EFFB0120FFF706FD04
:10CDB800144800F0C7FE144801F0AAF8BEE7012E97
:10CDC80004D1A5F10C035D425D41D6E70025D4E707
:10CDD800A4F81CB0DDE75046FFF7F0FC022384F806
:10CDE800383004F138001623A56484F84C3000F07C
:10CDF800A9FEA3E7480F002048F000088DFC0008B2
:10CE08000C010020800F0020560F00202DE9F04F64
:10CE180087B0DFF8A8B29DF864A09DF84C90029303
:10CE280014469DF854309DF85020BDF84880039270
:10CE380005468BF801A0BDF8446001930F4601F048
:10CE480030FABAF1000F18BF4FF00008DFF870A2EF
:10CE5800039AB9F1000F08BFFF22012D8AF80020BC
:10CE680000F0C880052D48D0002D40F0C08028462D
:10CE780000F0E6FC0B2238468BF844208BF838503B
:10CE8800CBF83C4001F0B0F9019B8BF8450041F626
:10CE98000402002BABF812209AF800208BF8162019
:10CEA80014BFF22201228BF81720F600012289F024
:10CEB80001098BF818208BF80E50ABF810608BF82E
:10CEC80014508BF81590FFF75FFB2846FFF776FCA8
:10CED8000BF1380000F036FE0BF10E0001F018F8E7
:10CEE80078490868496804AA03C204A800F0DEFF6C
:10CEF80040F2FF1000F012FF71E0012000F0A0FCEA
:10CF080009224FF000098BF8442038464FF4487244
:10CF1800CBF840208BF83890CBF83C4001F064F90E
:10CF28004FF48052ABF812209AF800208BF8450095
:10CF38008BF8162028460122F6008BF817208BF86C
:10CF48000E90ABF81060ABF814908BF81890FFF7C0
:10CF580035FC0BF1380000F0F5FD0BF10E0000F088
:10CF6800D7FF58498868C96804AA03C204A800F012
:10CF78009DFF40F2FF1000F0D1FE40F6B80000F02F
:10CF880057FE00F0EF0140F6B80000F081FD0421E3
:10CF980040F6B90000F07CFD40F69B0000F048FE2A
:10CFA80000F0E30141F0080140F69B0000F070FD3D
:10CFB80040F2D16000F03CFE40F01801C9B240F2E6
:10CFC800D16000F065FD40F2AC6000F031FE00F089
:10CFD8008F0141F0500140F2AC6000F059FD4FF470
:10CFE800FA5202FB08F8B8FBF4F4CBF8084007B093
:10CFF800BDE8F08F002000F023FC3349029BC95D97
:10D008008BF83850E2B28BF850208BF851108BF81F
:10D018005230002F40D10B3C012C8CBF002401243E
:10D028000121053A8A428BF853408BF80E103CD800
:10D038000B2E3AD80C22ABF81C209AF80020019B42
:10D048008BF81F209DF860208BF821208BF820306A
:10D058008BF81E90FFF798FA0120FFF7AFFB1B48EB
:10D0680000F070FD1A4800F053FF5FFA88F000F0F6
:10D078003BFD9BF82120012A40F2367018D100F0C0
:10D08800D7FD00F0FB0140F2367000F001FD4FF6CD
:10D09800FF72CBF80820AAE7012F04D1A4F10C03F2
:10D0A8005C425C41BCE70024BAE7ABF81C60C4E70B
:10D0B80000F0BEFD40F00401C9B2E4E7480F0020CB
:10D0C8000C01002048F000088DFC0008800F0020AB
:10D0D800560F0020F0B58BB00D46044617461E4685
:10D0E800FFF752FA0020FFF769FB204600F054FCD6
:10D0F80000240123CDE9084303234FF4167229467F
:10D108002046CDE90644CDE90444CDE90244CDE901
:10D1180000532346FFF77AFE2046FFF787FAFFF70A
:10D1280045FAF4F737FB01F067FC0446204601F0A6
:10D138006DFCB04205D30124FFF726FA20460BB058
:10D14800F0BD00F05CFC00B28742EFDA0024F3E7A0
:10D15800F7B500230C4640F201211A460646084658
:10D1680000F0E8FB654B664D4FF400529A6195F864
:10D178005600012100F0C9FF2B78012B40F68900E9
:10D1880013D195F85130062B0FD100F051FD00F066
:10D19800FB0140F6890000F07BFC2B78042B6ED84D
:10D1A800DFE803F0544D5481090000F041FD40F0E0
:10D1B8000401C9B2EDE7534A731E1046C6F10107D0
:10D1C8004FF0000CF9188C4271DC0023E700194677
:10D1D800BB4273D100294FEA81130CBF20220022E1
:10D1E80043EAC1131343661C0355F6B202234648AB
:10D1F800AB73AE7600F08CFE0021F12000F048FC05
:10D208000021F02000F044FCAB6C642B6FD170213E
:10D21800F32000F03DFC1D21F22000F039FCE10074
:10D228008C1CF420090A00F033FC04F0FE01F52000
:10D2380000F02EFC33486FF07F4231461DE0EC775A
:10D24800314800F065FE0022214615E001F02AF879
:10D258000128074625D121460DF10702304601F085
:10D2680026F80446A8B99DF807302748AB7500F0A2
:10D278004FFE9DF807102246304600F014FF6968FB
:10D28800224801F087FC214803B0BDE8F04001F0D6
:10D2980047BC1F4B3A460021022001F0C1F803B0F9
:10D2A800F0BDAC75CCE70223AB73AC76C8E713F8D6
:10D2B800011FC943197002F801CB83E7DA4302F072
:10D2C800070CDA100133B25C42FA0CF202F00102E8
:10D2D8004FEAE30C5140DA4310F80CE002F0070281
:10D2E80001FA02F242EA0E0200F80C2070E7E1218E
:10D2F800F32000F0CDFB04218EE700BF00040048B6
:10D30800480F00202C0E0020560F0020A40F0020EC
:10D318002FFC0008F0B5BDF814409DF818C09DF822
:10D328001C709DF8205040B1012819D0012200241A
:10D33800A0180138B0FBF2F0F0BDBCF1000F0CBF33
:10D3480008230023002D03EBC40414BF022000208F
:10D358001834384404EBC0004FF47A744443E7E7C8
:10D36800501F012803F1040302D80C2C38BF0C24E9
:10D37800002937D1A2F10B06012E8CBF0026012609
:10D38800002D14BF1020002000EBC700BCF1000FD7
:10D3980014BF00271427A0EB8200062A38444FEA5E
:10D3A8008205A2F1020702D9083006B1BD000028A3
:10D3B800ACBF2E182E1C701E90FBF5F503FB054420
:10D3C8000D4B5B5C062A8CBF0C340E340A2B12D82A
:10D3D800A4000A4A0134BC404FF47A7052F8232062
:10D3E8004443A5E7012904D10C2A14BF00260126CD
:10D3F800C6E70026C4E7FFDE8DFC000890FC0008A5
:10D4080008B5094B012193F8560000F07EFE4FF451
:10D41800D7602D2100F03CFB00F00DFABDE8084074
:10D42800024800F0ADB900BF480F0020FFFF0F0011
:10D4380073B5A44CB4F854300025202B8DF8035054
:10D44800019500F01B8114D8082B0DD87BB1013B46
:10D45800072B0CD8DFE813F042005B000B00CD006F
:10D468000B000B000B00FD00102B00F0008102B038
:10D4780070BDB3F5807F00F0988011D8402B00F084
:10D488001081802BF3D1284600F064F98E4B1B687D
:10D49800002BECD09B69002BE9D028469847E6E79B
:10D4A800B3F5007FE3D1894B01222946022000F021
:10D4B800B7FF00F049F9042840F08580844B85487F
:10D4C8004FF400529A6201F0DBFA284600F042F964
:10D4D8007D4B1B68002BCAD05B6814E07C4B7D48F1
:10D4E8004FF400529A6201F0CBFA002000F032F9B2
:10D4F80000F0DAFE012801D100F0DFFE724B1B6854
:10D50800002BB4D01B68002BB1D09847AFE7704B05
:10D5180071484FF480529A6201F0B2FA657895B971
:10D52800284600F017F9294640F6021000F0B0FA34
:10D5380040F6441000F07CFB40F00201C9B240F60E
:10D54800441000F0A5FAFF220DF1030163485E4D77
:10D5580000F0C2FD624800F05FFA2B68002B86D00D
:10D568009E68002E83D094F82430012B08D194F9BA
:10D57800313094F930209DF803105848B04776E7C9
:10D58800E06B01A900F044FE019B9DF8031053488D
:10D598004FF47A7203F5FA7393FBF2F32A685BB2DD
:10D5A800956894F92920A84761E7284600F0D2F841
:10D5B800454B1B68002B3FF45AAF9B69002B3FF487
:10D5C80056AF01206AE700F0BFF805287FF44FAF97
:10D5D8003F4B41484FF480529A6201F051FA284675
:10D5E80000F0B8F8384B1B68002B3FF440AFDB68FD
:10D5F80089E700213B4B0122022000F011FFA16DB9
:10D6080000293FF434AFC1F3074140F6031000F09E
:10D618003FFA94F8591040F6041000F039FA94F8DB
:10D62800581040F6051000F033FA40F6021000F0EA
:10D63800FFFA40F00101C9B240F6021000F028FAE2
:10D64800002340F262211A460846A36500F072F9E9
:10D658000DE7254B01220021022000F0E1FE00F039
:10D6680021FE01287FF403AF00F028FEFFE61F4BE0
:10D6780001220021022000F0D3FEF8E6164801F04E
:10D68800FFF9607808B900F065F80F4B1B68002BAC
:10D698003FF4EDAEDB68002B3FF4E9AE9847144B3E
:10D6A800E6E7144B01222946022000F0B9FE607813
:10D6B80008B900F04FF8044B1B68002B3FF4D7AEB5
:10D6C8001B6920E7480F00202C0F002044FC0008AD
:10D6D80000040048A40F0020300F00202C0E00206A
:10D6E8006C0F002058FC000861FC00086BFC000867
:10D6F80074FC00087DFC0008024BA3F85400FFF7F7
:10D7080097BE00BF480F002010B51346EFF31084F2
:10D7180072B60A4601460348F7F7F2FA84F310880E
:10D7280010BD00BFD001002010B51346EFF31084E0
:10D7380072B60A4601460348F7F71AFB84F31088C5
:10D7480010BD00BFD0010020014B1878704700BF02
:10D75800C20F002007B501228DF807000DF107015F
:10D768008020FFF7D1FF9DF80730002B034B0CBF3B
:10D77800012202221A7003B05DF804FBC20F0020D8
:10D7880007B5094B8DF8060004221A70030C8DF8B2
:10D7980004300322030A01A983208DF80530FFF71E
:10D7A800B3FF03B05DF804FBC20F002007B5094BB7
:10D7B8008DF8060005221A70030C8DF80430032238
:10D7C800030A01A982208DF80530FFF79DFF03B0F9
:10D7D8005DF804FBC20F002007B5030C8DF800307C
:10D7E800030A8DF801300B0C8DF802008DF8033018
:10D7F8008DF805100B0A0622694694208DF804302E
:10D80800FFF782FF024B06221A7003B05DF804FB93
:10D81800C20F0020002208B51146C520FFF774FF8B
:10D82800014B07221A7008BDC20F002000221146C2
:10D83800D120FFF769BF00221146D220FFF764BF4D
:10D8480007B501228DF807000DF107019F20FFF7AA
:10D858005BFF03B05DF804FB07B5F4F7EFFE431E6A
:10D86800584258418DF8070001220DF10701962012
:10D87800FFF74AFF03B05DF804FB07B500F07F002F
:10D888008DF8070001220DF107018920FFF73CFF01
:10D8980003B05DF804FB0000184B984207B50DD99A
:10D8A800E1238DF80430E9238DF80530022201A91F
:10D8B8009820FFF729FF03B05DF804FB104B98424E
:10D8C80004D9D7238DF80430DB23EDE70D4B9842BC
:10D8D80004D9C1238DF80430C523E5E70A4B9842E3
:10D8E80004D975238DF804308123DDE7074B98426E
:10D8F800DCD96B238DF804306F23D5E700E9A43514
:10D9080080F8A9328044E52D000B6B1B40FC5419AC
:10D9180007B58DF8062004228DF804008DF805104F
:10D9280095200DEB02018DF80730FFF7EDFE03B0EF
:10D938005DF804FB13B5040A8DF801008DF8031097
:10D94800080A8DF80520110A1A0A8DF806200822FF
:10D958008DF802008DF80410104669468DF80040D5
:10D968008DF80730FFF7D0FE02B010BD07B50B0CDD
:10D97800042200F007008DF804008DF805308DF8BA
:10D9880007100B0A97200DEB02018DF80630FFF700
:10D99800BBFE03B05DF804FB37B5104D2B78044689
:10D9A8001BB9FFF779FF01232B700D4A002360068E
:10D9B800E109F3F7F5F8030E8DF804300422030C9F
:10D9C8008DF805308DF80700030A0DEB020186205B
:10D9D8008DF80630FFF798FE03B030BDC00F002069
:10D9E8000048E80107B502228DF804008DF80510FB
:10D9F8008F2001A9FFF788FE03B05DF804FB07B587
:10DA0800012201A91520FFF78FFE9DF8040040426E
:10DA1800401003B05DF804FB13B50322044601A9C6
:10DA28001420FFF781FE184B1A7822704AB1012A98
:10DA380017D014220021204600F006FE0F23237081
:10DA48000DE09DF8043023719DF80530A2605B421B
:10DA58005B10A3719DF806305B425B10637102B0E6
:10DA680010BD9DF804305B425B1023739DF90530AF
:10DA780002339B1063739DF806305B425B10A373FF
:10DA8800024B1B682361EAE7C30F0020BC0F00208C
:10DA980007B501238DF807100DF107020146034869
:10DAA800F7F7BAF803B05DF804FB00BFD001002017
:10DAB80013B50C4B04460522972140F6AC001A70AA
:10DAC800FFF7E6FF230C8DF804300322230A01A98F
:10DAD80082208DF805308DF80640FFF715FE02B05C
:10DAE80010BD00BFC20F002007B501228DF8070046
:10DAF8000DF10701A020FFF707FE9DF807103F2949
:10DB080007D901F0F8010131C9B240F20670FFF7F8
:10DB1800BFFF03B05DF804FB07B5094B8DF807009C
:10DB28000146187018B940F2AC60FFF7B1FF012246
:10DB38000DF107018A20FFF7E7FD03B05DF804FB4C
:10DB4800C30F002013B5364A0446516810686B4667
:10DB580003C3344B20781B78834201D0FFF7DCFFE6
:10DB68002378032B29D8DFE803F0023B2A466268B2
:10DB78002D4BB3FBF2F31A0CA1688DF800208DF839
:10DB880002301A0A237B8DF80330637B8DF801205D
:10DB98008DF80430254A00234806C909F3F700F830
:10DBA800030C8DF80530030A8DF806308DF8070050
:10DBB800082269468B20FFF7A7FD02B010BD226935
:10DBC800194BB3FBF2F31A0C8DF800208DF80230D4
:10DBD8001A0A237D8DF801208DF803300422E8E726
:10DBE800237E8DF80030637E8DF80130A37E8DF89A
:10DBF8000230E37EF0E762680B4BB3FBF2F31A0CDA
:10DC08008DF800208DF802301A0A237B8DF8033036
:10DC1800637B8DF801208DF804300522C9E700BF29
:10DC280058F00008C30F00200000093D0048E80133
:10DC380007B5012301460DF107020448F7F725F857
:10DC48009DF8070003B05DF804FB00BFD001002079
:10DC580010B50446F4F7F2FC01280CD140F6231065
:10DC6800FFF7E6FF00F0F901214340F62310BDE875
:10DC78001040FFF70DBF10BD10B508B1174B186065
:10DC8800F3F790FC0220FFF7E3FF0024144B204633
:10DC98001C70FFF75FFDF4F7CFFC012812D14FF499
:10DCA8002071FFF763FE40F611102146FFF7F0FEE2
:10DCB8004FF07F00FFF7E1FDF4F762FC094B01220A
:10DCC8001A7010BD102140F61110FFF7E1FE102167
:10DCD80040F61210FFF7DCFEEEE700BFC40F00208D
:10DCE800C00F0020C20F002013B504460020F4F72F
:10DCF8007FFC0220FFF7ACFF04F0070401220DF1BE
:10DD0800070184208DF80740FFF7FEFC024B002234
:10DD18001A7002B010BD00BFC20F002010B50C4B26
:10DD28001B7804469BB94FF4D760FFF781FFC4F313
:10DD3800002100F0FE0001434FF4D760FFF7A8FE72
:10DD4800E1B240F2B960BDE81040FFF7A1BE10BDD6
:10DD5800C30F0020012873B50C46164637D10020A2
:10DD6800F4F76EFCA042B8BF44B20E2805461AD19B
:10DD780001231A4600210420FFF7CAFD6FF01001A5
:10DD88008C42B8BF0C46182140F6E700FFF780FE2A
:10DD9800022201A98E208DF804408DF80560FFF756
:10DDA800B3FC02B070BD01230A28E4B21A464FF052
:10DDB800000105D11846FFF7ABFD033464B2DDE777
:10DDC8000620C5F10E05FFF7A3FD2C44F6E740F643
:10DDD800D800FFF72DFF40F01E01C9B240F6D80069
:10DDE800FFF756FE0120F4F72BFCA042B8BF44B25F
:10DDF800142805464FF001034FF0000206D1052113
:10DE08000320FFF785FD023464B20DE0112805D127
:10DE180003210220FFF77CFD0534F5E70E280AD11F
:10DE280002210846FFF774FD6FF008018C42B8BF65
:10DE38000C463821A8E707210420C5F11605FFF78D
:10DE480067FD2C44E0E7000037B504460D46022282
:10DE580001A91320FFF768FC0A4B1B78012B0DD191
:10DE6800094B1B78012B09D140F20270FFF7E0FE45
:10DE780020709DF805302B7003B030BD9DF804303C
:10DE88002370F6E7C30F0020C10F002010B513461A
:10DE9800EFF3108472B60A4601460348F6F7BCFE53
:10DEA80084F3108810BD00BFD001002008B50146DA
:10DEB80008224FF4D860FFF7E9FF002008BD0000F2
:10DEC80007B5030A8DF80430064B8DF805001B785A
:10DED8002BB9022201A940F2BC60FFF7D7FF03B0BB
:10DEE8005DF804FBC30F002007B5030A8DF8043062
:10DEF800064B8DF805001B782BB9022201A940F2C8
:10DF0800BE60FFF7C3FF03B05DF804FBC30F00203A
:10DF18001FB5354A0446D1689068127C01AB03C32B
:10DF28001A70324B20781B78834201D0FFF7F4FD3A
:10DF38002378032B2ED8DFE803F002403B02637AF4
:10DF4800F12B29D14FF6FF70FFF7BAFF48F2050011
:10DF5800FFF7CAFF022362888DF80520110A22798B
:10DF68008DF8062062798DF80720A2798DF80820AF
:10DF7800E2798DF809208DF80B30227AA37A8DF892
:10DF88000A208DF804108DF80C30092201A98C2084
:10DF9800FFF7BAFB04B010BDF22BDCD141F60F50ED
:10DFA800FFF78EFF41F22100FFF79EFF0623D2E71D
:10DFB800237B8DF804300122E8E7E3898DF80530EA
:10DFC8001A0A8DF804200A4A237C13708DF806304B
:10DFD800637C8DF80730A37C8DF80830E37C8DF8DE
:10DFE80009300622D2E700BF58F00008C30F00200E
:10DFF800C10F002010B51346EFF3108472B60A461D
:10E0080001460348F6F741FE84F3108810BD00BFAF
:10E01800D001002073B5002640F6E2000196FFF714
:10E0280007FE00F0FE01054640F6E200FFF730FD6E
:10E0380040F6E500FFF7FCFD00F07F01044640F6DE
:10E04800E500FFF725FD6FF07F40FFF7AFFB0422E7
:10E058000DEB020140F61900FFF7CCFF3046FFF741
:10E0680079FB294640F6E200FFF712FD214640F60B
:10E07800E500FFF70DFD019802B070BD10B513461D
:10E08800EFF3108472B60A4601460348F6F7EBFE32
:10E0980084F3108810BD00BFD00100200A46014655
:10E0A8000020FFF7EBBF10B51446FFF7F7FF204637
:10E0B800BDE81040FFF764BB10B51346EFF31084BA
:10E0C80072B60A4601460348F6F700FF84F3108843
:10E0D80010BD00BFD0010020F7B50D46064600244C
:10E0E8000DF10701284617468DF80740FFF7ACFEEB
:10E0F8002A78BA4207D89DF807003146FFF7DCFFB7
:10E10800204603B0F0BD0120FBE7012908B503460E
:10E1180008460ED1012B07D10420FFF799FD0220F4
:10E12800BDE80840F4F764BA022B14BF0846032080
:10E13800F6E70120F4E738B50446F4F77BFA50B166
:10E14800022814BF01250225284602222146FFF78E
:10E1580001FE284638BD0F2CCCBF02250125F3E768
:10E168000A207047014B01201B681847C40F002084
:10E17800014B02201B681847C40F0020014B4020A8
:10E188001B681847C40F002011B1012904D070473B
:10E19800044B1B6880201847024B4FF480701B68A3
:10E1A800F9E700BFC40F0020024B4FF400701B6852
:10E1B800184700BFC40F0020014B20201B681847D8
:10E1C800C40F0020014B04201B681847C40F00200F
:10E1D800014B08201B681847C40F0020014B102072
:10E1E8001B681847C40F002068B1084A002352F87A
:10E1F8003310814203D902EBC30318797047013306
:10E20800162BF4D1FEE71F20704700BF44FD00081D
:10E2180073B51D4B0193064640F607000D46FFF700
:10E2280007FDC0F3C10308336B4413F8044C00F036
:10E238000703013B04FA03F3144CB4FBF3F4B4FBF7
:10E24800F6F007281DD8400003288CBF02230423BA
:10E258004FF4D6605C43FFF7EBFC000200F47066F5
:10E2680040F2B160FFF7E4FC3043030544BF6FEAB6
:10E2780000506FEA105063094343DB112B6002B072
:10E2880070BD0123E4E700BF04080A0C0048E80158
:10E298004FF0FF3070474FF0FF3070474FF0FF30BE
:10E2A80070477047002070470020704770474FF054
:10E2B800FF3070474FF0FF30704770477047704726
:10E2C80070B5EFF3108672B6144B5C8A1A8A9442C2
:10E2D80013D1C4F5806292B2904206D3844218D911
:10E2E80001229A7000221C805A825A8A0A8010449D
:10E2F800C0F30900588200200DE006D9C4F58065F6
:10E30800ADB28542F1D88242E9E7121B92B282424D
:10E31800EBD84FF0FF3086F3108870BDC81300208B
:10E32800EFF3108172B6034AD38A0133D38281F3A3
:10E3380010887047C8130020EFF3108172B6034AA3
:10E34800D38A013BD38281F310887047C813002019
:10E3580010B508481822002100F076F906484FF455
:10E368008062002100F070F9044B05481B68BDE885
:10E3780010401847C8130020C80F0020D0F000082C
:10E38800F5E40008014B5860704700BFC81300202F
:10E39800014B1872704700BFC813002073B5EFF324
:10E3A800108572B61B4CE08A00282ED1FFF7B8FF03
:10E3B800268A628A964226D0A178012911D123881B
:10E3C80020809B1B9BB20221A382A1705BB9A37022
:10E3D8002382238A9A428CBFD31AC3F58063A3820F
:10E3E80001E00029F5D0208A0B4E064485F31088F9
:10E3F800F3F7BEF9094BA18ADB680193304602B0F6
:10E40800BDE870401847FFF797FF85F31088002094
:10E4180002B070BDC8130020C80F0020D0F000085B
:10E4280008B4F0B586B00023ADF800302C4B0B9C37
:10E438001D7A85424DD3D86881434DD15B681BB1A5
:10E4480012B1694602A898470CAB22464FF40071F6
:10E458002448019300F0FAFBFFF762FFBDF8003093
:10E4680018440DF1020180B2FFF72AFF01302BD0CA
:10E478000022BDF80030BDF802701B480DF1080CF1
:10E48800164691B217FA82F58B42ADB216D83B44C4
:10E498009BB20EB1ADF80230BDF80250019B224686
:10E4A8004FF40071284400F0D1FBFFF745FFFFF758
:10E4B80075FF06B0BDE8F04001B070471CF8011BBD
:10E4C800415501320126DCE7FFF736FF6FF0020005
:10E4D800EFE76FF00400ECE76FF00500E9E700BF35
:10E4E800C8130020E0130020C80F002037B5EFF351
:10E4F800108472B6214B9A78022A1DBF1A8A998A0B
:10E508005218002218BFC2F309021A821D8A598ABA
:10E5180008BF9A708D4227D0DA8A012A24D19878C8
:10E52800012812D11A880220521B92B2987000203A
:10E538009A8218805AB99A701A821A8A91428CBFA4
:10E548008A1AC2F580629A8201E00028F5D01A8AF8
:10E558000B48104484F310880A4A998AD3680193B7
:10E5680003B0BDE83040184784F31088F3F704F986
:10E5780003B0BDE83040FFF7DFBE00BFC81300207E
:10E58800C80F0020D0F00008024A00231360024A96
:10E5980013607047E4150020E015002010B5EFF374
:10E5A800108472B641B1012903D1064A1368184391
:10E5B800106084F3108810BD024A136823EA000033
:10E5C800F6E700BFE415002010B5EFF3108472B62B
:10E5D80041B1012903D1064A13681843106084F336
:10E5E800108810BD024A136823EA0000F6E700BF4E
:10E5F800E015002038B5EFF3108572B60A4B0B4CC6
:10E608001B6833B1236898476368984785F3108877
:10E6180038BD074B1B681BB1A3689847E368F4E74C
:10E62800236998476369F0E7E41500206CF0000857
:10E63800E015002001380A44914200D1704711F8D2
:10E64800013B00F8013FF7E700F03CBC10B5EFF3E1
:10E65800108472B6064A136803431360054A52F8D9
:10E668003130184342F8310084F3108810BD00BFE0
:10E678000C1600200416002070477047030C1B047A
:10E68800C3B90004102310F07F4F02BF0833000203
:10E69800DBB210F0704F08BF0001074A4FEA107054
:10E6A80008BF0433105C08BFDBB2C3F11F03181A9C
:10E6B800C0B270470023E6E7F4FD00082DE9F84FE3
:10E6C800384D394ED5F80080DFF8E0B0DFF8E0A02B
:10E6D800DFF8E0903368384FDBF80010374C08EA71
:10E6E80000002860DAF80000D9F80020D5F800C04A
:10E6F8000CEA000E1EEA030F01D011421ED04FF0A3
:10E70800FF333B60FFF7B8FFEFF3108472B633684E
:10E71800DBF80020DAF800100B4029680B4205D11D
:10E72800D9F80030134201D1F2F7B6FF84F310880C
:10E73800FFF7A3FFC5F80080BDE8F88F23682368BA
:10E74800626803EA0C0303401A4204BF4FF0FF3229
:10E75800626060681840FFF791FF636838600122C3
:10E7680002FA00F023EA00006060EFF3108172B64D
:10E778003B6802FA03F3326822EA03023260226835
:10E7880022EA0303236081F310880D4A3B6852F89C
:10E79800233098473368DBF80010DAF80000D9F81E
:10E7A8000020A3E7100100200C160020EC15002023
:10E7B80014010020F0150020E815002004160020A0
:10E7C800F415002010B51146EFF3108472B6FFF768
:10E7D80055FF034B43F8201084F3108810BD00BF89
:10E7E800F415002082B082B00DF1080C0CE9060087
:10E7F800BDF8042003930B44BDF810100A4491B2ED
:10E8080012B2B2F57A7FA2BFA1F57A72013312B2C1
:10E818000360828002B002B0704782B082B00DF10E
:10E82800080C0CE90600BDF804200393CB1ABDF8C8
:10E838001010521A91B212B2002ABEBF01F57A72B4
:10E8480003F1FF3312B20360828002B002B0704756
:10E8580030B585B0114D6B4683E803000023029361
:10E86800ADF80C3003A82B699847009BBDF804400D
:10E878000290181ABDF80C30E41AA3B224B2002C86
:10E88800BEBF03F57A7400F1FF3024B22B689847B5
:10E89800AB682046984705B030BD00BF90F000082F
:10E8A80073B5114E002305460093ADF8043001A856
:10E8B80033699847F3680090984773680446984707
:10E8C800009B1844BDF8043023449AB21BB2B3F538
:10E8D8007A7FA2BF0130A2F57A731BB2286028465E
:10E8E800AB8002B070BD00BF90F0000837B50023C0
:10E8F8000093ADF80430074B04461B6901A89847FC
:10E908006D46009095E8030084E80300204603B0B4
:10E9180030BD00BF90F0000837B50F4D02AB03E9DA
:10E928000300EB6898476B6804469847BDF80430C5
:10E93800009A1B1B99B21BB2002BA2EB0002BEBFB0
:10E9480001F57A7302F1FF321BB24FF47A7000FBC3
:10E95800023003B030BD00BF90F000082DE9F0414F
:10E968004FF47A75B1FBF5F5C5EB4513DFF83C803C
:10E9780005EB8303A1EBC3039CB2D8F80C30064621
:10E988009847D8F8043007469847E3199AB21BB25B
:10E99800B3F57A7F0544A2BFA2F57A7301351BB29D
:10E9A8003560B3803046BDE8F08100BF90F00008C4
:10E9B800024B00221A60024B1B68184710160020F1
:10E9C800A4F00008F8B50446174608461E467CB170
:10E9D80073B1084B00255B6A25609847069B606009
:10E9E8002581A572E6602361E77265612846F8BD56
:10E9F8000120FCE7A4F0000810B5034CE369984730
:10EA0800A36ABDE810401847A4F0000870B5064D89
:10EA1800EB69064698476B6A044630469847AB6AE6
:10EA2800201ABDE870401847A4F00008054A0346BC
:10EA3800106800B97047984201D04069F9E7012091
:10EA4800704700BF101600202DE9F3410B4E336AC2
:10EA5800044698470123B7692372D4F80080054615
:10EA6800B8472844804502D2B84705442560B368B2
:10EA78002068019302B0BDE8F0411847A4F00008EF
:10EA880070B520B3EFF3108672B6124D2B680122D1
:10EA9800827253B10022984242720FD144690272C5
:10EAA8003CB120462C60FFF7CFFF86F3108800208A
:10EAB80070BD094BDB6898472C60F6E71A465B691E
:10EAC800002BF2D09842F9D143695361EDE7012058
:10EAD800EEE700BF10160020A4F00008094B10B59F
:10EAE8001B685A69596911B95861416108E004689D
:10EAF80011688C4202D913465269F3E758614261A2
:10EB080010BD00BF10160020044A13680BB1002185
:10EB1800197243611060FFF797BF00BF10160020FD
:10EB28002DE9F041044600282DD0FFF77FFF50BBA8
:10EB3800657A45BBEFF3108872B6144E6768336A7E
:10EB4800984787422CBF27602060114FA5724FF469
:10EB5800807323813B684BB9336998472046FFF798
:10EB6800D3FF88F310882846BDE8F081B369984739
:10EB7800236818443B6820601B6898422046EED3FF
:10EB8800FFF7ACFFEDE70125EDE700BFA4F00008B3
:10EB98001016002010B5044608467CB1084B5B6A85
:10EBA800984760602046FFF741FF40B12046FFF7D5
:10EBB80067FF2046BDE81040FFF7B2BF012010BD37
:10EBC800A4F000082DE9F041EFF3108772B61D4E4E
:10EBD8001D4D736998473369044698472B684BB9AC
:10EBE8004FF000082B688BB9286828BB87F310887A
:10EBF800BDE8F081011B241A1A688A428CBF1219D9
:10EC080000221A605B69002BF6D1E9E71C681CB189
:10EC1800B36998478442E7D22C6863692B60A4F8EB
:10EC28000880D4E9033098476389B3F5807FD9D148
:10EC38002046FFF775FFD5E7037A002BD6D1FFF7FB
:10EC480003FFD3E7A4F00008101600202DE9F04FC9
:10EC580097B000298046039140F307819A460446FD
:10EC680003991378A4EB0800013923B90023237012
:10EC780017B0BDE8F08F8842F8DA252B04D004F8E5
:10EC8800013B1646721CEBE792F801E0AEF1300347
:10EC9800D3F1000C4CEB030CAEF13003092B02F15D
:10ECA800010628D8324600254FF00A09164612F800
:10ECB800013BA3F13000092819D93378692B00F0FA
:10ECC80099801BD8632B27D0642B00F09380582B96
:10ECD80058D0252B18D13378002B00F08F8004F8FA
:10ECE800013BA4EB08038B4280F28680CAE709FB4C
:10ECF8000535303DDAE74FF0FF35DEE7752B7BD081
:10ED0800782B41D0732B1ED0252304F8013BA4EBAC
:10ED180008038B4270DADEE7002D05F1FF39D8BF12
:10ED28004FF000094A462046202100F0CBF8534610
:10ED3800A144002D53F8042B89F80020D8BF0125E1
:10ED48002C449A469EE74A4B5AF8047B002F08BF8A
:10ED58001F463846F1F70CFAA5EB000B8542B8BF01
:10ED68004FF0000B81465A462046202100F0AAF8B1
:10ED78005C4400234B4501DB4C4483E7FA5CE254D6
:10ED88000133F7E74CF0400C1020DFF8E8903A4FD9
:10ED98001CF0400F08BF4F465346BEF1300F019795
:10EDA800A4EB08020CBF302720271CF0020FA1EBB0
:10EDB8000202029753F8041B22D0002920DA4942A4
:10EDC800013D4FF02D0C05AF009700278946DDF86F
:10EDD80004A0B1FBF0F100FB119B48451AF80BB0F9
:10EDE800DDF800A00AF801BB07F10107CDF800A083
:10EDF800ECD90EE04CF0020C0A20C6E7013E70E7A1
:10EE080011B14FF0000CDEE730208DF814008C466D
:10EE18000127BEF1300FA5EB070504D02020002DF7
:10EE280005F1FF3508DCBCF1000F03D0013A04F806
:10EE380001CB86D025440AE0013A04F8010BEED153
:10EE48007FE7029904F8011B013A3FF47AAF291BC6
:10EE58000029F6DC05A92244013FFFF472AF785C73
:10EE680004F8010B9442F7D16BE7002000E700BFDC
:10EE780004FE000830FE00080BFE000870B50D4DBA
:10EE88000D4C641BA4100026A64209D10B4D0C4C56
:10EE980000F0A2F8641BA4100026A64205D170BD9C
:10EEA80055F8043B98470136EEE755F8043B984778
:10EEB8000136F2E760FE000860FE000860FE000808
:10EEC80064FE000802440346934200D1704703F8E9
:10EED800011BF9E7000000002DE9F843C1F30A58C7
:10EEE800A8F2FF36132E02460B4607460C46054687
:10EEF80033DC002E14DA34A3D3E90023F1F746F902
:10EF080000220023F1F776FB38B1002C58DA24F000
:10EF180000431D4301D02E4C002523462F4625E0F3
:10EF28002C4A42FA06F801EA080202431ED026A338
:10EF3800D3E90023F1F72AF900220023F1F75AFB5D
:10EF48000028EAD0002CBEBF4FF4801343FA06F61F
:10EF5800A41924EA08040025DFE7332E0ADDB6F5F4
:10EF6800806F03D1F1F712F907460B463846194668
:10EF7800BDE8F883A8F213484FF0FF3222FA08F8E8
:10EF880018EA000FF2D010A3D3E90023F1F7FEF836
:10EF980000220023F1F72EFB0028BED0002C02DA55
:10EFA800142E03D1013425EA0805B6E70123C6F17A
:10EFB800340603FA06F63544BD4238BFE418F2E7D2
:10EFC80000252C46A9E700BF9C7500883CE4377EE5
:10EFD8000000F0BFFFFF0F00F8B500BFF8BC08BC89
:10EFE8009E467047F8B500BFF8BC08BC9E467047FF
:10EFF8000000000001000000020000000000000006
:10F008008813000010270000204E00003075000013
:10F01800409C000050C3000060EA0000C0D401001A
:10F0280080A903000053070000EA0637000000002B
:10F038005000000040F709370000000050000000B1
:10F04800C194C10000000000B227000000000000C9
:10F0580000000000000000000000000000000000A8
:10F0680000000000331500082115000805150008E8
:10F0780025150008011500084515000825647325A5
:10F088003033643A0000000009190008A919000883
:10F0980019190008B519000879190008C1190008DC
:10F0A8000000000029190008E1180008AD18000840
:10F0B80065180008BD180008D11800087118000864
:10F0C8007518000889180008291C0008511C000838
:10F0D800D51B0008C11B0008537769746368207446
:10F0E8006F20436C61737320256320646F6E650D18
:10F0F8000A00414243004C6D48616E646C657220A1
:10F1080053746F70206F6E20676F696E67202E2EA4
:10F118002E0D0A004C6D48616E646C657220537444
:10F128006F707065640D0A004C6D48616E646C65A3
:10F13800722073776974636820746F20414250208D
:10F148006D6F64650D0A00564444413A2025640DEC
:10F158000A0074656D703A2025640D0A0053454E07
:10F168004420524551554553540D0A004E65787454
:10F1780020547820696E20203A207E25642073650B
:10F18800636F6E642873290D0A000D0A2323232355
:10F19800232320424541434F4E204C4F53540D0AE0
:10F1A800000D0A23232323232320424541434F4EA6
:10F1B800205245434549564544207C2044523A252F
:10F1C80064207C20525353493A2564207C20534EB6
:10F1D800523A2564207C2046513A2564207C2054EC
:10F1E800494D453A2564207C20444553433A2564DB
:10F1F800207C20494E464F3A303258253032582527
:10F20800303258202530325825303258253032587F
:10F218000D0A000D0A2323232323232042454143BB
:10F228004F4E204E4F542052454345495645440DB4
:10F238000A004E564D20444154412053544F5245E4
:10F24800440D0A004E564D20444154412052455326
:10F25800544F5245440D0A004E41434B000D0A23BA
:10F268002323232323203D3D3D3D3D3D3D3D3D3D65
:10F27800204D4350532D436F6E6669726D203D3D9E
:10F288003D3D3D3D3D3D3D3D3D3D3D0D0A0023237A
:10F298002323232320552F4C204652414D453A2500
:10F2A800303464207C20504F52543A2564207C200E
:10F2B80044523A2564207C205057523A2564002055
:10F2C8007C204D534720545950453A00434F4E46F1
:10F2D80049524D4544205B25735D0D0A00554E4348
:10F2E8004F4E4649524D45440D0A000D0A2323232B
:10F2F800232323203D204A4F494E4544203D2000EA
:10F30800414250203D3D3D3D3D3D3D3D3D3D3D3D26
:10F318003D3D3D3D3D3D3D3D3D3D0D0A004F544188
:10F3280041203D3D3D3D3D3D3D3D3D3D3D3D3D3D1E
:10F338003D3D3D3D3D3D3D0D0A000D0A2323232360
:10F348002323203D204A4F494E204641494C4544FD
:10F358000D0A004C4544204F46460D0A004C4544D2
:10F36800204F4E0D0A0023232323232320442F4C10
:10F37800204652414D453A25303464207C20504F78
:10F3880052543A2564207C2044523A2564207C203B
:10F39800534C4F543A2573207C20525353493A25F5
:10F3A80064207C20534E523A25640D0A004E564D77
:10F3B800204441544120555020544F204441544545
:10F3C8000D0A004E564D20444154412053544F528B
:10F3D80045204641494C45440D0A004150504C498E
:10F3E800434154494F4E5F56455253494F4E3A2078
:10F3F8005625582E25582E25580D0A004D575F4C76
:10F408004F524157414E5F56455253494F4E3A204D
:10F41800205625582E25582E25580D0A004D575F81
:10F42800524144494F5F56455253494F4E3A202066
:10F4380020205625582E25582E25580D0A004C32C6
:10F448005F535045435F56455253494F4E3A20202B
:10F458002020205625582E25582E25580D0A0052B2
:10F46800505F535045435F56455253494F4E3A20DB
:10F47800202020205625582D25582E25582E255831
:10F488000D0A0031003200435F4D4300505F4D4389
:10F49800000000008BF400088DF40008FCF0000860
:10F4A8008FF4000888F7000894F4000801000000B1
:10F4B800030000000500000001000000010000003A
:10F4C800060000000A000000200000000200000002
:10F4D80004000000080000001000000040000000C8
:10F4E8008000000000010000000200000000000091
:10F4F8000000000000000000000000000100000003
:10F50800020000000300000004000000A0860100C3
:10F51800400D0300801A060000350C0040420F0021
:10F5280080841E0000093D0000127A000024F400C7
:10F5380000366E010048E801006CDC0200000000A3
:10F5480000000000000000000000000004020800A5
:10F558001010100410101002101010080100020002
:10F568000400060008000A000C00100020004000FB
:10F5780080000001080402040801010101010103DF
:10F58800070100006572726F723A20526567696FF1
:10F598006E206973206E6F7420646566696E656499
:10F5A80020696E20746865204D573A207365742071
:10F5B8006C6F726177616E5F636F6E662E68206133
:10F5C80063636F7264696E676C790D0A0023232385
:10F5D80023232320446576416464723A2020202046
:10F5E80020253032583A253032583A253032583AA8
:10F5F800253032580D0A004D414320727854696D08
:10F60800654F75740D0A004D414320747854696D37
:10F61800654F75740D0A004D4143207278446F6E32
:10F62800650D0A004D4143207478446F6E650D0ADC
:10F6380000080A0C0D0E10121415181A1B1D1E2195
:10F648002403050205010602020500000600000168
:10F658000504040048E8010048E8010048E8010002
:10F6680048E8010048E8010048E8010090D003009C
:10F6780000000000030000000201000C0B0A09084A
:10F68800070732000000000000010201000000002E
:10F69800000203020100000000030403020100004D
:10F6A8000004050403020100000506050403020125
:10F6B80000060706050403020107070706050403F9
:10F6C8000207070202020202020202020202020208
:10F6D80002020302020202020203040302020202FD
:10F6E80002040504030202020205060504030202DD
:10F6F80002060706050403020207070706050403B6
:10F7080002070733337373F2F2F2F200000B357D10
:10F71800F2F2F233337373DEDEDEDE52585F2573A6
:10F72800206F6E206672657120256420487A2061FA
:10F73800742044522025640D0A005258206F6E2010
:10F748006672657120256420487A206174204452CD
:10F758002025640D0A005458206F6E20667265716A
:10F7680020256420487A2061742044522025640DA5
:10F778000A004D756C74695F43004D756C74695F60
:10F78800500000008BF400088DF40008FCF000081D
:10F798007AF7000888F7000882F70008C6F8EEF63E
:10F7A800FFD6DE916002CE56E7B54DEC8F1F89FA81
:10F7B800EFB28EFB41B35F452353E49B75E13D4CAB
:10F7C8006C7EF5836851D1F9E2AB622A0895469DB3
:10F7D80030370A2F0E241BDFCD4E7FEA121D583416
:10F7E80036DCB45BA476B77D52DD5E13A6B900C1E2
:10F7F80040E379B6D48D67729498B085BBC54FED58
:10F80800869A66118AE904FEA078254BA25D8005D8
:10F818003F2170F16377AF4220E5FDBF811826C311
:10F82800BE35882E9355FC7AC8BA32E6C0199EA315
:10F8380044543B0B8CC76B28A7BC16ADDB6474140F
:10F84800920C48B89FBD43C43931D3F2D58B6EDAD8
:10F8580001B19C49D8ACF3CFCAF447106FF04A5CA9
:10F8680038577397CBA1E83E96610D0FE07C71CCB9
:10F878009006F71CC26AAE6917993A27D9EB2B2272
:10F88800D2A907332D3C15C987AA50A50359091ACF
:10F8980065D784D082295A1E7BA86D2CA584998DA2
:10F8A8000DBDB1545003A97D1962E69A459D408764
:10F8B80015EBC90BEC67FDEABFF7965BC21CAE6A95
:10F8C8005A41024F5CF434089373533F0C52655EFF
:10F8D80028A10FB509369B3D2669CD9F1B9E742E26
:10F8E8002DB2EEFBF64D61CE7B3E7197F568002C8C
:10F8F800601FC8EDBE46D94BDED4E84A6B2AE51630
:10F90800C5D75594CF100681F044BAE3F3FEC08AF8
:10F91800ADBC4804DFC17563301A0E6D4C14352F29
:10F92800E1A2CC3957F28247ACE72B95A098D17F5A
:10F93800667EAB83CA29D33C79E21D763B564E1EC0
:10F94800DB0A6CE45D6EEFA6A8A4378B324359B787
:10F958008C64D2E0B4FA0725AF8EE918D5886F72A7
:10F9680024F1C751237C9C21DDDC86859042C4AA02
:10F97800D8050112A35FF9D0915827B93813B333CA
:10F98800BB7089A7B622922049FF787A8FF8801732
:10F99800DA31C6B8C3B07711CBFCD63A637C777B33
:10F9A800F26B6FC53001672BFED7AB76CA82C97D73
:10F9B800FA5947F0ADD4A2AF9CA472C0B7FD932604
:10F9C800363FF7CC34A5E5F171D8311504C723C308
:10F9D8001896059A071280E2EB27B27509832C1A4C
:10F9E8001B6E5AA0523BD6B329E32F8453D100EDA6
:10F9F80020FCB15B6ACBBE394A4C58CFD0EFAAFB8A
:10FA0800434D338545F9027F503C9FA851A3408F51
:10FA1800929D38F5BCB6DA2110FFF3D2CD0C13EC69
:10FA28005F974417C4A77E3D645D197360814FDCFE
:10FA3800222A908846EEB814DE5E0BDBE0323A0AE2
:10FA48004906245CC2D3AC629195E479E7C8376D66
:10FA58008DD54EA96C56F4EA657AAE08BA78252E8B
:10FA68001CA6B4C6E8DD741F4BBD8B8A703EB56614
:10FA78004803F60E613557B986C11D9EE1F8981105
:10FA880069D98E949B1E87E9CE5528DF8CA1890DF4
:10FA9800BFE6426841992D0FB054BB162323232398
:10FAA8002323204170704B65793A202020202020A4
:10FAB80000232323232323204E776B4B65793A2099
:10FAC800202020202000232323232323204170707B
:10FAD800534B65793A202020202000232323232319
:10FAE80023204E776B534B65793A20202020200045
:10FAF800232323232323204D43526F6F744B6579AF
:10FB08003A20202000232323232323204D434B4541
:10FB18004B65793A202020202000253032583A259C
:10FB28003032583A253032583A253032583A253052
:10FB380032583A253032583A253032583A25303240
:10FB4800583A253032583A253032583A253032580A
:10FB58003A253032583A253032583A253032583A18
:10FB6800253032583A253032580D0A0023232323F2
:10FB78002323204F544141202323232323230D0AE9
:10FB880000232323232323204142502020232323FF
:10FB98002323230D0A0023232323232320494473EB
:10FBA80020202323232323230D0A00232323232375
:10FBB80023204465764575693A2020202020202599
:10FBC8003032583A253032583A253032583A2530B2
:10FBD80032583A253032583A253032583A253032A0
:10FBE800583A253032580D0A002323232323232093
:10FBF8004170704575693A20202020202025303238
:10FC0800583A253032583A253032583A2530325849
:10FC18003A253032583A253032583A253032583A57
:10FC2800253032580D0A00526164696F53656E645D
:10FC3800204F76657273697A650D0A004952515FE3
:10FC480052585F54585F54494D454F55540D0A005A
:10FC5800505245204F4B0D0A0053594E43204F4BED
:10FC68000D0A00484452204F4B0D0A0048445220C8
:10FC78004B4F0D0A004952515F4352435F45525260
:10FC88004F520D0A00040506841E0000093D0000BD
:10FC9800127A000024F4000048E8010090D0030024
:10FCA80020A1070000000000B128000061510000F9
:10FCB800C3A2000002010003C9C6000899C50008D4
:10FCC800C5C7000809C60008DDD00008B1C600088D
:10FCD80015CE000899CC000891C400081DD300086F
:10FCE80059D100089DC6000891C5000835C600080E
:10FCF8000DC60008D1C50008C7C50008D9C400084A
:10FD0800D5C40008C3C50008BFC500085DC7000802
:10FD180089C70008B5C5000839D4000829C50008F6
:10FD2800F1C4000809D40008DDC400088DCA000821
:10FD380011C8000899E200089FE20008C0120000FC
:10FD48001F000000A816000017000000841C000017
:10FD58000F000000E42500001E000000B42D000084
:10FD680016000000083900000E0000002C4C0000AE
:10FD78001D000000685B00001500000074720000A0
:10FD88000D000000589800001C00000034B7000067
:10FD980014000000E8E400000C00000078310100C5
:10FDA8001B000000686E01001300000034CA010047
:10FDB8000B000000286202001A00000040DB02006D
:10FDC800120000003C9303000A000000C0C20400B7
:10FDD8001900000060B3050011000000382007007A
:10FDE8000900000020A1070000000000040302022F
:10FDF8000101010100000000000000003C4E554CCC
:10FE08004C3E00303132333435363738394142438D
:10FE18004445464748494A4B4C4D4E4F5051525322
:10FE28005455565758595A003031323334353637CD
:10FE380038396162636465666768696A6B6C6D6EA0
:10FE48006F707172737475767778797A0000000034
:08FE5800800DFF7F0100000096
:08FE60005D0100080000000034
:08FE6800390100080000000050
:10FE70000200000000000000DD020020A5160008BE
:10FE8000D5160008ED16000855170008051E0008D5
:10FE900015230008691D0008D1200008000000009B
:10FEA000D521000821210008352200082D1D000859
:10FEB0005520000800000000711D0008151D0008F5
:10FEC000211D0008ED2000080000010000000000D6
:10FED0000000000004000000401F00001027000088
:10FEE00000093D00100000000000000000000000BC
:10FEF0000000000000000000000000000A000001F7
:10FF00007800002000FF00000000000078000020C2
:10FF10000000000000000000FF00000000000000E2
:10FF20007800002000000000000000000000000039
:10FF30000000000000000000E0000000256A00084A
:10FF40005969000865690008896900080000000017
:10FF5000000000007D6A000871690008E56D000876
:10FF60000000000000000000000000000000000091
:10FF7000008182800103028401000000FF00000074
:08FF8000FFFFFFFFFFFFFFFF81
:020000040803EF
:10E500000080E1010101010101010101010101019D
:10E51000002B7E151628AED2A6ABF7158809CF4F73
:10E520003C012B7E151628AED2A6ABF7158809CF75
:10E530004F3C022B7E151628AED2A6ABF7158809E4
:10E54000CF4F3C032B7E151628AED2A6ABF715880D
:10E5500009CF4F3C04000000000000000000000054
:10E5600000000000007F000000000000000000002C
:10E57000000000000000800000000000000000001B
:10E58000000000000000008100000000000000000A
:10E5900000000000000000008200000000000000F9
:10E5A00000000000000000000083000000000000E8
:10E5B000000000000000000000000000000000005B
:040000050800265574
:00000001FF
